:020000040800F2
:1000000000800020156700080D740008F1660008E4
:100010000F74000811740008137400080000000039
:1000200000000000000000000000000091C3000874
:10003000157400080000000021C4000865C4000811
:1000400017740008197400081B7400081D74000858
:100050001F74000821740008A1730008A77300082A
:10006000AD730008B3730008B97300082374000867
:100070002574000827740008297400082B740008F0
:100080002D7400082F7400083174000833740008C0
:10009000357400083774000839740008BF7300080D
:1000A0003B7400083D7400083F7400084174000868
:1000B0004374000845740008477400084974000838
:1000C0004B7400084D7400084F7400085174000808
:1000D00053740008117B0008A17F000855740008C4
:1000E000E37300088D740008577400085974000801
:1000F0005B74000800000000000000000000000029
:1001000000000000000000005FF808F110B5054C89
:10011000237833B9044B13B10448AFF300800123B3
:10012000237010BD78070020000000001CEF0108BC
:1001300008B5034B1BB103490348AFF3008008BD6A
:10014000000000007C0700201CEF01087047000041
:100150008168014809F0D4BF42B2010838B50446AD
:1001600081680D4809F0CCFF20690C4D036800211F
:100170001B68984701222846032106F08BFF20695F
:10018000002103685B6898472846BDE83840012293
:10019000022106F07FBF00BF28B201080000024024
:1001A0000B4B13B51A68B2F5007F04D21A68511CC4
:1001B0001960084B9854084B1C680DF049FC00234B
:1001C00002460093072120460EF026FB02B010BD28
:1001D00094090020940700209809002010B50446D7
:1001E0003C2115F089FF204610BD000070B5154C6C
:1001F0002368092B1FD92268134D023A2946134858
:1002000015F0A3FE06462068023828440AF075F867
:100210008642014610D10E4E30680CF0D3FF2268A2
:100220000023294630680DF019F810B9094809F083
:1002300067FF0023236070BD3246074809F060FF66
:10024000F7E700BF94090020940700200400002075
:100250009C090020ECB1010800B2010870B5044609
:100260002048214E60602148C4E90312A060204864
:1002700086B020606361194604F1180004F1280576
:1002800005F0FEFF0FCE0FC5336801222B60002161
:100290004FF400700CF054FF164B186018B94A2147
:1002A000154806F093F9154B0A21009300231448D2
:1002B0001A460EF08FFA134B41F221011860012308
:1002C000CDE900334FF6FF7303A81A4615F0EAFD97
:1002D0000D4A03AB03CB106020461B88516013818D
:1002E00006B070BD7BB20108D8B1010885B2010823
:1002F000A0B201089C09002085E50108ED01000875
:100300008BB2010898090020040000200148006811
:100310000DF036B89C09002010B50446C0680749A6
:1003200003685B699847E06804F1280103681B686B
:1003300098470022024B1A6010BD00BFA1010008BF
:1003400094090020C06810B50368084C5B689847A2
:1003500001220221204606F09DFE012203212046B3
:1003600006F098FE0022024B1A6010BD0000024009
:100370009409002081F001021830082106F043B8EA
:1003800081F001021830022106F03DB881F001022F
:100390001830042106F037B881F00102183001212D
:1003A00006F031B810B5044681680F4809F0A8FE80
:1003B00004F1180006F014F8002184F82400204607
:1003C000FFF7E4FF20460021FFF7DAFF2046002177
:1003D000FFF7D0FF20460121FFF7DEFF2046BDE8F2
:1003E00010400021FFF7D8BF1EB2010810B5044627
:1003F00081681A4809F084FEA168194809F080FE56
:1004000020460121FFF7C8FF01212046FFF7B8FF72
:100410004FF496700DF06EFC20460021FFF7B0FF00
:1004200001212046FFF7B2FF4FF496700DF062FCF9
:1004300020460021FFF7AAFF01212046FFF79AFF7F
:100440004FF496700DF056FC20460021FFF792FF06
:100450002046BDE810400021FFF79EBF51B20108C1
:1004600061B2010807F08CBE10B50446406C10B1B3
:10047000042115F041FE204610BD000070B5164E57
:10048000164D346814F001041CD128461A22214666
:1004900040F8044B18F0B9F91A22214605F124005E
:1004A0002C6218F0B2F901230D4A0E492846C5E91D
:1004B0001044C5E9124485F8504085F85140336036
:1004C00016F066FC95F851301BB11D21064806F068
:1004D0007DF8024870BD00BFA0090020A4090020DB
:1004E000000000206904000885E5010810B50446F5
:1004F000C06910B1012115F0FFFD206910B1012183
:1005000015F0FAFD204610BDF8B50025C0E901122E
:100510000570C0E90335C0E90555C0E907554562D6
:1005200006990446164600F11C0713F035FD38B94C
:100530003146074809F0E4FD2021064806F046F858
:10054000069A3946204613F0EFFC2046F8BD00BF5E
:1005500089B4010885E5010830B58DB014F006FEB8
:10056000044603F0ADF9214603F0A6FC294B2A4AC4
:1005700000930321294B02A8FFF7C6FF02A92046DA
:1005800014F09AFE02A8FFF7B1FF254B254A00930D
:100590000321254B02A8FFF7B7FF02A9204614F05C
:1005A0008BFE02A8FFF7A2FF0222002303921F4D39
:1005B0001F4A012102A88DF808300495CDE90523D2
:1005C000CDE90733CDE909330B9313F001FC38B9BA
:1005D0002946184809F094FD2021174805F0F6FF38
:1005E000012209A902A813F0DDFB02A9204614F09C
:1005F00063FE02A8FFF77AFF104B114A114920460B
:1006000014F01CFD00F05CFA0522214603F068FCA2
:100610000DB030BDE2B20108F0B20108B8B2010875
:1006200056B301084DB30108F9B2010880B30108BF
:100630008EB3010889B4010885E501086504000846
:10064000B1B30108D5B301082DE9F843D0E900346E
:10065000E41AA410B4F5705F06460F46914602D125
:10066000244815F00BFD002C14BF22460122A418CB
:10067000A1EB03081AD2B4F5705F17D8CCB1A00073
:1006800009F0DAFD054615EB080F18BFD9F8003060
:10069000306818BF45F808302A4603469F420AD002
:1006A0000AB11968116004320433F7E74FF470544B
:1006B000E5E72546E7E73B1A043303EB050EBC46A6
:1006C00072467168614507D012B1DCF800301360E2
:1006D00004320CF1040CF5E7CF1B774410B1042170
:1006E00015F00AFD05EB8404C6E90057B460BDE8C7
:1006F000F88300BFB4B401082DE9F04790B014F0BE
:1007000035FD0646FFF7BAFE0025044610AF304619
:1007100007F8215D14F0DAF8304605F09BFB231D45
:1007200000933A4623463E49304614F0E1FB3D48EB
:1007300010AA206242F8205D04F1240109F0C6FAF3
:10074000089B1BB18521384805F040FF37493046EA
:1007500014F075FB0546DFF8E890DFF8E8A02064A8
:1007600004F14408ADB10EAB03930DAB02930CAB97
:1007700001930BAB009309AA0AAB4946284618F02F
:10078000BDFF06281FD02A4809F0BAFC01238DF8C6
:100790001F30012302222749CDE90032304604F1FF
:1007A00050033A4614F064FB9DF81F302BB12248E9
:1007B00009F0A6FC102007F0DEFC012384F851307C
:1007C00010B0BDE8F0870D2017F0BCFF0F9008B9FE
:1007D0001A48D9E70E9B0D2104930D9B52460393B3
:1007E0000C9B02930B9B01930A9B0093099B18F0AF
:1007F00031FFD4E9121399420CD009B10F9B0B6061
:100800000431A1642C21284618F0E7FF0028C0D04D
:10081000451CA7E70FAA4046FFF716FFF2E700BF07
:10082000F0B20108DBB3010885E501084DB301080A
:10083000F9B3010880B3010876B4010849B401088E
:10084000E7B301085DB4010810B9034809F058BCCA
:1008500003C809F0BBBC00BFADB8010810B92648F9
:1008600009F04EBC0178406801F07002402A01F0A6
:100870000F030ED004D8A2B10268204809F040BC92
:10088000502A20D0602AF7D1012B0CD101781C48C6
:1008900005E01C491C4B002818BF19461B4809F0ED
:1008A0002FBCFFF7D1BF022B02D101881848F6E711
:1008B000042B02D101881748F1E7082B01680CBF0F
:1008C00015481648EBE7012B03D190F900101448A6
:1008D000E5E7022B03D1B0F900101248DFE7042B43
:1008E00003D1B0F900101048D9E7082B01680CBFFC
:1008F0000E480F48D3E700BF10B8010891B80108AF
:1009000016B801080AB8010805B80108F1B40108D1
:1009100022B801082FB801083CB801084AB80108FC
:1009200056B8010861B801086DB8010879B8010826
:1009300086B8010870B50020002105F065FA04466C
:100940000F4D104EC4B16179802911D122792168EF
:10095000306813F049FF204605F08CFB2046082143
:1009600015F0CAFB0020002105F04EFA0446E9E725
:10097000284609F0C5FBEEE7034B187870BD00BFB1
:1009800033B70108640E00201C0F002008B502F0E8
:1009900097FFBDE8084002F0DBBF1FB56123CDE93A
:1009A000013101A9039204F06BF905B05DF804FB75
:1009B00007B58DF8041001A98DF805208DF80630D3
:1009C00004F01CFA03B05DF804FB000070B5124E91
:1009D000346814F001041DD1104D1A222846214616
:1009E00040F8044B17F011FF1A22214605F12400AC
:1009F0002C6217F00AFF0123094A0A492846C5E973
:100A00001044C5E9124485F8504085F851403360E0
:100A100016F0BEF9014870BDA0090020A40900200D
:100A2000000000206904000808B5FFF7CFFF90F828
:100A300051301BB93321034805F0C8FDFFF7C6FF4D
:100A400008BD00BF85E5010870B5154C154809F0D3
:100A500057FB2368DB0708D414F0A2FB8022014671
:100A6000114813F0F5FB012323600F4A0F4B104D83
:100A70001A600CF0E7FF0F4B18600F4809F040FBBD
:100A8000FFF7D2FFD0E91146A64205D054F8041B67
:100A9000284609F035FBF7E7084B187870BD00BF12
:100AA000FC090020CEB401085C0D0020640E00207B
:100AB000EFB40108180D0020E1B40108200F002058
:100AC00002F0FEBE10B50C4C02F0FAFE2368DB0704
:100AD0000FD400F1580300F1440200F14801074827
:100AE000FFF7BCFB0123064A06490448236016F0C1
:100AF0004FF9024810BD00BFF8090020200D00206A
:100B0000000000204D0100082DE9F047FFF7DAFF53
:100B100004460121FFF740FC2046FFF7FDFB0CF0E7
:100B200091FF4EF65F273C4E4FF4407233683B49CD
:100B3000C01AB8424FF47A73394D204642D8FFF7B5
:100B4000E5FBDFF8ECA0DFF8D4902860D5F8008052
:100B5000B8F1000F1DD10CF075FF3368C01AB84210
:100B600017D8504609F0CCFA01212046FFF708FCBF
:100B7000C8200DF0BFF841462046FFF701FC4FF4B6
:100B80007A734FF4407249462046FFF7BFFB286056
:100B9000DCE72046FFF7D6FB2B68002B39D001217C
:100BA0002046FFF7F3FB1F4809F0AAFA41F288300C
:100BB0000DF0A0F800212046FFF7E8FB1A4B18784B
:100BC000BDE8F087FFF7A2FB0526DFF86490DFF8A9
:100BD0004C8028602F68002FDED1013E16F0FF0602
:100BE000DAD0484609F08CFA01212046FFF7C8FB0D
:100BF000C8200DF07FF839462046FFF7C1FB4FF4BF
:100C00007A734FF4407241462046FFF77FFB28601D
:100C1000E0E7064BD3E700BF180D0020040A0020D0
:100C2000140D0020F5B70108200F00201E0F002032
:100C3000CDB701082DE9F041444809F061FAFFF70A
:100C400041FF04460121FFF7A7FB2046FFF764FBA5
:100C500041F288334FF440723D492046FFF756FB7E
:100C60003C4D28602046FFF76DFB2E68002E42D1D8
:100C7000394809F045FA01212046FFF781FB4FF47E
:100C80007A700DF037F831462046FFF779FB314690
:100C90002046FFF781FB314B1E70314809F030FAD6
:100CA000304D94F82420304F2C4E304B002A14BF86
:100CB0003A462A462E492F4809F022FA32782B4B21
:100CC000002A14BF3A462A462B492A4809F018FA46
:100CD0002A4B94F824102A48002914BF19462946A3
:100CE00009F00EFA274809F00BFA33785BB3264B6C
:100CF0001878BDE8F081254809F002FA0026DFF8EF
:100D00005080234F2B689E4206D218F806103846B2
:100D100009F0F6F90136F5E71E4809F0F1F901216D
:100D20002046FFF733FB4FF47A700CF0E3FF00210D
:100D30002046FFF72BFB00212046FFF72DFB012269
:100D4000064B1A70A9E7144BD2E700BF56B701084B
:100D5000040A0020140D0020CDB70108680E002001
:100D60007DB701084EB7010849B7010885E50108BC
:100D700047BD01088DB70108A4B7010853B70108A2
:100D8000AAB70108BFB70108200F00206AB7010801
:100D90000EDB010884E501081E0F0020F8B530487D
:100DA00009F0AEF9FFF78EFE01210446FFF7F4FAD1
:100DB0002C4B1A786AB10025012120461D70FFF7DF
:100DC000D9FA41F288300CF095FF29462046FFF70A
:100DD000D1FA02F075FD036E60301B689847224B14
:100DE000224DC3E900012046FFF796FA41F288330D
:100DF0004FF440721E492046FFF788FA28602046CB
:100E0000FFF7A0FA2E681B4FA6B91B4809F078F926
:100E100001212046FFF7B4FA4FF496700CF06AFFF8
:100E200031462046FFF7ACFA31462046FFF7B4FAC8
:100E30003878F8BD01212046FFF7A8FA4FF49670E4
:100E40000CF058FF20460021FFF7A0FA20460021B1
:100E5000FFF7A2FA2A680649084809F0C7F9E7E748
:100E600056B701081800002028020020140D0020A9
:100E7000040A00201C0F0020CDB701086AB7010842
:100E80002DE9F04F8BB0FFF7CFFD00240190FFF765
:100E900019FEA54BA54F1B688046102BC7F8F441DF
:100EA000C7F8F841C7F8FC41C7F800421CD82146F2
:100EB0009F4815F0C3F801214046FFF76DFA012164
:100EC0004046FFF75DFA4FF496700CF013FF214691
:100ED0004046FFF755FA40460021FFF75DFA954B73
:100EE00018780BB0BDE8F08FCDE907443C46924A34
:100EF000103B05920693DDE906329A4220D205A8FE
:100F000001F041FF20B9012105A801F044FFF2E7FB
:100F100005A801F069FC064605A801F029FF38B3D1
:100F2000DDE906320899854809F0EAF8844809F0B5
:100F3000E7F8DDE906130598C91A184409F046F9DF
:100F4000D7F8F421D7F8F8117E4809F0D9F84046CF
:100F50000121FFF721FA01214046FFF717FA4FF46C
:100F600096700CF0C7FE00214046FFF70FFAB2E77B
:100F7000754809F0C5F873687448197809F0C0F825
:100F8000B3687348197809F0BBF833697148198858
:100F900009F0B6F8704809F0B3F83068FFF754FC70
:100FA000F3686E481B68196809F0AAF8F3681B68B3
:100FB0001A6840F201739A4243D1694809F0A0F8D7
:100FC000F368DFF8C4915B68DFF8C0A11D69DFF842
:100FD000C0B1002D35D02B682BB1484609F090F8F0
:100FE0002868FFF731FC6B682BB15A6819781278C2
:100FF000504609F085F8AB6813B1584609F080F8FF
:10100000EB6823B11A785748114609F079F82B6933
:1010100023B193F90010544809F072F86B6933B1A9
:101020005248197809F06CF86869FFF717FCAB694A
:101030002BB14F4809F064F8A869FFF705FCED698A
:10104000C7E7F3681A68116840F20172914240F0F4
:10105000D2805B680293019B9B6C0393019BD3F846
:1010600044A0039A5346524500F0C580186801F029
:10107000E0FC81463F4809F043F84846FFF7E4FBAF
:10108000029B0AF1040AD3F810B0BBF1000F00F084
:10109000B680DBF8003073B9B9F1000F1AD13648C9
:1010A00009F02EF8DBF81400FFF7D8FBDBF814305A
:1010B0009BB91D461EE0B9F1000F0BD05A68D9F854
:1010C00004108A4206D1D9F80010186817F06AFB9C
:1010D0000028E4D0DBF81CB0D7E71D7815F07002CB
:1010E00004D0402A14D005F00F0503E05A68556873
:1010F000F72D06D8DBF800004268062A0AD01F4800
:1011000000E01F4808F0FCFF484601F045FCA8E756
:101110000125EFE7D4F8F42105F10801C2F5FA7CC6
:10112000614537D91748EDE7140D00202000002055
:10113000040D00201C0F00200C0A0020F5B401084B
:1011400012B501085CB601081FB501082DB50108EC
:101150003EB5010852B501085FB5010872B5010836
:1011600084B50108CAB50108DCB50108EBB5010872
:10117000FDB501080CB6010888B6010836B60108AD
:1011800021B6010848B6010899B50108A3B50108C0
:10119000BCB50108016804EB020C0868A0508A88FD
:1011A000ACF80420D4F8F421D01D2244C4F8F40192
:1011B0009571DBF814202044127812F0700F03BFF1
:1011C0005B682A4619682A4618BF596817F0F9FA69
:1011D000D4F8F4311D44C4F8F451DBF8103003B1F5
:1011E0001B786355D4F8F8316A1C0133C4F8F42134
:1011F000C4F8F83188E7304601F0DEFA7BE60448AF
:1012000008F07EFF5946034814F018FF7CE700BF42
:1012100078B60108040D00202DE9F04F89B0FFF7E2
:1012200051FC0446FFF700FC012180462046FFF7F1
:10123000B3F8FFF747FC0121FFF79CF84FF49670D5
:101240000CF058FDFFF73EFC0021FFF793F8204615
:10125000854C0021FFF7A0F823685E6896B18348AB
:1012600008F04EFF246804F0C7FD8149024604AB34
:10127000204613F047F87E4902469DF8100004F01E
:10128000A7FD5EE006F01AFA7A4B6F46D3E90045F7
:10129000B5F1004F08BF002C9C4608D0021B61EB43
:1012A00005030025744C944275EB03034EDACCE938
:1012B000000104AC714808F023FF14227049204655
:1012C00014F091FE05F078FB064615F0FDF80021BC
:1012D0000546204614F0B2FE0521204614F0AEFE6D
:1012E0000021204614F0AAFE0021204614F0A6FE9C
:1012F0006449304616F082FC16F06CFE01B22046BE
:1013000014F0AEFE2946204614F0AAFE94E80F0021
:1013100087E80F00384614F09EFE0646E0B15A48B2
:1013200008F0EEFE384614F094FE0446384614F0F9
:1013300092FE2146C2B2012004F04AFD384614F064
:101340008CFE524B187809B0BDE8F08F1022314660
:10135000384617F05AFADDE74D4CD4F8FC21D4F8A2
:10136000F8319A426DD004F047FD98F850300746A6
:10137000022B4AD104F50273D3E900233C4808F05C
:10138000C0FF05264FF00408D4F8F831D4F8FC214A
:101390004FF0000B9A422CBF0025D4F80032DFF842
:1013A000D0903CBF1B199D79DFF8FCA03CBF0835ED
:1013B000EDB2BF1B002D38D0A7EB0B039D4227DDFC
:1013C000BBF1000F34D1504608F09AFED4F8FC214E
:1013D000D4F8F8118A420DD2D4F8000223189B7970
:1013E000083313F0FF031FBF01321B18C4F8FC21A0
:1013F000C4F80032D4F8FC318B4216D2D4F8003253
:1014000023449D790835EDB2D4E74FF00308BBE7DC
:10141000D4F8001206EB0B002A4621444844AB44A2
:1014200017F0CFF95FFA8BFBD0E7BBF1000F08D0C4
:101430005E443146174808F063FEF2B20C4940465C
:101440001DE7154C23783BB1144808F059FE0022E3
:1014500007492270104612E7114808F051FE04F0C7
:10146000E5FF104B6EE700BF640E002096B6010842
:101470006C0D00201000002008510100ACB60108DE
:10148000500E002000007A44CBB601081F0F002048
:1014900020000020F0B60108E60F002006B7010882
:1014A0001DB70108200F0020E0B601082DE9F04F1C
:1014B00089B00BF0C3F804460BF0CEF82146024683
:1014C0009F4808F01DFE02F0FBF904460BF0B6F849
:1014D00005460BF0C1F829460246994808F010FE6F
:1014E000984808F00DFEFFF7EDFA0146204615F08A
:1014F000DFFB204615F096FB934808F001FEFFF74E
:101500002BF8FA200CF0F6FB13F04AFE13F0DEF98C
:10151000FFF7F2F8204615F09BFB8C4808F0F0FD31
:10152000FFF782FA8A4D06462B688A4C13F0010FAA
:1015300004D103F08BFB012320602B60256802F0AF
:10154000BFF900F16001284603F04EFA2068824995
:1015500003F04CFA25683268804905A803F02EFA9A
:1015600005A9284603F084FA256800238DF80E00AB
:101570000F227B4905A803F0F5F905A9284603F0D9
:1015800077FA784A8DF80F0077492068FFF705FA57
:10159000764A824676492068FFF7FFF9754A074682
:1015A00075492068FFF7F9F9744A8DF80700744906
:1015B0002068FFF7F2F9714A8DF80A007149206836
:1015C000FFF7EBF94FF0000B70256F4B8DF80B0018
:1015D00005A92068059506938DF81CB003F050FB13
:1015E0006A4B05A98DF808002068069305958DF8CB
:1015F0001CB003F045FB8DF80900206804F08AFA5E
:1016000063498146206804F06FFA624A8DF80C0045
:1016100061492068FFF7C1F9804620685F4A80F879
:1016200028A05F49FFF7B9F95E4A06465E4920687F
:10163000FFF7B3F95D4D8DF80D003B462A78514612
:101640002068FFF7B5F9DFF874A19DF80B302A7810
:1016500039462068FFF7ACF93946554F4B469AF8A2
:1016600000202068FFF7A4F94B463A789DF80B104C
:101670002068FFF79DF943462A7849462068FFF71E
:1016800097F99DF807302A7841462068FFF790F9CE
:101690009DF809309AF8002041462068FFF788F944
:1016A00043469DF80F209DF809102068FFF780F948
:1016B0009DF80A303A789DF807102068FFF778F90E
:1016C00033463A789DF80A102068FFF771F9394AD5
:1016D0009DF80C30314620681278FFF769F99DF8C3
:1016E0000D302A789DF80C102068FFF761F9334619
:1016F0003A789DF80D102068FFF75AF99DF80830E8
:101700002A7831462068FFF753F99DF807309DF895
:101710000E209DF808102068FFF74AF9206803F0B2
:1017200029FD254808F0ECFC01224FF4C87120681F
:1017300003F0BAFC58460CF043F809B0BDE8F08F4E
:10174000B2B80108D1B80108E5B80108F6B8010837
:10175000000A00204C0E00208D09000813B9010872
:101760001CB90108490A0008CAC30108350C000861
:101770002CB901089D0D00083FB90108810E000831
:1017800044B901084DB90108F0C2010864B9010863
:1017900049C30108090B000872B9010819120008B1
:1017A0007EB901083509000887B90108200F00201B
:1017B0001C0F00201F0F002096B901081E0F0020EB
:1017C00073B502F07DF8036804469B6898470AF0F9
:1017D00047FF05460AF044FF01262946002500F58B
:1017E0007052164808F08CFC04F020FE4FF49672FC
:1017F0002B46CDE90065124912480BF0E1FE236843
:101800003146DB68204698474FF4FA7005F020FA1D
:1018100023682946DB68204698470B4808F070FC8F
:101820000A4808F06DFC0CF0BBF840F25131084852
:1018300004F0CCFE284602B070BD00BFB0B901086C
:10184000C9B90108AD140008D2B90108E5B9010809
:1018500085E50108FF22014B1A7070471C0D00201E
:1018600008B5102008F0E8FC1022002116F0CDFF8A
:1018700008BD10B5044680B1006801F08DF86068BD
:1018800001F08AF8A06801F087F8E06801F066FDD1
:101890002046BDE8104008F0B9BC10BD38B504467C
:1018A000FFF7DEFF0546204601F067FA702806D0F4
:1018B0000123E3602846FFF7DCFF002528E02046EF
:1018C00001F036FA0428F3D1204601F072F82860BE
:1018D000204601F04DFA0028ECD1204601F069F8CD
:1018E0006860204601F044FA0028E3D1204601F068
:1018F00060F8A860204601F03BFA0028DAD12046C3
:1019000001F0D3FDE860204601F032FA0028D1D181
:10191000284638BD10B50446012008F08DFC04703F
:1019200010BD70B5044601F03AFA30B9204601F016
:1019300024FA402803D00123E360002070BD204634
:1019400001F0F6F901280546F5D1204601F01BFA11
:1019500006462946204636B101F01DFAFF20BDE8B3
:101960007040FFF7D7BF01F016FA3046F7E708B12D
:1019700008F04CBC704708B5042008F05DFC00235B
:10198000036008BD10B5044638B1006801F004F8E2
:101990002046BDE8104008F039BC10BD38B50446FB
:1019A000FFF7E9FF0546204601F0E7F9702806D069
:1019B0000123E3602846FFF7E5FF00250DE0204600
:1019C00001F0B6F90128F3D1204600F0F2FF2860BB
:1019D000204601F0CDF90028ECD1284638BD08B5E5
:1019E000042008F029FC0023036008BD10B504465C
:1019F00038B1006800F0D0FF2046BDE8104008F084
:101A000005BC10BD38B50446FFF7E9FF0546204682
:101A100001F0B3F9702806D00123E3602846FFF7F0
:101A2000E5FF00250DE0204601F082F90128F3D101
:101A3000204600F0BEFF2860204601F099F90028FA
:101A4000ECD1284638BD10B5044698B1006800F0C6
:101A5000A3FF606800F0A0FF206900F09DFFA06870
:101A600000F09AFFE06800F097FF2046BDE81040C4
:101A700008F0CCBB10BD38B50446142008F0DCFBE0
:101A800014220021054616F0C0FE204601F075F92B
:101A9000702806D00123E3602846FFF7D4FF002515
:101AA00031E0204601F044F90528F3D1204600F04A
:101AB00080FF2860204601F05BF90028ECD1204629
:101AC00000F077FF6860204601F052F90028E3D16A
:101AD000204600F06EFFA860204601F049F900287A
:101AE000DAD1204600F065FFE860204601F040F9B9
:101AF0000028D1D1204600F05CFF2861204601F08B
:101B000037F90028C8D1284638BD08B51C2008F090
:101B100093FB1C22002116F078FE08BD10B5044688
:101B2000C8B1006800F038FF606800F035FFA068B9
:101B300000F032FFE06801F089F9206900F0E6FC6E
:101B4000606900F029FFA06901F080F92046BDE836
:101B5000104008F05BBB10BD38B50446FFF7D5FF59
:101B60000546204601F009F9702806D00123E360FC
:101B70002846FFF7D3FF002543E0204601F0D8F8C0
:101B80000728F3D1204600F014FF2860204601F01A
:101B9000EFF80028ECD1204600F00BFF68602046EB
:101BA00001F0E6F80028E3D1204600F002FFA8602B
:101BB000204601F0DDF80028DAD1204601F055F981
:101BC000E860204601F0D4F80028D1D1204600F08A
:101BD000A7FC2861204601F0CBF80028C8D1204698
:101BE00000F0E7FE6861204601F0C2F80028BFD18E
:101BF000204601F03AF9A861204601F0B9F8002822
:101C0000B6D1284638BD08B5142008F015FB1422BB
:101C1000002116F0FAFD08BD10B5044698B1006821
:101C200000F0BAFE606800F0B7FEA06800F0B4FEF5
:101C3000E06801F065F9206900F0AEFE2046BDE8DD
:101C4000104008F0E3BA10BD38B50446FFF7DBFFDB
:101C50000546204601F091F8702806D00123E36084
:101C60002846FFF7D9FF002531E0204601F060F853
:101C70000528F3D1204600F09CFE2860204601F0A4
:101C800077F80028ECD1204600F093FE68602046EB
:101C900001F06EF80028E3D1204600F08AFEA8602B
:101CA000204601F065F80028DAD1204601F044F919
:101CB000E860204601F05CF80028D1D1204600F011
:101CC00078FE2861204601F053F80028C8D1284644
:101CD00038BD08B50C2008F0AFFA0022026042605F
:101CE000826008BD10B5044668B1006800F054FE7B
:101CF000606801F005F9A06801F030FB2046BDE8FE
:101D0000104008F083BA10BD38B50446FFF7E1FF74
:101D10000546204601F031F8702806D00123E36023
:101D20002846FFF7DFFF00251FE0204601F000F8FE
:101D30000328F3D1204600F03CFE2860204601F045
:101D400017F80028ECD1204601F0F6F8686020462C
:101D500001F00EF80028E3D1204601F0A6FBA860B0
:101D6000204601F005F80028DAD1284638BD08B52C
:101D7000242008F061FA2422002116F046FD08BD57
:101D800010B50446F8B1006800F006FE606801F086
:101D90005DF8A06800F0E5FDE06801F0B1F82069A9
:101DA00001F054F8606900F0DCFDA06900F0DCFA95
:101DB000E06900F0F1FD206A00F0EEFD2046BDE88C
:101DC000104008F023BA10BD38B50446FFF7CFFF26
:101DD0000546204600F0D1FF702807D00123284691
:101DE000E360FFF7CDFF0025284638BD204600F010
:101DF0009FFF0928F2D1204600F0DBFD2860204635
:101E000000F0B6FF0028E9D1204601F02EF8686006
:101E1000204600F0ADFF0028E0D1042260212046DA
:101E200000F056FDA860204600F0A2FF0028D5D1A2
:101E3000204601F081F8E860204600F099FF002874
:101E4000CCD1204601F011F82861204600F090FF27
:101E50000028C3D108226021204600F039FD6861C6
:101E6000204600F085FF0028B8D10F4A0F492046D0
:101E700000F0A3FAA861204600F07AFF0028ADD157
:101E8000204600F096FDE861204600F071FF002832
:101E9000A4D1204600F08DFD2862204600F068FFA6
:101EA0000028A1D09AE700BFD5320008953300087A
:101EB00008B5242008F0C0F92422002116F0A5FC62
:101EC00008BD70B5044638B3006800F065FD606871
:101ED00000F062FDA06800F05FFDE068FFF747FDDD
:101EE000206900F0B3FF606900F0B0FFA06901F065
:101EF00007F8E56945B1D5E9000600F04DFD284633
:101F000008F084F93546F5E7206A01F027FA204603
:101F1000BDE8704008F07AB970BD2DE9F843044679
:101F2000FFF7C6FF0546204600F027FF702806D0C1
:101F30000123E3602846FFF7C4FF002550E0204658
:101F400000F0F6FE0928F3D1204600F032FD2860AB
:101F5000204600F00DFF0028ECD1204600F029FDBE
:101F60006860204600F004FF0028E3D1204600F01E
:101F700020FDA860204600F0FBFE0028DAD12046B4
:101F8000FFF7CFFCE860204600F0F2FE0028D1D138
:101F9000204600F06AFF2861204600F0E9FE002894
:101FA000C8D1204600F061FF6861204600F0E0FEE5
:101FB0000028BFD1204600F0BFFFA861204600F0F6
:101FC000D7FE0028B6D1204600F0E9FE58B12046E1
:101FD00001F06BFA2862204600F0CAFE0028A9D161
:101FE0002846BDE8F883204600F0C7FE70289FD140
:101FF000204600F09DFE4FF000080746C146002F26
:10200000E5DD082008F018F90646C0F80090C0F891
:102010000490204600F0CDFC3060204600F0A8FE81
:10202000002887D1EB691BB9EE61013FB046E6E7B6
:10203000C8F80460F9E710B5044668B1006800F01C
:10204000ABFC606800F08DFCA06800F08AFC2046C4
:10205000BDE8104008F0DAB810BD10B5044680B1F4
:10206000006800F0F3FE606800F07BFCA06800F000
:102070007BF9E06800F090FC2046BDE8104008F0D5
:10208000C5B810BD10B5044650B1006801F060FA43
:10209000606800F081FC2046BDE8104008F0B6B84A
:1020A00010BD08B5202008F0C7F82022002116F046
:1020B000ACFB08BD10B50446E0B1006800F06CFC54
:1020C000606800F0C3FEA06800F04BFCE06800F020
:1020D00017FF206900F048F9606900F045F9A06930
:1020E00000F05AFCE06900F057FC2046BDE81040C3
:1020F00008F08CB810BD000038B50446FFF7D1FFDA
:102100000546204600F039FE702807D001232846F6
:10211000E360FFF7CFFF0025284638BD204600F0DA
:1021200007FE0828F2D1204600F043FC2860204634
:1021300000F01EFE0028E9D1204600F096FE6860FF
:10214000204600F015FE0028E0D104226021204640
:1021500000F0BEFBA860204600F00AFE0028D5D1A2
:10216000204600F0E9FEE860204600F001FE00286D
:10217000CCD1144A1449204600F01FF928612046AA
:1021800000F0F6FD0028C1D1104A1149204600F0A8
:1021900014F96861204600F0EBFD0028B6D1204616
:1021A00000F007FCA861204600F0E2FD0028ADD158
:1021B000204600F0FEFBE861204600F0D9FD002833
:1021C000AAD0A3E737200008E72100085B20000819
:1021D0006922000808B50C2008F02EF800220260E1
:1021E0004260826008BD38B50446FFF7F3FF05463C
:1021F000204600F0C2FD702807D001232846E36086
:10220000FFF719FF0025284638BD204600F090FD55
:102210000328F2D1204600F0CCFB2860204600F0D5
:10222000A7FD0028E9D101226021204600F050FBE3
:102230006860204600F09CFD0028DED1012250217C
:10224000204600F045FBA860204600F091FD0028E4
:10225000D9D0D2E708B5102007F0EEFF10220021F8
:1022600016F0D3FA08BD000038B50446FFF7F2FFB8
:102270000546204600F081FD702807D0012328463E
:10228000E360FFF7EAFE0025284638BD204600F04F
:102290004FFD0428F2D1204600F0E7FD28602046DB
:1022A00000F066FD0028E9D108226021204600F0F8
:1022B0000FFB6860204600F05BFD0028DED10A4A73
:1022C0000A49204600F079F8A860204600F050FD49
:1022D0000028D3D1204600F06CFBE860204600F0D7
:1022E00047FD0028D0D0C9E7852000080123000859
:1022F00008B5082007F0A0FF00220260426008BD78
:1023000038B50446FFF7F4FF0546204600F035FDDA
:10231000702807D001232846E360FFF7B3FE0025AD
:10232000284638BD204600F003FD0228F2D12046A1
:1023300001F024F92860204600F01AFD0028E9D1B8
:10234000204600F036FB6860204600F011FD0028B2
:10235000E6D0DFE710B504460C2007F06DFF002241
:1023600002604260846010BD38B5044688B938BD4B
:1023700050F82500A36898470135D4E900039D4231
:10238000F6DB08B107F042FF2046BDE8384007F011
:102390003DBF0025F1E738B504460D4641680131DF
:1023A00041608900006817F0E3F86368206003F17A
:1023B0008043013B40F8235038BD2DE9F8430546E2
:1023C0008846164600F0D9FC70281AD13046FFF72F
:1023D000C1FF0446284600F0ABFC00260746BE427B
:1023E00002DB2046BDE8F8832846C04781462846E0
:1023F00000F0BEFC28B949462046FFF7CCFF013665
:10240000EDE701232046EB60FFF7AEFF0024E8E78D
:1024100008B5202007F010FF2022002116F0F5F962
:1024200008BD38B5044600F0A8FC702804D001238C
:102430000025E360284638BD204600F079FC0728D7
:10244000F5D1FFF7E5FF0546204600F0B2FA286017
:10245000204600F08DFC0028E9D1204600F0BDFCAC
:102460006860204600F084FC0028E0D1204600F09F
:10247000FCFCA860204600F07BFC0028D7D101229C
:102480006021204600F024FAE860204600F070FC4D
:102490000028CCD101225021204600F019FA2861F1
:1024A000204600F065FC0028C1D1204601F066F806
:1024B0006861204600F05CFC0028B8D1204600F09E
:1024C00078FAA861204600F053FC0028B2D0AEE7AD
:1024D00010B50446C8B1006800F05EFA606800F00C
:1024E00070FCA06800F0B2FCE06800F03AFA2069E5
:1024F00000F037FA606901F02BF8A06900F04CFA9F
:102500002046BDE8104007F081BE10BD10B530B1C7
:10251000C469FFF7DDFF14B12046E469F9E710BD97
:10252000F8B5054600F03BFC044608B1002406E07F
:10253000284600F022FC702803D00123EB602046DF
:10254000F8BD284600F0F4FB061EEFDD2846FFF735
:1025500068FF0446284600F00BFC70B92746013E90
:10256000002EECD02846FFF75CFFF861284600F00B
:10257000FFFB10B9FF69013EF2E701232046EB6043
:10258000FFF7C4FFD2E7000038B50546082007F082
:1025900053FE0023044603604360284600F0EDFB31
:1025A000702806D00123EB60204607F02FFE0024A0
:1025B00059E0284600F0BCFB0228F3D10422602138
:1025C000284600F085F92060284600F0D1FB00285D
:1025D000EAD123681968B1F5806F52D01DD8B1F5E2
:1025E000007F46D00AD8B1F5807F38D040F2011381
:1025F00099423AD02F4816F04BFF34E0B1F5407FB6
:102600003FD040F20133994237D040F20123994242
:10261000F0D12846FFF7F6F924E0B1F5C06F3CD0C1
:102620000ED8B1F5A06F30D040F20153994230D0AE
:1026300040F201439942DDD12846FFF7C5FB11E086
:1026400040F2017399422CD04FF6017399422CD07D
:10265000B1F5E06FCED12846FFF70DFA02E028462B
:1026600000F033FA6060204638BD284600F0AAFA30
:10267000F8E72846FFF792F9F4E72846FFF73CFD14
:10268000F0E72846FFF749FCECE72846FFF7DCFABD
:10269000E8E72846FFF738FBE4E7284600F003FBAD
:1026A000E0E72846FFF758FADCE72846FFF7F6F898
:1026B000D8E700BF4BBA010810B50446002875D012
:1026C00003681A68B2F5806F54D01ED8B2F5007F47
:1026D0004CD00BD8B2F5807F39D040F201139A422A
:1026E00040D03349334816F0D3FE33E0B2F5407F93
:1026F00040D040F201339A4240D040F201239A4246
:10270000EFD14068FFF772F924E0B2F5C06F41D015
:102710000ED8B2F5A06F35D040F201539A4235D0B1
:1027200040F201439A42DCD14068FFF729FB11E0F7
:1027300040F201739A4231D04FF601739A4231D080
:10274000B2F5E06FCDD14068FFF77DF902E0406857
:1027500000F09DF9206800F004F92046BDE8104023
:1027600007F054BD406800F012FAF3E74068FFF745
:1027700009F9EFE76068FFF7A4FBEBE74068FFF7B4
:1027800099FCE7E74068FFF747FAE3E74068FFF79F
:10279000A9FADFE7406800F06EFADBE74068FFF770
:1027A000BDF9D7E74068FFF764F8D3E710BD00BF75
:1027B00016BA01082CBA010810B5044698B1006891
:1027C00000F0EAF8606800F0CCF8A06800F0C9F802
:1027D000E068FFF771FF206900F0C3F82046BDE80C
:1027E000104007F013BD10BD38B50446142007F0A3
:1027F00023FD14220021054616F007F8204600F0BC
:10280000BCFA702806D00123E3602846FFF7D4FF06
:1028100000253FE0204600F08BFA0628F3D1204641
:1028200000F0C7F82860204600F0A2FA0028ECD19A
:1028300001226021204600F04BF86860204600F03D
:1028400097FA0028E1D101226021204600F040F8EB
:10285000A860204600F08CFA0028D6D12046FFF769
:1028600093FEE860204600F083FA0028CDD10222D2
:102870006021204600F02CF82861204600F078FA0C
:102880000028C2D1204600F07EFA18B90121204666
:1028900000F081FA284638BDB0B5CB1D23F0070300
:1028A00000AFADEB030D0A4604460D4601466846EF
:1028B00015F087FF0023013C0DEB0502AB4201DB65
:1028C000BD46B0BD01335942515C04F8011FF5E724
:1028D0002DE9F84305460C46174600F060FA064617
:1028E00038B9284600F049FAA042814603D00123B6
:1028F000EB6000242FE0284600F01AFAB0F100083F
:10290000F5DBB845F3DC384607F096FC31463A462D
:10291000044615F07AFF284600F035FAB9F1500F59
:1029200008BFC0F3C016284600F031FAA7EB08092B
:10293000A14401464246484615F043FF1EB12346D6
:10294000FF224B450AD139462046FFF7A5FF4146F5
:10295000284600F020FA2046BDE8F88303F8012B52
:10296000EFE708B107F052BC704770B50646082083
:102970000D4607F061FC00239D420446036043605E
:1029800008DD284607F058FC2A462060314615F03D
:1029900018FF6560204670BD10B5044640B1006860
:1029A00008B107F033FC2046BDE8104007F02EBC0C
:1029B00010BD70B5044600F0F2F928B9204600F0C9
:1029C000DCF918B10123E36000250FE0204600F098
:1029D000AFF9061EF6DB204600F0D9F93146FFF7C5
:1029E000C4FF31460546204600F0D5F9284670BDA3
:1029F00003463038C0B209280DD9A3F16102052A77
:102A000002D8573BD8B27047A3F14102052A01D83A
:102A1000373BF7E70020704710B504460078FFF712
:102A2000E7FF01466078FFF7E3FF40EA0110C0B21C
:102A300010BD2DE9F84300AF044616F0EDFEC307C4
:102A40001AD44510EB1D23F00703ADEB030DE84648
:102A50000DF1FF3604EB45094C4506D129464046A9
:102A6000FFF783FFBD46BDE8F8832046FFF7D4FF9C
:102A7000023406F8010FEFE70020F3E708B51C2049
:102A800007F0DAFB1C22002115F0BFFE08BD10B5CF
:102A90000446C8B10068FFF77FFF6068FFF77CFF5E
:102AA000A068FFF779FFE068FFF776FF2069FFF77E
:102AB00073FF6069FFF770FFA069FFF752FF2046C0
:102AC000BDE8104007F0A2BB10BD38B50446FFF7C3
:102AD000D5FF0546204600F050F9702806D00123A6
:102AE000E3602846FFF7D3FF002545E0204600F0CD
:102AF0001FF90728F3D12046FFF75BFF2860204627
:102B000000F036F90028ECD12046FFF752FF68604C
:102B1000204600F02DF90028E3D12046FFF749FFB9
:102B2000A860204600F024F90028DAD12046FFF7FB
:102B300040FFE860204600F01BF90028D1D1204674
:102B4000FFF737FF2861204600F012F90028C8D1AE
:102B50002046FFF72EFF6861204600F009F90028A3
:102B6000BFD1012260212046FFF7B2FEA8612046B6
:102B700000F0FEF80028B4D1284638BD08B518206A
:102B800007F05AFB1822002115F03FFE08BD10B5D2
:102B90000446B0B10068FFF7FFFE6068FFF7FCFE77
:102BA000A068FFF7F9FEE068FFF7F6FE206900F085
:102BB0004DF96069FFF7D5FE2046BDE8104007F0EB
:102BC00025BB10BD38B50446FFF7D8FF05462046A3
:102BD00000F0D3F8702806D00123E3602846FFF701
:102BE000D6FF00253CE0204600F0A2F80628F3D1ED
:102BF0002046FFF7DEFE2860204600F0B9F80028E6
:102C0000ECD12046FFF7D5FE6860204600F0B0F812
:102C10000028E3D12046FFF7CCFEA860204600F054
:102C2000A7F80028DAD12046FFF7C3FEE860204667
:102C300000F09EF80028D1D1204600F016F9286156
:102C4000204600F095F80028C8D1012260212046D6
:102C5000FFF73EFE6861204600F08AF80028BDD1EB
:102C6000284638BD08B5142007F0E6FA14220021E2
:102C700015F0CBFD08BD10B5044698B10068FFF70C
:102C80008BFE6068FFF788FEA068FFF785FEE068AE
:102C900000F036F9206900F061FB2046BDE81040E5
:102CA00007F0B4BA10BD38B50446FFF7DBFF0546A0
:102CB000204600F062F8702806D00123E360284621
:102CC000FFF7D9FF002531E0204600F031F8052854
:102CD000F3D12046FFF76DFE2860204600F048F84B
:102CE0000028ECD12046FFF764FE6860204600F023
:102CF0003FF80028E3D12046FFF75BFEA86020469E
:102D000000F036F80028DAD1204600F015F9E86026
:102D1000204600F02DF80028D1D1204600F0C5FB58
:102D20002861204600F024F80028C8D1284638BD84
:102D3000F0B5836805680022EB5C466803F0700319
:102D4000703B18BF4FF0FF338168B14201F10104BD
:102D500002D38460D018F0BD695C01F00F0709064A
:102D600047EA0212F5D58460002BEDD0013BEBE77A
:102D7000C068003018BF0120704702688368D05CCB
:102D800000F07000704702688368D05C704702688A
:102D90008068104470478368194481607047826876
:102DA00003689B5C012B03BF013282601846002040
:102DB000704708B5082007F03FFA00220260426021
:102DC00008BD10B5044638B14068FFF7CAFD20467B
:102DD000BDE8104007F01ABA10BDF8B50646FFF777
:102DE000DEFF20BB3046FFF7C8FF05463046FFF741
:102DF000CAFF0746FFF7DDFF602D057004464FF060
:102E0000010517D0F5600BE06D00AF42FCDC2A46EF
:102E100060213046FFF75CFD237860601D4325701C
:102E20003046FFF7A5FF18B12046FFF7CAFF002480
:102E30002046F8BD07F00F07013FE6E708B5082078
:102E400007F0FAF900220260426008BD10B504469E
:102E500050B10068FFF785FD6068FFF782FD2046EE
:102E6000BDE8104007F0D2B910BD38B50446FFF7F1
:102E700096FF60B9FFF7E2FF05462046FFF77DFFAA
:102E8000702806D00123E3602846FFF7DFFF002506
:102E90001AE02046FFF74CFF0228F3D101226021FF
:102EA0002046FFF715FD28602046FFF761FF002848
:102EB000EAD1042260212046FFF70AFD686020461F
:102EC000FFF756FF0028DFD1284638BD08B5082097
:102ED00007F0B2F900220260426008BD38B504462E
:102EE0000D460168013101608900406816F040FB21
:102EF0002368606003F18043013B40F8235038BDF4
:102F000038B50446B8B1436813B10368002B10DC30
:102F10002046BDE8384007F079B950F82500FFF7A2
:102F20003BFD0135D4E90030AB42F6DC07F06EF929
:102F3000EEE70025F6E738BDF8B50546FFF72FFFA9
:102F400048B9FFF7C3FF04462846FFF716FF70286D
:102F500003D00123EB60002405E02846FFF7E8FEDC
:102F60000646002E01DC2046F8BD2846FFF721FD6D
:102F700007462846FFF7FCFE30B91FB13946204608
:102F8000FFF7ACFF013EECE701232046EB60FFF7C3
:102F9000B7FFE0E708B5102007F04EF91022002136
:102FA00015F033FC08BD38B504460D46C168013143
:102FB000C1608900806816F0DBFAE368A06003F165
:102FC0008043013B40F8235038BD08B5082007F086
:102FD00033F900220260426008BD08B55C2007F0AA
:102FE0002BF95C22002115F010FC08BD10B5044639
:102FF000002849D00068FFF7CFFC6068FFF726FF84
:10300000A068FFF7AEFCE068FFF7ABFC2069FFF7B4
:10301000A8FC6069FFF7A5FCA069FFF7A2FCE069C6
:10302000FFF79FFC206AFFF79CFC606AFFF799FCA2
:10303000A06AFFF796FCE06AFFF793FC206BFFF7AE
:10304000ABFC606BFFF78DFCA06BFFF78AFCE06BBD
:10305000FFF787FC206CFFF784FC606CFFF781FCB6
:10306000A06CFFF77EFCE06CFFF77BFC206DFFF7A8
:1030700078FC606DFFF775FCA06DFFF78DFC2046B6
:10308000BDE8104007F0C2B810BD38B50446FFF7E0
:1030900086FE60B9FFF7A1FF05462046FFF76DFEEB
:1030A000702806D00123E3602846FFF79FFF002524
:1030B00005E12046FFF73CFE1728F3D12046FFF735
:1030C00078FC28602046FFF753FE0028ECD120460C
:1030D000FFF7CBFE68602046FFF74AFE0028E3D1E9
:1030E000082260212046FFF7F3FBA8602046FFF787
:1030F0003FFE0028D8D1012260212046FFF7E8FBDF
:10310000E8602046FFF734FE0028CDD1012250218F
:103110002046FFF7DDFB28612046FFF729FE002847
:10312000C2D1082250212046FFF7D2FB6861204619
:10313000FFF71EFE0028B7D1012260212046FFF7CD
:10314000C7FBA8612046FFF713FE0028ACD101227F
:1031500050212046FFF7BCFBE8612046FFF708FE40
:103160000028A1D1082250212046FFF7B1FB286298
:103170002046FFF7FDFD002896D101226021204660
:10318000FFF7A6FB68622046FFF7F2FD00288BD10F
:10319000012250212046FFF79BFBA8622046FFF743
:1031A000E7FD002880D1082250212046FFF790FB40
:1031B000E8622046FFF7DCFD00287FF475AF20466B
:1031C000FFF7F7FB28632046FFF7D2FD00287FF4C6
:1031D0006BAF012260212046FFF77AFB686320462F
:1031E000FFF7C6FD00287FF45FAF01225021204683
:1031F000FFF76EFBA8632046FFF7BAFD00287FF4B7
:1032000053AF082250212046FFF762FBE8632046B7
:10321000FFF7AEFD00287FF447AF01226021204672
:10322000FFF756FB28642046FFF7A2FD00287FF435
:103230003BAF012250212046FFF74AFB686420463D
:10324000FFF796FD00287FF42FAF0822502120467B
:10325000FFF73EFBA8642046FFF78AFD00287FF4B5
:1032600023AF012260212046FFF732FBE8642046AD
:10327000FFF77EFD00287FF417AF01225021204682
:10328000FFF726FB28652046FFF772FD00287FF434
:103290000BAF082250212046FFF71AFB6865204635
:1032A000FFF766FD00287FF4FFAE2046FFF781FBA5
:1032B000A8652046FFF75CFD00287FF4F5AE2846A0
:1032C00038BD08B5142006F0B7FF1422002115F010
:1032D0009CFA08BD10B5044698B10068FFF75CFB86
:1032E0006068FFF73EFBA068FFF73BFBE06800F07B
:1032F0002FF92069FFF750FB2046BDE8104006F08B
:1033000085BF10BD10B5044638B3D0E90030FBB11D
:103310001B78013B032B16D8DFE803F0020C0F12D9
:1033200000F016F92068FFF71CFB2046BDE81040AE
:1033300006F06CBFFFF7CEFFF4E7FFF757FEF1E7AB
:10334000FFF784FDEEE70028ECD006F05FFFE9E729
:103350000028EAD006F05AFFE7E710BD38B504466A
:10336000B8B10068FFF718FB6068FFF7CBFF0025D6
:10337000D4E902039D4206DB06F048FF2046BDE883
:10338000384006F043BF50F82500FFF7E7FF01354E
:10339000EEE738BD38B50446FFF701FD60B9FFF729
:1033A00090FF05462046FFF7E8FC702806D0012371
:1033B000E3602846FFF78EFF002535E02046FFF743
:1033C000B7FC0528F3D12046FFF7F3FA2860204622
:1033D000FFF7CEFC0028ECD1012260212046FFF748
:1033E00077FA68602046FFF7C3FC0028E1D101228C
:1033F00050212046FFF76CFAA8602046FFF7B8FC82
:103400000028D6D1204600F0B9F8E8602046FFF742
:10341000AFFC0028CDD12046FFF7CBFA286120462B
:10342000FFF7A6FC0028C4D1284638BD38B50546AC
:10343000FFF7B5FC60B9FFF7C8FD04462846FFF763
:103440009CFC702806D00123EB602046FFF75AFF52
:1034500000241CE02846FFF76BFC0228F3D1012270
:1034600060212846FFF734FA20602846FFF780FCE9
:103470000028EAD123681B78013B032BE3D8DFE85F
:1034800003F002080C10284600F078F8606020462F
:1034900038BD2846FFF77EFFF8E72846FFF7F5FD21
:1034A000F4E72846FFF7E1FCF0E7F8B50446FFF73C
:1034B00076FC60B9FFF76EFD05462046FFF75DFC20
:1034C000702806D00123E3602846FFF747FF002558
:1034D00025E02046FFF72CFC0328F3D12046FFF718
:1034E00068FA28602046FFF743FC0028ECD120460C
:1034F000FFF79CFF68602046FFF73AFC0028E3D105
:103500002046FFF74CFC50B92046FFF736FC7028E8
:10351000D8D12046FFF70CFC0646002E01DC2846D9
:10352000F8BD2046FFF7C1FF07462046FFF720FC05
:103530000028C9D11FB139462846FFF734FD013EA6
:10354000EBE708B5082006F077FE0023036008BD0E
:1035500010B5044688B12378406823B1402B09D0C8
:10356000FFF7FFF901E0FFF717FA2046BDE810402A
:1035700006F04CBEFEF7FBF9F7E710BDF8B50546BF
:10358000FFF70DFC38BB2846FFF7F7FB0646284639
:10359000FFF7F9FB0746FFF7D4FFF1B2402E0446D0
:1035A00001701BD003DC5EB10123EB600CE0502EF8
:1035B00001D0602EF8D107F00F070126013F12E07D
:1035C0002846FFF7F6F960602846FFF7D1FB18B1EF
:1035D0002046FFF7BDFF00242046F8BD2846FEF731
:1035E000A0F9F0E77600B742FCDC32462846FFF748
:1035F0006FF9237860601E432670E5E738B50A4C02
:1036000005460121204603F0C9FD002320461A4645
:10361000012103F001FD85F001022046BDE838409C
:10362000012103F0C7BD00BF0000024008B5012022
:10363000FFF7E4FFBDE80840032004F0F1BC0846B2
:10364000FFF7DCBF10B50446024B036013F04AFBE2
:10365000204610BD84BA010810B50446054B503011
:1036600040F8503C044B40F8083CFFF7EBFF204685
:1036700010BD00BF60BE010824C0010810B504469B
:10368000FFF7E0FF2046082112F036FD204610BD6E
:1036900010B50446FFF7E0FF20467C2112F02CFD18
:1036A000204610BD04F06CBD024B01211868036870
:1036B0001B681847780E0020021C18BF0122032146
:1036C000014803F077BD00BF0004024010B50C466E
:1036D0000AF0A8FD022808D14FF47A704443B4FBE5
:1036E000F0F0BDE810400AF005BB2046BDE81040F0
:1036F00003F0AEBA0321014803F065BD00040240A7
:1037000008B5034806F0FCFCBDE8084004F038BDED
:1037100074BE010810B5094C094806F0F1FC2046BA
:103720000B2103F03BFD002320461A460B2103F03A
:1037300073FCBDE8104003F071BA00BF0000024006
:10374000FCBD010808B5022003F0CCF903F02EFA05
:1037500000F09EFC03F054FA00F088FE03F0B8FF7E
:103760000C4802F0FDFE4FF4E13004F0B5FA0A4BCC
:103770001A680AB9094A1A60094B1A680AB9074A4D
:103780001A60084806F0BCFCBDE80840064806F090
:10379000B7BC00BF2D36000860110020797B0008FF
:1037A00064110020F4BA01080CBB01082DE9F347AD
:1037B000044626464FF01B0913F02AFA284B04F161
:1037C000210846F8113B10220021304615F01DF863
:1037D0004A460021404615F018F800252146214BA5
:1037E000C4E90F5504F1480041F8443F01F02EF8B8
:1037F0001D4B1E4FA3651E4B84F85C50C4E9183561
:103800001C4BC4E91B55A36684F87450A5671A487D
:1038100006F076FC3B68DFF86CA00193DAF8003024
:10382000164D00932B68164A4946404615F012FF84
:103830002968304606F06FFDDAF8001004F1150033
:1038400006F069FD396804F1190006F064FD296885
:1038500004F11D0006F05FFD204602B0BDE8F087D0
:1038600060BE01082CBF01083CBF01086400F81FBE
:1038700094BF010858BF010830BE01085000F81F6E
:1038800045BE01085400F81F10B5094CFFF75AFF58
:103890002368DB0709D40748FFF788FF0123064A9E
:1038A00006490448236013F073FA024810BD00BFB4
:1038B000700E00207C0E0020000000205936000809
:1038C00038B5064D064C2B6813F0010F04D1FFF7F5
:1038D000DBFF012320602B60206838BD740E0020C0
:1038E000F80E002010B5FFF7EBFF836F11203BB1FE
:1038F00004F034FCFFF7E4FFBDE81040836F184785
:10390000BDE8104004F037BC08B50B21054803F0B2
:103910005FFC28B1BDE808400B21024803F06CBCF5
:1039200008BD00BF0000024008B519B1BDE808405D
:10393000FFF7F0BE044806F0E3FBBDE808400222B2
:103940000B21024803F0A6BB18BE0108000002408C
:1039500070B504462E4804F1440506F0D1FB284614
:10396000002100F09FFD0021284600F0B1FD204617
:1039700013F07EF90CF056FB20460021FFF7D4FF30
:103980000BF052FA01220C21224803F083FB03F0D2
:10399000CFFF04F1480000F03BFF23682046DB68BE
:1039A00004F16805002198471B4E0021284600F0CD
:1039B00015FE03F07FFC194806F0A2FB04F07AF82C
:1039C00003F01EF9304601220D2103F063FB0122B2
:1039D00030460E2103F05EFB0021084603F054FF41
:1039E00004F1580000F08AFD0121284600F0F6FDA0
:1039F0004FF4E13004F070F9094806F081FB0BF058
:103A000039F903F093FF2046BDE8704013F040B948
:103A1000CABD01080004024000000240EEBD0108DA
:103A200015C4010838B50546FFF76EFF044628B1F6
:103A300000212846FFF778FF03F0F0F802F0BCFF02
:103A400005460CB1FFF766FE284638BD70B50C463A
:103A500006461549204614F08DFA20B9002120466B
:103A600014F06AFA70B11149204614F0C7F814F046
:103A70008BFA01460E4806F043FB4FF4C0710D4827
:103A800002F0A4FD3046FFF73FFF054648B9304637
:103A9000FFF7C8FF0146204614F06CFA08B1FFF7A3
:103AA00039FE284670BD00BF3333534000007A44CE
:103AB00022BB010885E5010870B52D4AD6B0136810
:103AC0000546DB0705D42B4900F168030B60012391
:103AD000136029492846FFF7B9FF0646274806F034
:103AE0000FFB002105F1440000F0F2FC244C254BB3
:103AF000E360254B2361254BA360254B6360254B79
:103B00002360254B6361254BA361254BE36104F1E1
:103B100010030FCB8DE80F0094E80F0012F0B4FDF6
:103B2000002305A8EB632B6412F03AFD9DF81430D6
:103B300005F13C04012B14D1DDF8153005A8EB6329
:103B4000DDF819302B6412F0FBFC164806F0D8FAA9
:103B50000821204606F03AFBBDF91611124806F07E
:103B6000CFFA31462846FFF7DFFE56B070BD00BFE2
:103B70006C0E0020780E0020000040408DBA010835
:103B8000A81F0020516C0008D96B0008A936000856
:103B9000F5360008B936000801A10008B5C30008D1
:103BA000F5C30008AEBA0108D4BA01087FB5F823FE
:103BB00000F1580504AC0646284604F8013D00F023
:103BC000A3FC0223214600930122A123284600F0F2
:103BD0009FFC4FF400430822009306F16C01A123DF
:103BE0000446284600F0BEFC0440E4B2284600F03B
:103BF0008DFC204604B070BD30B58BB0044604F097
:103C00003DFA01465A4806F07BFA04F091FA014663
:103C1000584806F075FA584806F072FA204600F047
:103C2000DBFB04F1580500F00FFB00F0B9FA534834
:103C3000534906F065FA284600F060FC38B951484F
:103C400006F05EFA40F23B114F4802F0BFFC02F072
:103C5000E5FF2046FFF7AAFF20B94FF4A0714A48BC
:103C600002F0B4FC94F8730094F86E30049094F869
:103C7000720094F86D20039094F8710094F86C1021
:103C8000029094F87000019094F86F0000903F4803
:103C900006F036FA284600F085FA284600F0E6FAE3
:103CA00004F14405002184F87400284600F0FAFB72
:103CB000012000F0D9FD0021284600F009FC012078
:103CC00000F0F0FD2046FFF7F7FE00F01BFB304848
:103CD00006F016FA4FF4FA7014F034FD0546002889
:103CE0003ED12C4806F00CFA2B4806F009FA2B4876
:103CF00006F006FA2A4806F003FA2A4806F000FA07
:103D0000294806F0FDF9294806F0FAF9284806F096
:103D1000F7F9284806F0F4F9274A2849284806F018
:103D2000EFF92849284806F0EBF9284806F0E8F9A9
:103D300004F12101264806F0E3F92649264806F059
:103D4000DFF907A803F05CFC07A806F02FF901468D
:103D5000224806F0D5F9114806F0D2F90BB030BD73
:103D60001F4806F0CDF9284614F0F4FCBCE700BF6C
:103D700051BB010867BB01087DBB010894BB01086A
:103D8000A0860100AFBB010885E50108C5BB01089D
:103D9000FABB01082DBC010883E501086BBC0108D2
:103DA0009CBC0108ABBC0108CDBC0108F0BC0108FB
:103DB00014BD010884E5010837BD01083DBD0108B7
:103DC0004CBD01085BBD010862BD01086DBD010865
:103DD0008DBD010898BD01089EBD0108B8BD010850
:103DE00061BC01082DE9FF4100F15805284600F0AB
:103DF0008BFB04240226284F013C14F0FF0432D030
:103E0000A123012239460096284600F081FB4FF499
:103E10000043804600930422A12302A9284600F013
:103E2000A1FBB8F1000FE7D00028E5D09DF80830DD
:103E3000442B1FD19DF809306E2B1BD10DF10A00C8
:103E400006F04DFA013084B221460DF109008DF8DB
:103E5000086006F069FA002303220093A02302A958
:103E6000284600F055FB284600F050FB204604B0E1
:103E7000BDE8F0814FF488430024ADF808306E238C
:103E800000210DF10B008DF80A3006F04DFA009478
:103E9000A0230522E3E700BF8CBA010838B50C4621
:103EA000113105460BF07EFF214651F86C3F284644
:103EB0002B604B686B6038BD30B50D469DB0044635
:103EC00001466846FFF7EAFF694628460BF0A8FC62
:103ED00004F1110321346B632C631DB030BD00006D
:103EE00030B508468DB014460F4B104A104911F0FA
:103EF000A5F800210F4A0A9107920F4A06910892ED
:103F00000E490F4A0F4D09920494059104AA01AC81
:103F100007CA0B9584E8070007AB00950FCB11F09B
:103F2000C3FB0DB030BD00BFA5360008B1B301081A
:103F3000D5B301080D6D0008956C00080000080855
:103F400001370008E5380008024B186803685B6811
:103F5000184700BF080F0020024B186803689B68D1
:103F6000184700BF080F00202DE9FF410023154628
:103F70001370022206460D4F04AC386804F8011D88
:103F800003680092D3F80C80012233462146C047D3
:103F900048B14FF4004238682946036800921C6912
:103FA00001223346A04704B0BDE8F081080F00208D
:103FB00030B585B08DF80D200022074B8DF80C1020
:103FC0001C6803A923680092DD680222034620468C
:103FD000A84705B030BD00BF080F002037B54FF42B
:103FE0000045064B1C68236800951D6913460A4668
:103FF00001462046A84703B030BD00BF040F002093
:1040000037B50025054B1C6823680095DD6813460D
:104010000A4601462046A84703B030BD040F0020E1
:1040200037B50225054B1C6823680095DD681346EB
:104030000A4601462046A84703B030BD040F0020C1
:10404000024B186803681B68184700BF040F002064
:10405000024B186803685B68184700BF040F002014
:10406000024B186803689B68184700BF040F0020C4
:104070004FF47A735843B0FBF3F009F03BBE10B530
:104080000446FFF71DFC2146BDE81040FFF7AABE1D
:1040900010B5424C0AF01AFF20460222002102F01D
:1040A000F9FF01222046114602F0F4FF20460122CA
:1040B000022102F0EFFF20460222032102F0EAFF74
:1040C00020460022042102F0E5FF204602220821BA
:1040D00002F0E0FF20460122092102F0DBFF20462A
:1040E00001220A2102F0D6FF204602220B2102F013
:1040F000D1FF02F085FD002320461A460C2102F074
:104100008BFF204600220C2103F054F820460022A9
:1041100004F580640F2102F0BDFF2046012200213A
:1041200002F0B8FF20460022022102F0B3FF204631
:104130000022032102F0AEFF20460222062102F0F7
:10414000A9FF20460022082102F0A4FF20460022F9
:10415000092102F09FFF204601220C2102F09AFF64
:10416000204602220D2102F095FF204602220E2158
:1041700002F090FF204602220F2102F08BFF002365
:1041800004F5806420461A460D2102F045FF2046C2
:10419000BDE8104000220D2103F00CB800000240E1
:1041A00003F096BA1D4B00B51A6889B0D2075FBFFD
:1041B0001B4A106001221A601A4B1B4A04931B4BC6
:1041C00005931B4B03931B4B02931B4B079308ABAD
:1041D00043F8082D93E803008DE8030002AB0FCBF2
:1041E00012F002F990B1154805F08AFF0022144838
:1041F000114602F04FFF0F2302220021104802F067
:10420000E9FD09B05DF804EB12F088B86A210D48A9
:1042100009B05DF804EB02F0D9B900BF000F00202F
:10422000080F0020493F000871400008593F00086E
:10423000693F0008B13F000801A1000810BF010854
:104240000000024085E50108002307B5ADF8043001
:1042500001238DF8063001980AF094FD02F0D0FC9D
:1042600003B05DF804EB0AF0DFBD0000194B10B598
:104270001A688CB0D2075FBF174A106001221A601B
:10428000164B0793164B0593164B0693164B089344
:10429000164B0993164B0A93164B0B930CAB13E971
:1042A00007008DE8070005AB0FCB11F0C1FF0446F6
:1042B00001220F21104802F0EDFE3CB10F4805F03D
:1042C0001FFF11F093FF20460CB010BD0C4805F005
:1042D00017FFF8E7FC0E0020040F0020DD3F000868
:1042E00001400008214000084140000851400008FA
:1042F0006140000801A100080000024092BE0108D0
:10430000C5BE01082DE9F0479AB00BF06BF9DFF854
:10431000C0A0274C274FDFF8BC8012AD50B9CDE9C3
:104320001544CDE91387CDF848A0009495E80F0017
:104330000BF072F9204B00261393204B4FF001092C
:1043400012931F4B06A914931E4B284615931E4B20
:10435000CDE91887CDE916340423CDE906368DF86A
:104360001D9006F0EBFB06F0DDFB06F023F8174A84
:10437000CDE9096611920322CDE90C440B9608920F
:104380008DF8269008AB02AC0FCBCDE90F87CDF8A6
:1043900038A084E80F0010AB93E803008DE8030019
:1043A0000CAB0FCB0BF040FD1AB0BDE8F08700BF9F
:1043B00001A100080DA20008ADED000875EC000891
:1043C00085EB00081DEB000831EB00087F4000087A
:1043D000BD76000839A200082DE9F047044602F036
:1043E000EBFA1E49054613F009FC13F0CDFD01461A
:1043F0001B4805F085FE4FF08041284613F09CFDD8
:1044000048B30025DFF86090DFF85080154E02F0C9
:10441000D3FA4946074613F0A3FDA8B941463846EA
:1044200013F0ECFB13F0B0FD0146304605F068FEDA
:10443000236885F001052046DB68294698474FF43C
:104440007A7002F005FCE2E723682046BDE8F047F9
:10445000DB6800211847BDE8F08700BF00007A4400
:10446000E3BE0108F5BE01080000204008B5094977
:10447000012002F083FF08490B2002F07FFF07496B
:104480000A2002F07BFFBDE808400549072002F042
:1044900075BF00BF81BE000809C2000835C0000812
:1044A0007DC20008002310B50C461A460D210748AE
:1044B00002F0B2FD14B1012C00D010BD2246BDE8BF
:1044C00010400D21014802F075BE00BF00080240F7
:1044D000002310B50C461A460C21074802F09CFD3B
:1044E00014B1012C00D010BD2246BDE810400C21B3
:1044F000014802F05FBE00BF00000240014802F028
:10450000C7BE00BFA086010002F092BE02F0ACBEA2
:104510002DE9F041069F1E4607F00303032B80465A
:104520000C46154603D12F210D4802F04FF82046C6
:10453000BC07324629460AD502F0E4FE10B101203C
:10454000BDE8F0810123002088F80430F8E7FB077C
:1045500002D502F0E5FEF1E702F0C6FEEEE700BF8D
:1045600085E501082DE9F041069C0D46E1078046EE
:1045700016461F4603D54C210D4802F027F8A20726
:1045800003D54F210A4802F021F823043A46314668
:1045900028460AD502F0D2FE10B10120BDE8F08114
:1045A0000123002088F80430F8E702F08FFEF3E7DB
:1045B00085E5010808B50321034802F004FE003038
:1045C00018BF012008BD00BF000402400A4602488F
:1045D000032102F0EFBD00BF0004024008B581B125
:1045E000012303211A460A4802F016FD0321084858
:1045F00002F0D4FDBDE8084003220548114602F050
:10460000EBBC0122BDE808400321014802F042BD95
:104610000004024003F052B81FB501A805F088FC61
:1046200001A803F02BF905B05DF804FB03F094B882
:1046300003F0ACB8084602F023BFDFB50023CDE994
:104640000133ADF80C3001238DF807308DF80830B8
:104650006FF01D038DF809300723044601A88DF87B
:104660000A3005F08AFC236806461B6820460F4680
:104670009847864277EB0103B4BF0120002004B0C5
:10468000D0BD70B50646194610461D4614460BF0BF
:104690000DF8736823B120462946BDE870401847DD
:1046A00070BD00002DE9FF4714461D46824603F009
:1046B00005F880468946261A22462B4601A865EB56
:1046C000010705F035FC4046494605F099FC2946AE
:1046D0008046204605F094FC39460446304605F0F5
:1046E000A5FC224603464146074805F009FD01A8FE
:1046F00002F076FF20B132463B465046FFF7C1FF3D
:1047000004B0BDE8F08700BF64BF01087047704780
:104710007FB500F10806054630460C4612F00CFB4A
:1047200060BB334805F0ECFCA27C617C314805F0AD
:10473000E7FC637C3BB16868002103681B6898470D
:10474000022000F091F8A37C3BB168680021036867
:104750005B689847022000F0A5F861684E2918D0E0
:104760004F2916D0452914D01621234801F02EFFD9
:104770001721224B224A234813F006FE64213046BB
:1047800012F0C6FA0028CFD143211B4801F01EFFCA
:10479000CAE7A268082A0BD0092A09D0072A07D03D
:1047A0002421154801F012FF144B174A2521E2E796
:1047B000E3680A2B10D009DC052B0ED034210E48FB
:1047C00001F004FF0D4B114A3521D4E70F2B04D023
:1047D000142BF3D1022300E00123A07C0290607C23
:1047E0000190207C0090206803F0B0FA04B070BD06
:1047F000B0BF0108C9BF010885E501080AB8010872
:1048000044C00108E6BF0108A8C0010874C001083F
:1048100010B5044603F06CFA04F10800BDE810403E
:1048200012F08DBA084603F079BB38B50C468D18E6
:10483000AC4204D014F8010B03F070FBF8E738BD6C
:1048400003F07CBA084603F099BB000010B504469B
:10485000044BC0E900310121083012F07BFA2046F8
:1048600010BD00BF24C00108042817D8DFE800F0FD
:104870000309100E1200002303211A46084802F013
:10488000CBBB00220321064802F004BC0222F9E758
:104890000122F7E70321024802F022BC704700BF63
:1048A00000000240042817D8DFE800F00309100ECA
:1048B0001200002302211A46084802F0ADBB002274
:1048C0000221064802F0E6BB0222F9E70122F7E7DF
:1048D0000221024802F004BC704700BF0000024001
:1048E00010B50446C06908B105F090FC206908B114
:1048F00005F08CFC606808B105F088FC204610BD0E
:1049000010B50446006808F061FB204610BD0000A9
:104910001FB50B46546801780294127801925A68C8
:10492000009242681B68024805F0EAFB04B010BD23
:10493000E0C00108CB21014801F048BE85E501082F
:10494000FE2307B502A901F8043D054B18680023B2
:1049500000681A4608F02AF803B05DF804FB00BFAF
:10496000180F0020D0B51F467423C0E90031002382
:10497000044683600820164611F09EFBC0E90067DC
:10498000A0602046D0BD0000036837B5632B044605
:104990000D4601D0FFF7CEFF002302AA42F8043DE6
:1049A000A168284605F092F9019B1BB13821024805
:1049B00001F00CFE03B030BD85E5010870B563233E
:1049C0000025C0E90031044685601A20164611F022
:1049D00073FB1A22294613F018FF3146A0602046C7
:1049E000FFF7D2FF204670BD81647047C1647047F5
:1049F0002DE9F843D0E90173884600254FF00C09F2
:104A0000DB1B0A4E9B105E43ECB2B4420BD209FB97
:104A100004724146506814F0EDFE01350028F3D1D0
:104A20002046BDE8F8834FF0FF30FAE7ABAAAAAA08
:104A30002DE9F843D0E90473884600254FF00C09AE
:104A4000DB1B0A4E9B105E43ECB2B4420BD209FB57
:104A500004724146506814F0CDFE01350028F3D1B0
:104A60002046BDE8F8834FF0FF30FAE7ABAAAAAAC8
:104A70002DE9F0410E4649680446FFF7B9FFC0B280
:104A8000FF2803D07C21294801F0A0FDD4E90123AF
:104A9000274F9B1A9B107B437E2B03D97F212348F2
:104AA00001F094FDD4E901120C25E068531A9B1023
:104AB000121A7B4392107A430133934205FB03F8A9
:104AC0000ED84144A160D4E9013496E80700E31A06
:104AD00004E9070016489B1058430138BDE8F081EF
:104AE000404605F0A9FB054618B969210F4801F0B9
:104AF0006DFDD4E901C30027A3EB0C039A100C4B06
:104B00005343002B09DD05EB070E0CEB070207CA28
:104B1000013B8EE807000C37F3E7604605F076FBB3
:104B200065604544C4E90255CDE700BF85E501084D
:104B3000ABAAAAAA1FB56E23CDE90131002301A9B2
:104B40000393FFF795FF05B05DF804FBFF2270B5F6
:104B5000002380F828204FF000424FF0FF31C0E9D9
:104B60000D23C2636FF07F42C0E910120522C0E935
:104B70000033C0E91423C0E902330022C0E9043342
:104B8000C0E90633C0E908330363C0E91233836523
:104B90004FF000431E4DC0E918232A68044612F066
:104BA000010213D101211B4E08463260716007F0EB
:104BB00023FE306018B95121174801F007FD012389
:104BC000164A174913482B6012F0E2F8154B1A6881
:104BD0000AB9104A1A6014492046FFF7ABFF134B7D
:104BE000134918702046FFF7A5FF124B12491870A1
:104BF0002046FFF79FFF114B114918702046FFF721
:104C000099FFFE220F4B18700F4B20461A7070BD93
:104C1000140F0020980F002085E5010800000020F7
:104C200001490008180F00204CC20108200F002085
:104C300054C201081E0F00205CC201081C0F002096
:104C400061C201081F0F00201D0F002010B5084C85
:104C50002368DB0709D40748FFF778FF0123064ADA
:104C600006490448236012F093F8024810BD00BFC3
:104C7000100F0020300F002000000020E148000845
:104C80002DE9F0410E4649680446FFF7D1FEC0B257
:104C9000FF2803D08721294801F098FCD4E9042398
:104CA000274F9B1A9B107B437E2B03D98A212348D5
:104CB00001F08CFCD4E904120C25A069531A9B1056
:104CC000121A7B4392107A430133934205FB03F897
:104CD0000ED841446161D4E9043496E80700E31A30
:104CE00004E9070016489B1058430138BDE8F081DD
:104CF000404605F0A1FA054618B969210F4801F0B0
:104D000065FCD4E904C30027A3EB0C039A100C4BF9
:104D10005343002B09DD05EB070E0CEB070207CA16
:104D2000013B8EE807000C37F3E7604605F06EFAAA
:104D300025614544C4E90555CDE700BF85E5010877
:104D4000ABAAAAAA38B5D0E901239B1A074A9B103F
:104D50005343CDB29D42044603D3A621044801F03B
:104D600035FC0C20636800FB053038BDABAAAAAA4D
:104D700085E5010838B5CCB2114905460B6813F03A
:104D8000010307D10F4A70201372012310600E48EF
:104D90000B605060FF2C10D0D5E904239B1A0B4AFE
:104DA0009B1053439C4203D3B221094801F00EFCEF
:104DB0000C23286903FB040038BD0248FCE700BF50
:104DC0000C0F0020240F0020FEC00108ABAAAAAAE5
:104DD00085E5010810B5D0E90730C9B2D2B28342E7
:104DE00009D01C788C4204D15C78944201D1987827
:104DF00010BD0333F3E74FF0FF30F9E72DE9F04141
:104E0000D0E904239B1A4F4A9B1053430D4609785F
:104E10000446994203D393214B4801F0D7FBD4E9D0
:104E200001239B1A474A9B1053436978994203D345
:104E30009421454801F0CAFBD4E904239B1A414A56
:104E40009B105343A978994205D3FE2903D095219D
:104E50003D4801F0BBFB6A7829782046FFF7BAFF8E
:104E6000C3B2FF2B064629D029782046FFF782FFE0
:104E7000697807462046FFF765FF314680462046A1
:104E8000FFF778FF414602463846FFF741FD297893
:104E90002046FFF76FFF697806462046FFF752FF6E
:104EA000A97807462046FFF765FF39460246304697
:104EB000FFF72EFD9C21244801F088FBD4E907234D
:104EC000204F9B1A7B437E2B03D99F211E4801F064
:104ED0007DFBD4E90762616A931B7B43521A5743F7
:104EE0000133BB4203EB43080AD8464426622A88B2
:104EF000236A23F8032CAA7803F8012CBDE8F0817B
:104F0000404605F099F9064618B969210E4801F0A6
:104F10005DFBD4E90702131A0A4A5A430023002A08
:104F20000ADDC118B1F800C0F71826F803C0897867
:104F3000013AB9700333F2E705F068F9E6614644D7
:104F40006662D3E7ABAAAAAA85E50108FF2337B5B5
:104F50008DF804300A4B0D461C6823681BB92921C3
:104F6000084801F033FB2A4601A9206807F0C2FD7A
:104F7000012814BF4FF0FF309DF8040003B030BD8E
:104F8000180F002085E5010838B5816800681D46C6
:104F9000144605F002FA0346201845EBE37138BDCC
:104FA00008682DE9F04172281F461FD074280FD0E1
:104FB000632820D1886804F049FF002871F10003BC
:104FC00004460D460EDADD210D4801F0FFFA09E036
:104FD0008B68D3E90045B5F1004F08BF002C01D024
:104FE000A4187D4120462946BDE8F0818868BDE8C7
:104FF000F041FFF7C9BF00244FF00045F2E700BFC2
:1050000085E501082DE9F0410F4606460024FFB270
:10501000FFF7B0FED6E90758454511D02B78BB42C3
:105020000CD169783046FFF78DFE0368692B05D1F6
:1050300083681B6803B198470134E4B20335EBE79A
:105040002046BDE8F0812DE9F34180460F4600255A
:10505000FFF790FED8F81C40D8F8206003340336E0
:10506000FFB2A6421BD0234633F8032D9B78ADF840
:1050700004208DF8063014F8033C9F420DD19DF8B2
:1050800005104046FFF75EFE0368692B05D1836873
:105090005B6803B198470135EDB20334E1E7284678
:1050A00002B0BDE8F0810000836C73B504460D4684
:1050B000164623B94FF48E710B4801F087FACDE9FB
:1050C000006423462A460949094808F079FA01286C
:1050D00007D04FF49171044802B0BDE8704001F070
:1050E00075BA02B070BD00BF85E501082EC2010887
:1050F0003157000838B590F847300446032B0D4669
:1051000004D940F23511064801F060FA94F84730AE
:105110005A1C84F847201C4484F8425038BD00BF14
:1051200085E5010810B590F84730044623B94FF4DF
:105130009D71064801F04AFA94F84730013BDBB212
:1051400084F847301C4494F8420010BD85E50108FE
:10515000CBB2FE2B10B504460AD0FFF70BFE036856
:105160006D2B05D1017A2046BDE81040FFF702BE45
:1051700010BD00002DE9F84304460026114FD4E984
:1051800004239B1A9B107B435FFA86F8434516D98C
:1051900041462046FFF7DCFFD4E90759A9450CD06A
:1051A0002B78434507D169782046FFF7CBFDA978D6
:1051B0002046FFF7CDFF0335F0E70136DFE7BDE816
:1051C000F88300BFABAAAAAA38B50546002495F813
:1051D0004730A34207DD2B1993F842102846FFF70A
:1051E000C9FD0134F3E738BD00232DE9F74FC0E9CD
:1051F000083388461946D8E907594FF0004304465A
:10520000C0E90613C0E90013C0E90213C0E90413A2
:10521000FF208A469B46D2B284F8200001924D4579
:10522000D4E9006720D02B78019A93421AD169788B
:105230004046FFF787FDDDE90C2301464046FFF7B6
:10524000AFFE594508BF50450CD05F4508BF5645D5
:1052500003D0B04271EB070304DA6B78C4E90001B4
:1052600084F820300335DAE7B7F1004F08BF002E8D
:1052700008D0DDE90C23B21A67EB030316461F467C
:10528000C4E90467204603B0BDE8F08FF8B50D46C9
:105290000B4B896906464B434FF47A71B3FBF1F12E
:1052A000FFF754FE0446C7B2B06C03681B6898470A
:1052B000FF2FC6E90E010CBF95F820002046F8BD6F
:1052C00040420F0038B5C36C04460D461BB9BDE81B
:1052D0003840FFF7DBBF806C174903685B6998476C
:1052E000A06C0368DB689847D5E9020104F088FEEA
:1052F0000146124804F004FFA06C03689968D5E9E0
:1053000002238847A06C03681B699847E36C9847A1
:10531000A06C0368DB689847A06C03681B6898471B
:10532000C4E90E0100212046FFF710FEC0B2FE289E
:1053300008BF95F8200038BD4149000839C201086E
:10534000F8B5D1E90667B7F1004F08BF002E054652
:105350000C4608D11AB1BDE8F840FFF797BFBDE889
:10536000F840FFF7AFBF012E77F1000302DA91F8A2
:105370002000F8BD92B121462846FFF787FF94F838
:105380002030C0B28342F4D1D5E90E67D4E90023BE
:10539000964277EB0303B8BFFF20EAE7D0E9142376
:1053A000964277EB0303E6DBFFF78CFFE7E70000AD
:1053B0002DE9F04F8DB004460D46FFF7DBFC036886
:1053C0008046702B04D04FF4A0716B4801F0FEF8BA
:1053D000A06C03681B6898472A46C4E90C01CDE914
:1053E0000001214602A8FFF7FFFE29462046FFF7ED
:1053F00009FE9DF828300646FF2B05D120B940F262
:105400004B115D4801F0E2F8D4E90C0104F0F8FD1D
:1054100001465A4804F074FE3146594804F070FEC3
:105420009DF82810FF297ED100224FF00043CDE9DE
:105430000623DDE90223CDE90423DDE90623CDE9D6
:105440000823A36D13B39847DDE90223D4E91801BB
:10545000B3F1004F08BF002A09D0DDE9062310F19F
:105460000B0641F10007964277EB03030EDAD4E90D
:105470000C23161843EB0107CDE90801CDE90467B9
:1054800004F0D4FD01463F4804F03AFE4FF0000A14
:105490004FF0004BDFF8F89098F8082002A920465A
:1054A000FFF74EFFA36D064603B19847F3B2FF2BFB
:1054B0005AD1DDE90223D4E90E01161A63EB010784
:1054C00039463046CDE90423CDE90667CDE90867C2
:1054D00004F0ACFD0146484604F012FEA36D002B1B
:1054E000DAD0DDE90223D4E918015B4508BF524553
:1054F00009D0DDE9062310F10B0641F100079642C1
:1055000077EB0303C8DAD4E90E23161843EB01073F
:10551000CDE90801CDE9046704F088FD014619488A
:1055200004F0EEFDB8E72046FFF70CFCD0E9006779
:10553000DDE9020104F064FD3A46034631461248B3
:1055400004F0DEFDD4E90C23DDE90201801A61EBF1
:1055500003010F460646CDE9066704F067FD0146E4
:105560000A4804F0CDFD64E729462046FFF76BFDAD
:1055700030460DB0BDE8F08F85E501080CC101088B
:105580002BC1010888C1010846C101086AC1010890
:10559000A0C1010870B504460D46FFF7EBFB036898
:1055A0006D2B11D0702B09D0612B14D1836894F826
:1055B000411094F84000BDE8704018472946204645
:1055C000BDE87040FFF7F4BE034840F22F1100F031
:1055D000FDFF4FF0FF3070BD85E501082DE9F04774
:1055E00090F828300446FF2B04D14FF4E5714A4867
:1055F00000F0ECFF94F828102046FFF7BBFB426850
:105600000178464804F07CFD94F82830DFF81C81CE
:1056100084F8463094F846102046FFF7ABFB036849
:1056200005466D2B204694F846100BD1FFF762FD1E
:10563000297A204684F84610FFF79CFB2046FFF7A6
:10564000C3FDE7E7FFF7A6FFC3B2FF2B06460BD16A
:1056500040F2DF11304800F0B9FF40F2DF11304B6B
:10566000304A314812F090FE024694F84610204627
:10567000FFF7B0FBC5B2FF2D09D140F2E511264876
:1056800000F0A4FF264B274A40F2E511E9E794F821
:105690004610FE2D204621D1FFF744FD0746014666
:1056A0002046FFF767FB324639462046FFF792FB5C
:1056B000C5B2FF2D0DD131462046FFF743FB40F226
:1056C000F111154800F082FF154B164A40F2F11116
:1056D000C7E72046FFF778FD3946DAE7FFF74AFBD0
:1056E000314607462046FFF72DFB294681462046D6
:1056F000FFF740FB8246404604F002FD5246494611
:105700003846FFF705F994F8463084F8416084F88C
:10571000403084F846507DE785E50108C8C101089E
:105720000AB8010869C20108E6C101081EC20108E1
:1057300008B504F049FEFFF789FAFFF74FFFD0B52F
:105740001F461646FFF7FEFA03688468742B01D0E3
:10575000FFF7F0F8C4E90067D0BD0000836C10B516
:10576000044623B94FF42771024800F02FFFA06CC4
:1057700010BD00BF85E50108FF23054A1370054AE7
:105780001370054A1370054A1370054A1370704769
:10579000200F00201E0F00201C0F00201F0F0020D4
:1057A0001D0F002010B50446006807F00FFC2046CE
:1057B00010BD00002DE9F3480AF07AFC4FF6FF71A6
:1057C000344A13888B421CBF01331380FFF73EFA23
:1057D000FFF7C4FF03681B6898472F4B83465A782E
:1057E0008C46D2B92D4A1289BAB12D4C30CCB5F1C4
:1057F000004F08BF002C0ED0844275EB0C010CDA70
:10580000BBEB0406274C6CEB05075443E517A64297
:1058100077EB050201DB01225A700022ADF804206B
:105820008DF806205A782AB101228DF804201C4AEE
:10583000C2E900BC1A781C4B92B101228DF80520F8
:105840001A701A4A1A491B48019B12780978006895
:105850000AF098FCD8B1184B187802B0BDE8F0886F
:105860001A700E4B9B89002BEBD04AF6C0025A43AC
:10587000124CD31730CCBBEB04006CEB050190420B
:1058800071EB0303A4BF01238DF80530D9E70C4B5E
:10589000E2E700BFE20F0020C00F0020CC0F002085
:1058A0004002002080510100C90F0020C30F0020DA
:1058B000C20F0020BC0F00201C0F0020300200206F
:1058C0001E0F0020104B1B8913B9104B187870471E
:1058D0000F4BD3E90023B3F1004F08BF002AF4D1E6
:1058E0000C4A13780133DBB2012B1370EDD800237F
:1058F000094A1370094A1370094A1360094A137060
:1059000001235370084BE1E7CC0F00201C0F00204F
:1059100038020020F40F0020C30F0020C20F002027
:10592000BC0F0020C00F00201F0F00201FB57023E8
:10593000CDE90131002301A98DF80C30FFF7A0F962
:1059400005B05DF804FB00002DE9F04F4A4B85B02F
:105950001A780446002A40F08B80012747491F70BF
:10596000FFF7E8F8464B474918702046FFF7E2F882
:10597000DFF868A144498AF800002046FFF7DAF80A
:10598000DFF85C910A22002389F800003F4901A852
:10599000FEF7E8FF01A92046FFF76AF83C4E3D49B3
:1059A00030702046FFF7C6F83B4B3C491870204644
:1059B000FFF7C0F83A4B3B4918702046FFF7BAF89A
:1059C000394B3A4918702046FFF7B4F8384B394A3A
:1059D000187039492046FAF7E0FFDFF808B1374A76
:1059E0008BF8000036492046FAF7D7FF35490546BF
:1059F0002046FFF79BFF70230193334B804601A99C
:105A0000204602938DF80C70FFF73AF907462F4AAB
:105A10002B4612789BF800102046FAF7C9FF434640
:105A20009AF8002029462046FAF7C2FF3B4699F82B
:105A3000002029462046FAF7BBFF2B463278414624
:105A40002046FAF7B5FF2B46327839462046FAF75A
:105A5000AFFF1F4A2B46127829462046FAF7A8FFC7
:105A60001C4B1D4A1B78127829462046FAF7A0FFE6
:105A700005B0BDE8F08F00BFF50F0020E1C20108BE
:105A8000C40F0020EBC20108F6C2010802C30108DE
:105A9000A90F00200FC30108E10F00201DC301085A
:105AA000E00F002029C30108E40F002036C30108DD
:105AB000E50F0020B557000844C30108B561000890
:105AC0004EC3010862C3010875C301081C0F002002
:105AD0001F0F00201D0F0020200F0020C80F0020E6
:105AE000A80F0020C60F002030B5044685B00D4633
:105AF000FFF72AFF6D22064B01A91B782046CDE94E
:105B000001258DF80C30FFF7BBF805B030BD00BFA4
:105B1000C60F00202DE9F84F424B434D1A6804464A
:105B200012F0010F01BFFF222A7001221A602B78A8
:105B3000FF2B73D1FFF708FF3C4A3D492046FAF797
:105B40002CFF3C4A28703C492046FAF726FF3B4F81
:105B50003B4A38703B492046FAF71FFF3A4E3B4913
:105B600030702046FFF7C0FF394982462046FFF7D4
:105B7000DDFE384983462046FFF7D8FE8146364A87
:105B80003B78127829782046FAF712FF334ADFF87B
:105B9000E0803378127829782046FAF709FF3378C5
:105BA00098F8002039782046FAF702FF2B7898F809
:105BB000002031782046FAF7FBFE294A5B4612782E
:105BC00039782046FAF7F4FE26493B780A782046D1
:105BD0005946FAF7EDFE244A4B46127839782046AA
:105BE000FAF7E6FE1F493B780A7820464946FAF75D
:105BF000DFFE1A4A5346127831782046FAF7D8FE6B
:105C0000337898F8002051462046FAF7D1FE174A1B
:105C10002B78127831782046FAF7CAFE2878BDE84A
:105C2000F88F00BFA40F0020F70F0020455F000889
:105C3000C5C30108955C0008CFC30108C50F00204B
:105C4000C5580008D9C30108C70F0020E3C30108E5
:105C5000EFC30108FDC30108C40F00201F0F00207F
:105C6000C80F0020A90F00201E0F00201C0F0020CD
:105C7000200F002070B50D460446FEF7E7FF0449EB
:105C800022462B46BDE870400978FFF758BD00BF9B
:105C9000A90F0020F8B5454D2B682F4601332B6026
:105CA0000AF006FA0AF032FA44F620600AF016FA10
:105CB00041780646042908D03D4804F021FA3046D0
:105CC00004F0A4FA0120002147E00478466804F0BB
:105CD0009DFA012C4AD12B68042B0CD90FF060FAE5
:105CE000037843B1334B9B6803B1984740F29B1153
:105CF000314800F06BFC3B681E22013BDBB21E2BDF
:105D000028BF1E23A3F12005C3F1200402FA05F1E8
:105D100022FA04F4002521434FF4E14402FA03F08F
:105D20008D4208BF84421CD3002908BFB0F5616FC3
:105D300004460D4615D2B0F5167F71F1000313DA53
:105D40003C2871F10003ACBF11460A21002004F089
:105D500024FB0346201845EBE371FFF78BFF174B3D
:105D60000BE04FF41671F1E73C21EFE7032C06D16D
:105D700030460021FFF77EFF114B1878F8BD74B94B
:105D80002C600AF04FF9FEF761FFFFF7E7FC0368AC
:105D90001B6898470B4BC3E900010B4BEDE70B4821
:105DA000214604F0ADF90A208DE700BFF00F002076
:105DB0008EC20108F80F002085E501081E0F0020A3
:105DC000C80F002030020020200F0020AFC20108C1
:105DD000054B1870054B1A700022054B1960054BD6
:105DE0001A705A70704700BFC30F0020C20F002006
:105DF000BC0F0020C00F002008B50AF06DFAC0B239
:105E0000DE2828BFDE2008BD002337B54FF47A74A2
:105E100001930B4B60431D68B0FBF4F42B681BB976
:105E20002921084800F0D2FB224601A9286806F083
:105E300061FE012814BF0020019803B030BD00BFEF
:105E4000AC0F002085E50108022818BF00200AF0E9
:105E50003BBB00002DE9FF412E4B05461F78002F6C
:105E600054D1012204AE06F8017D1A7009F0B4FD88
:105E700007230C22284CCDE9003228493246231D45
:105E800028460EF0F5FF0E23254928466371A371BD
:105E90004FF47A7827610EF0AFFF04F108036070C9
:105EA000324620492846CDE900780FF001F842F249
:105EB00010733246CDE900731B4904F10A032846EA
:105EC0000EF0F6FF194928460EF096FF04F10C0378
:105ED000A070324616492846CDE900780EF0E8FF5A
:105EE000144928460EF088FF9DF80F30E07053B13A
:105EF000114804F005F9114B1B6803B19847602164
:105F00000F4800F063FB2069FFF79EFF04B0BDE877
:105F1000F08100BFF60F0020CC0F002089C30108DC
:105F20008CC3010890C3010899C301085DE401080E
:105F3000A2C30108ADC30108B2C30108F80F0020D5
:105F400085E5010870B5294BC0B21B78984206D18F
:105F50000FF026F90EF07CFF254B187870BD254C0C
:105F60000FF01EF9FFF776FF94F905000CF036F8F4
:105F70000AF0C6F920790BF0FFFF0AF0B7F91E4DC1
:105F8000A0790AF0C5F960780AF098FA2A6812F048
:105F9000010213D10421194E08463260716006F0E7
:105FA0002BFC306018B95121154800F00FFB01237C
:105FB000144A154911482B6010F0EAFE134B1A6879
:105FC0000AB90E4A1A60FEF741FEFFF7C7FB0368E5
:105FD0001B68984701220E4BC3E900010D4B5A7212
:105FE000E3780BB10C4BB8E70C4BB6E7C70F0020BA
:105FF000200F0020CC0F0020A00F0020E80F002071
:1060000085E5010800000020A5570008AC0F00201E
:1060100030020020B00F0020C40F00201F0F00200E
:10602000034B93F82F30022B0CBF02200020704747
:10603000D0020020F8B51D4600234171BDF81810AC
:1060400004460360C180174602B115B9237120468A
:10605000F8BD0749284610F04BF8064610B92071E4
:106060002660F4E72A46394612F0ABFB2571F7E7C4
:1060700018EC010810B50446006808B110F03AF8B1
:10608000204610BD2DE9FF4142F210700AF026F8BB
:106090000546002875D00778032F03D140680021FA
:1060A000FFF7E8FD384ED5F8A040336823B940F239
:1060B000C911364800F08AFA002C56D00022344B21
:1060C0001A80D4E91C23134318D0324BD3F8008034
:1060D00007F0B8FC01463048C047FEF7B7FDFFF7B0
:1060E0003DFB03685968D4E91C238847D4E91C2385
:1060F0002A49C1E900232A49C1E90023FEF7A6FD88
:10610000FFF72CFB03681B689847264B264AC3E918
:106110000001237AC3F3C0031370637F2BB3237F83
:106120001BB3224908200FF0D9FF804630B16289A5
:10613000237F617F0092A26EFFF77CFFCDF80C8079
:10614000B8F1000F11D0002330681A4603A9006887
:1061500006F076FB012808D0039C34B12046FFF7F7
:1061600089FF082120460FF0C7FF2B7A13B10022C8
:106170000F4B1A7028460BF0F1FC384604B0BDE80E
:10618000F0810127F9E700BFAC0F002085E5010889
:10619000E20F0020D0020020D4C201083802002003
:1061A0004002002030020020E60F002018EC010819
:1061B000C90F0020002310B5114C84F8343009F0C9
:1061C00055FF08B109F074FFFFF75CFF012809D9FA
:1061D00003280AD00B484FF4317100F0F7F94FF063
:1061E000FF3001E0084B187810BDFFF719FF0228B7
:1061F00009BF0123054B84F83430054BF3E700BF9A
:10620000D002002085E50108200F0020C80F0020E3
:10621000A80F0020FF2300210D4A13700D4A1370B0
:106220000D4A13700D4A13700D4A13700D4A137006
:106230000D4A13700D4A13700D4A13700D4A1370F6
:106240000D4A13700D4AC2E900111372704700BF66
:10625000C60F0020C50F0020C70F0020E10F00204F
:10626000E00F0020E50F0020E40F0020C40F002005
:10627000C80F0020A80F0020A90F0020B00F002099
:10628000034AC0E900210022027242728272704702
:106290004849F8F9437A10B504461BB92121094849
:1062A00000F094F9207A08B9002010BDA37A002BE1
:1062B000FBD0606803681B6898470028F4D000236F
:1062C000A372F2E785E5010830B5044685B08DF884
:1062D0000F10FFF7DFFF9DF80F30606803F00F032A
:1062E0008DF80F3003685B68984768B100216068DB
:1062F000237802680091D5680DF10F010122A847AB
:10630000606803689B68984705B030BD30B50446A7
:10631000002585B0FFF7BEFF60688DF80F50036859
:106320005B68984760B1606863780268009515699A
:106330000DF10F010122A847606803689B68984728
:106340009DF80F0000F00F0005B030BD7FB504468A
:106350000E46FFF79FFF606803685B689847054635
:1063600020B30221637860688DF80C30E3788DF8F3
:106370000D3002680091D568A378012203A9A847CF
:106380000546606815B90123A3720CE04FF4004183
:10639000026800911569A37803223146A847054693
:1063A0006068002DEFD003689B689847284604B0CA
:1063B00070BD13B501A90446FFF7C8FF70B19DF881
:1063C000043043B99DF80530082B04D19DF8063000
:1063D0000BB901232372207A02B010BD2072FAE7B4
:1063E000002310B543720372837204464068036849
:1063F0001B68984730B1012320466372BDE8104006
:10640000FFF7D7BF10BD70B5164605460C46FFF71F
:106410007DFF3EB140EA04012846BDE87040C9B2A4
:10642000FFF752BF20EA0401F6E700002DE9F0472C
:1064300041488AB003F064FE07F012FB2425079060
:1064400007993E4803F05CFE0798684303F0F4FEAA
:1064500004463B4803F054FE94B107990DEB050246
:10646000204607F077FE0023DFF8F0A0354F0790B5
:106470000893089A079B9A421DD3204603F0C6FE54
:1064800006F0DCF8044606F0E7F8214602462E48FE
:1064900003F036FE2D4B2E4819889A888B1A03F08C
:1064A0002FFE2C4B1B6803B198472B4803F028FEA6
:1064B0000AB0BDE8F087089B05FB03431B7B042B58
:1064C00098BF1AF80320099B88BF3F22642B83BF23
:1064D0006420B3FBF0F30899002382BF05FB014160
:1064E0008969B1FBF3F308990898DDF820C0DDF85D
:1064F00020E0DDF82080DDF8209005FB004005FB62
:106500000949D9F81C6005FB0141CDE9033605FBBB
:1065100008439B69029305FB0E439B68019305FBAF
:106520000C431B8C009303694968384603F0E8FD6F
:10653000089B013308939CE711C401081DC401089E
:1065400028C401085DC40108B2B80108161F002064
:106550008FC40108801000200ABA01080CC4010889
:10656000014B1860704700BF9C10002073B5124C9F
:10657000064623780D46114A1BB913780BB172B643
:10658000FEE70123002113700D48642212F03DF94B
:106590002B4600960B4A6421094813F05BF80A4B1E
:1065A0001B6803B198470125054E304603F0ECFD0A
:1065B00072B62570F9E700BF781000200C1000209B
:1065C0000E100020C6C401089C100020F7B5184C1E
:1065D000064623780D46174A1BB913780BB172B6DD
:1065E000FEE70123002113701348642212F00DF915
:1065F0002B460096114A64210F4813F02BF8104BDC
:106600001B680BB10C4898470E4B1B6803B19847A9
:106610000125094E0C4F304603F0B6FD384603F015
:10662000B3FD72B6094B257000BF013BFCD1F2E708
:10663000791000200D1000200E100020EEC401087B
:10664000081000209C100020FDC40108FFFF0F006F
:10665000F8B5DFF898C003681A4FCCF800304368EB
:10666000194E3B608368194D3360C368184C2B602A
:10667000036918492360436982690B60164BC0693E
:106680001A60164A1060DCF8000038683068286824
:1066900020681C460968124D1968124E126864225F
:1066A0000021284612F0B1F82368324664212846BA
:1066B00012F0D0FF284603F067FD0B4B00BF013BF3
:1066C000FCD1ECE78C1000209410002098100020E2
:1066D00090100020741000207C10002084100020F6
:1066E0000E100020B3C40108FFFF0F008810002027
:1066F000074B1B6803B198471EF0040F0CBFEFF364
:106700000880EFF309808169004A1047516600084C
:106710009C100020002103E00A4B5B5843500431D9
:1067200009480A4B42189A42F6D3094A02E000236C
:1067300042F8043B074B9A42F9D300F00DF8FBF7FF
:106740003FF8704728EF010800000020780700207C
:1067500078070020CC1F0020314B82B01A6842F429
:1067600080721A6099682F4A0A409A601A6822F06B
:10677000885222F001121A601A6822F480221A60EC
:106780009A6822F47D029A600022DA6001921B6806
:1067900013F4007318BF01230193019B012B37D120
:1067A0004FF48051204B1A68A3F5806322F0010258
:1067B000C3F80024D3F8002422F00202C3F8002416
:1067C000D3F8002422F00402C3F800245A6A42F0ED
:1067D00080525A62154A11605168C906FCD49A6801
:1067E0009A609A689A609A689A605A6822F460423D
:1067F0005A605A6842F440425A609A6822F0030292
:106800009A609A689A60064A936813F00C0FFBD15D
:106810004FF00062064B9A60064ADA6002B0704799
:10682000003802400CC0FF88003C0240007000406D
:1068300000ED00E00003FA0570B5064688B02E486A
:1068400001F0C6FC2D4B1A680092009A91073CD5C6
:1068500001214FF4007001F015FF012001F008FD47
:10686000274A536843F400335360A2F53742536814
:106870001B07FCD50024012502A801F0E3FC02A9B6
:106880001D488DF80D4006948DF81C508DF80C4075
:1068900001F0B2FC2A4606233146174801F0F4FC09
:1068A0002946154801F0DAFC0221134801F07EFD6B
:1068B000114801F06DFD134D01940F4C022120464B
:1068C00001F06EFD58B108B070BD1A6842F00102C7
:1068D0001A60009A9207BBD41A680092F9E7019BEC
:1068E00001330193019BB3F5805FE7DB3821284634
:1068F000FFF76CFEE2E700BF0024014000380240D1
:106900000027014085E5010808B5002001F0B0FC32
:106910000021074801F0A2FC00214FF4007001F0B3
:10692000B1FE044A136823F00103136008BD00BFE1
:10693000002401400038024013B50723012201461C
:10694000114801F0A1FC02210F4801F02FFD0E4873
:1069500001F01EFD00230D4C019302210A4801F0B5
:106960001FFD28B1084802B0BDE8104001F015BD78
:10697000019B01330193019BB3F5805FEDDB4C215B
:106980002046FFF723FEE8E70024014085E50108E3
:1069900070B506460825FFF74FFF00243046FFF785
:1069A000CBFF013D0444F9D1FFF7AEFFC4F3CF00A4
:1069B00070BD00000000000008B51120FFF7E8FFDF
:1069C00011F0C4F80146084811F0CCF910F0A6FC0B
:1069D00003A3D3E9002310F0F9FC10F0B1FF08BDC8
:1069E0002FDD24068195F33F00F07F450F4A536A5F
:1069F00043F0805353620E4B1A465968C906FCD4C3
:106A00001B68022823F4C05306D143F4C05313601B
:106A10005368DB06FCD47047012802D143F480534D
:106A2000F5E70028F3D143F40063F0E700380240B3
:106A30000070004010B50C4B5A68D206FCD41C689C
:106A400014F4C05F0BD114F480500AD114F4006424
:106A500004D106482A21FFF7B9FD204610BD0220C7
:106A6000FCE70120FAE700BF0070004085E501085F
:106A700038B50546012001F0A9FC022D01BF154AD9
:106A8000136843F001031360134B1A6842F4803219
:106A90001A601A689203FCD542F690529A6099687F
:106AA0009142FCD19A6842F002029A600A4B9C68BB
:106AB00014F00804FBD14FF480321A60074B084AE7
:106AC00028461A60FFF792FF2046BDE8384001F0E3
:106AD00071BC00BF003C0240003802404802002068
:106AE00000093D0038B50546012001F06FFC022D7C
:106AF00001BF144A136843F001031360124B1A6874
:106B000042F480721A601A689205FCD55A6822F421
:106B1000604242F440425A6000229A600A4B9C68EC
:106B200014F00C04FBD14FF480721A60074B084A32
:106B300028461A60FFF75AFF2046BDE8384001F0AA
:106B400039BC00BF003C024000380240480200202F
:106B5000D0FE3F000C4B5A6B900513D45A6A42F09A
:106B600080525A62094A116841F480711160596B70
:106B700041F480715963596B8905FCD5136823F47E
:106B800080731360704700BF0038024000700040FF
:106B9000054B5A6B910706D45A6B42F001025A63B7
:106BA0005A6B9207FCD5704700380240094B5A6A6D
:106BB00042F020025A629A6942F020029A619A6970
:106BC00022F020029A610022A3F509331A801A8567
:106BD0005A627047003802401521023800224843AB
:106BE0000121064B1A85D86299825A621A8219804D
:106BF0001A8AD207FCD500221A8070470014004080
:106C0000002349F6FE7282B00193019B934201DD9D
:106C100002B07047019B01330193F6E7002340F671
:106C2000FE7282B00193019B934201DD02B0704776
:106C3000019B01330193F6E7002382B00193019B8E
:106C4000B3F5CC7F01DD02B07047019B0133F5E75E
:106C5000D0B1012801D1FFF7EFBF0C4B00211A681A
:106C60004FF47A73B2FBF3F2094B013A92B21A85F0
:106C700001220138D8629A82596219821A801A8ACE
:106C8000D207FCD500221A80704700BF48020020BE
:106C90000014004000F1774303F57803B3F5804F0B
:106CA0002DE9F04106460C4617462DD202F1F73386
:106CB00003F608030344B3F5804F25D2FFF7BAFE6D
:106CC000804610B10020FFF791FE01F097FB0125EF
:106CD0002744361BA7420AD101F0A0FBB8F1000FF0
:106CE00002D04046FFF782FE2846BDE8F08141F61B
:106CF000027001F09BFB301914F8011B01F0F2FB4C
:106D0000042818BF0025E5E70025EDE710B50C467F
:106D100000F1774101F57801B1F5804F0DD202F114
:106D2000F73303F608030344B3F5804F05D2014659
:106D3000204611F046FD012010BD0020FCE70000B8
:106D400008B5114B984215D003F58063984213D0D3
:106D500003F58063984211D003F5806398420FD009
:106D600003F5006398420DD0084B094A14210948E5
:106D700011F00AFB002008BD0120FCE70220FAE721
:106D80000320F8E70520F6E7000002405FC5010890
:106D900019C5010878C501080F2808B505D9094BA0
:106DA000094A3B21094811F0EFFA012303FA00F0E8
:106DB000C043074A51680140516013681840106091
:106DC00008BD00BFB7C5010823C5010878C5010883
:106DD000000401400F292DE9F84F82460D469346E5
:106DE0001F4605D95A4B5B4A54215B4811F0CCFA37
:106DF0004FF0010909FA05F900F0B8F86FEA090344
:106E0000564E032D7268564C02EA030272603268D5
:106E100003EA0203534A3360136A43F00103136227
:106E20002ED80F22A3684FEA850802FA08F223EA57
:106E30000203A3605046FFF783FFA36800FA08F03F
:106E40001843A0601BF0020F18BFB368464A1CBF6E
:106E500043EA0903B3601BF0040F1EBFF36843EA63
:106E60000903F360336843EA090333603B01DBB293
:106E7000002D45D182F8063340231360BDE8F88F1A
:106E8000072D13D80F22A5F10408E3684FEA8808FC
:106E900002FA08F223EA0203E3605046FFF750FFCC
:106EA000E36800FA08F01843E060CBE70B2D13D835
:106EB0000F22A5F1080823694FEA880802FA08F2B0
:106EC00023EA020323615046FFF73AFF236900FAE1
:106ED00008F018432061B5E70F22A5F10C0863699B
:106EE0004FEA880802FA08F223EA02036361504677
:106EF000FFF726FF636900FA08F018436061A1E715
:106F0000012D03D182F807338023B6E7022D04D187
:106F100082F808334FF48073AFE7032D04D182F871
:106F200009334FF40073A8E7042D04D182F80A3323
:106F30004FF48063A1E7092D04D882F817334FF48A
:106F400000039AE782F828334FF48073536095E783
:106F5000C3C501083EC5010878C501080004014009
:106F6000000001400038024000E100E0144B98426C
:106F700005D1144AD36943F00103D3617047124B22
:106F8000984204D10F4AD36943F00203F5E70F4B4F
:106F9000984204D10B4AD36943F00403EDE70C4B4C
:106FA000984204D1074AD36943F00803E5E7094B47
:106FB0009842E3D1034AD36943F02003DDE700BFE1
:106FC0000000024000380240000402400008024075
:106FD000000C0240001402400323490010B58468ED
:106FE0008B4024EA030484600124022A04FA01F499
:106FF00007D0032A0DD0012A07D183682343836079
:1070000003E083688A401A43826083681C4384607B
:1070100010BD82681343F2E70F29F8B504460F4606
:1070200015461E4603D94B211948FFF7CFFA2046D3
:10703000FFF79CFF03237A009340DB43216819404C
:1070400021600121D4F800C001FA02F04CEA000CE2
:10705000B940C4F800C009B266B1A688314389B20C
:10706000A180E168012D03EA0103E36006D0022D4F
:1070700008D0F8BDA68826EA0101F1E7E3680343DA
:10708000E360F6E7E36805FA02F21A43E260F0E72C
:1070900085E501080F2970B505460C46164603D94B
:1070A0006B210E48FFF792FA2846FFF75FFF032394
:1070B00061008B40DB43EA68012E02EA0302EA60CA
:1070C00005D0022E03D02A6813402B6070BDEA68F9
:1070D00006FA01F11143E960F5E700BF85E5010813
:1070E0000F2910B505D9074B074A8121074811F030
:1070F0004BF9FFF73BFF4B00032102689940114316
:10710000016010BDB7C50108CFC5010813C601084D
:107110000F2938B50446154605D987211B4B1C4A53
:107120001C4811F031F90F2A03D91B4B184A88214A
:10713000F6E7FFF71BFF07294FF00F0318D8006A87
:107140008A00934020EA03032362236A05FA02F2CD
:107150001A4322620322236849008A4023EA020379
:1071600023600223226803FA01F11143216038BD34
:10717000A1F10802406A9200934020EA030363628F
:10718000636A95401D436562E4E700BFB7C5010827
:10719000E2C5010813C6010800C60108012303FA6D
:1071A00001F189B201837047012303FA01F189B229
:1071B00041837047012303FA01F189B20AB10183C7
:1071C000704741837047008A084100F00100704712
:1071D0000F2938B505460C4603D9B4210548FFF7F9
:1071E000F5F928686400E04000F00300431E5842AF
:1071F000584138BD85E50108808A084100F001004A
:107200007047000010B5084C23681BB9012005F039
:10721000BBFB206023682BB9BDE810403621034832
:10722000FFF7D4B910BD00BFA010002085E501080C
:1072300010B50B4C22681AB93C210A48FFF7C6F971
:10724000206842F2107105F0E7FC01280CBF012410
:10725000002403D040210348FFF7B8F9204610BDB1
:10726000A010002085E5010810B5074C22681AB966
:1072700051210648FFF7AAF9002320681A46BDE805
:107280001040194605F0DCBAA010002085E5010881
:1072900010B50446FFF7B6FFFFF7CAFF21461022DC
:1072A000034801F0FBFE0446FFF7DEFF204610BD59
:1072B0000054004010B5FFF7A5FFFFF7B9FF01F03C
:1072C000A5FE0446FFF7D0FF204610BD08B51346C3
:1072D0000A460146034801F0D9FA003018BF0120E0
:1072E00008BD00BF0054004008B513460A460146D9
:1072F000034801F0CBFB003018BF012008BD00BFE0
:107300000054004008B513460A460146034801F000
:1073100099FC003018BF012008BD00BF0054004098
:1073200008B513460A460146034801F01BFD00302C
:1073300018BF012008BD00BF0054004008B5134627
:107340000A460146034801F065FD003018BF0120E0
:1073500008BD00BF005400400123064A8340516924
:10736000194205D05361044B53F8203003B118473C
:10737000704700BF00040140A41000200F2838B55A
:1073800004460D4603D926210348FFF71FF9034B96
:1073900043F8245038BD00BF85E50108A410002043
:1073A0000020FFF7D9BF0120FFF7D6BF0220FFF76B
:1073B000D3BF0320FFF7D0BF0420FFF7CDBF08B530
:1073C0000920FFF7C9FF0820FFF7C6FF0720FFF7D6
:1073D000C3FF0620FFF7C0FFBDE808400520FFF708
:1073E000BBBF08B50F20FFF7B7FF0E20FFF7B4FFB4
:1073F0000D20FFF7B1FF0C20FFF7AEFF0B20FFF7CA
:10740000ABFFBDE808400A20FFF7A6BFFEE7FEE796
:10741000FEE7FEE7FEE7FEE7FEE7FEE7FEE7FEE744
:10742000FEE7FEE7FEE7FEE7FEE7FEE7FEE7FEE734
:10743000FEE7FEE7FEE7FEE7FEE7FEE7FEE7FEE724
:10744000FEE7FEE7FEE7FEE7FEE7FEE7FEE7FEE714
:10745000FEE7FEE7FEE7FEE7FEE7FEE70A23B0FBF6
:10746000F3F203FB120040EA0210C0B270470000C2
:10747000CA22024B5A6253225A62704700280040C7
:10748000014B1860704700BFE41000204FF4003239
:107490000F4B10B50F4C5A61E368DB0503D4302164
:1074A0000D48FFF793F8FFF7E3FF4FF40072A3686E
:1074B00023F48853A360094BC3F88420FF2363623D
:1074C000074B1B6813B1BDE81040184710BD00BF43
:1074D000000401400028004085E5010800E100E0CB
:1074E000E41000202DE9F04F9846374B85B01B780B
:1074F000824691469DF838709DF83C602BB9334B1D
:10750000334A8C21334810F03FFF431E1E2B59D8BD
:107510000C2957D8A2F5FA63632B53D8B8F1170F8B
:1075200050D83B2F4ED83B2E4CD802F13000C0B281
:10753000FFF794FF83460846FFF790FF0446504646
:10754000FFF78CFF40F400554046FFF787FF45EA00
:107550000B4545EA042504463846FFF77FFF000245
:1075600040EA04443046FFF779FF20431A4CFFF706
:107570007FFFE36843F08003E360E3685B06FCD5CC
:1075800065602060E36823F08003E360124BDA68F3
:107590009206FCD5FF2204A85A6200F80C6D8DF803
:1075A00007A08DF80810ADF809908DF806808DF8C9
:1075B000057002F0E2FC094BC3E90001012005B0AF
:1075C000BDE8F08F0020FAE7E810002083C601082C
:1075D00077C601088CC6010800280040F010002082
:1075E00037B50578C4788378B0F80520017901951E
:1075F000407800902046FFF775FF03B030BD0000D3
:1076000038B52B4B04461B781BB9E4212948FEF7FB
:10761000DDFF294AD36823F02003D360D3689B069B
:10762000FCD513685268C2F30741080900EB8000DB
:1076300001F00F0101EB4001C9B201F5FA61A4F8B4
:107640000510C2F30721C1F300108500284401F0A2
:107650000F0101EB4001D2B22171C2F3011101EB24
:10766000810102F00F0202EB4102E270C3F3074214
:10767000C2F3011101EB810102F00F0202EB4102A2
:10768000A270C3F30722C2F3021101EB810102F0E1
:107690000F0202EB4102DBB26270C3F3021202EB93
:1076A000820203F00F0303EB4203237038BD00BFD7
:1076B000E810002085E50108002800401FB501A85A
:1076C000FFF79EFF01A802F058FC05B05DF804FB2F
:1076D00008B5FFF73FFA1B4A136843F48073136041
:1076E000FFF7C6FE184A536B23F4403343F482037A
:1076F0005363164BDA6842F08002DA60DA685106AA
:10770000FCD5FF221A611A6942F4FE021A619A68D6
:1077100022F040029A609A6822F44C529A60DA6829
:1077200022F08002DA60094BDA689206FCD5FF226B
:107730005A620122064B1A70FFF7C0FF054BC3E9DE
:10774000000108BD007000400038024000280040E1
:10775000E8100020F010002008B5094B1B7823B971
:1077600040F21F110748FEF731FFFFF781FE064B7D
:107770009A6822F480729A60FF225A6208BD00BFA4
:10778000E810002085E501080028004008B5144BEA
:107790001B7833B9134B144A40F22711134810F0E9
:1077A000F3FDFFF765FE124BDA6822F48072DA60AF
:1077B000104A916841F400319160116841F4003140
:1077C0001160F0210C4A82F829134FF400715160C6
:1077D0009A6842F488529A60FF225A6208BD00BF3C
:1077E000E810002083C6010850C601088CC60108B5
:1077F000002800400004014000E100E0F8B51E460A
:10780000194B17461B7833B9184B194A4FF4A57119
:10781000184810F0B9FD184CFFF72AFEA56825F4AA
:107820008075A560E56825F48075E560FFF716FEB4
:1078300005460846FFF712FE000440EA0561384697
:10784000FFF70CFE05463046FFF708FE084340EA06
:107850000520E368DB07FCD5FF23E0616362BDE838
:10786000F840FFF793BF00BFE810002083C601086F
:1078700065C601088CC601080028004003784278DC
:107880008178C078FFF7BABF38B50D46044604F0DA
:1078900091FD1F4A136823F00103136004F0AAFD51
:1078A00025B11C4A536843F00603536072B6BFF318
:1078B0004F8FBFF36F8F184A0120136823F0030323
:1078C00043F4007343F00103136000F08BFD134B8E
:1078D0001A6942F004021A6130BF1A6922F00402E8
:1078E0001A610F4B0F4A1B6893420AD10220FFF71F
:1078F000F9F8074A136843F00103136004B162B654
:1079000038BD094A9342F4D10220FFF7B1F8F0E7FD
:1079100010E000E0002004E00070004000ED00E016
:1079200048020020D0FE3F0000093D0062B67047CB
:1079300000220E4B10B51A700D4A0E4C13882046CB
:1079400023F040031B041B0C13800D210222FFF7C0
:10795000A1FB204602220E21FFF79CFB2046BDE83A
:10796000104002220F21FFF795BB00BFF810002046
:107970000038004000040240284A38B5136A054622
:1079800043F480531362052225480C461146FFF745
:10799000BFFB052206212248FFF7BAFB052207217B
:1079A0001F48FFF7B5FBC5B1022205211C48FFF7B0
:1079B00013FB022206211A48FFF70EFB02220721C1
:1079C0001748FFF709FB012C21D144F4517401221F
:1079D000144B1C80144B1A7038BD2A4605211048E0
:1079E000FFF7FAFA2A4606210D48FFF7F5FA2A466C
:1079F00007210B48FFF7F0FA012C05D0022C03D029
:107A0000032C14BF0024032444F45974DFE7022C30
:107A1000DBD0032C0CBF03240024D6E7003802403F
:107A20000000024000300140F910002000220E4BFF
:107A300010B51A700D4A0E4C1388204623F04003EF
:107A40001B041B0C138005210222FFF723FB204699
:107A500002220621FFF71EFB2046BDE8104002224D
:107A60000721FFF717BB00BFF910002000300140CD
:107A700000000240064B074A988111781A4618897F
:107A8000C00701D40029FAD19089C0B2704700BF65
:107A900000300140F9100020054AD36823F4E06368
:107AA0001B041B0C43F0BF6343F40033D3607047E7
:107AB00000ED00E020220021114B10B5C3F8842016
:107AC000104B114C1A6A204642F480421A625A69DD
:107AD00042F480425A615A6922F480425A610B4A48
:107AE00091811A6A092122F480421A620222FFF768
:107AF000D1FA2046BDE8104002220A21FFF7CABA97
:107B000000E100E00038024000000240003801407F
:107B100010B50B4C40F22551204600F090FE48B1C4
:107B2000204600F06AFE074BC0B21B6833B1BDE8C7
:107B300010401847A388044ADBB2137010BD00BF81
:107B400000380140FC100020141F002010B504462E
:107B50008021084800F06DFE0028F9D02146054834
:107B600000F047FE034C4021204600F062FE002852
:107B7000F9D010BD0038014010B5441E14F8010FB3
:107B800000B910BDFFF7E2FFF8E7000008B50248B2
:107B900000F033FEC0B208BD003801402DE9F043CB
:107BA0008846012189B08146084614461D4600F0EA
:107BB0005DFD01214FF4804000F064FD4FF4C0678B
:107BC00002230122002602A93F488DF80C308DF8CF
:107BD0000D308DF80F2002978DF80E6000F0A8FC94
:107BE00007220921384800F0E5FC07220A2136481F
:107BF00000F0E0FCB8F1450FCDF810903CD14FF407
:107C00008063ADF81830072C42D10023ADF8143052
:107C1000052D4ED14FF48053ADF816300023ADF84A
:107C20001C300C2304A92948ADF81A3000F086FD59
:107C3000274B1A6802B1012240F22551234800F077
:107C4000E0FD0121214800F0C9FDFFF79FFF25233A
:107C50008DF804309DF840308DF8053000238DF804
:107C6000063001238DF80730FFF716FF01A800F05A
:107C700093FA09B0BDE8F083B8F14F0F02D1ADF827
:107C80001870C0E7072CADF818600DD1592107E036
:107C9000082C02D14FF48053B8E7092CB8D15421F5
:107CA0000C48FEF793FCB3E7082CAED0092CAFD1FB
:107CB000F0E70F2D02D14FF44053ADE7022D0CBF7A
:107CC0004FF400530023A7E70000024000380140B2
:107CD000FC10002085E501080E2307B5082200935B
:107CE0004E210123FFF75AFF03B05DF804FB0000AB
:107CF000402200210D4B0E48C3F884200D4B5A6AD8
:107D000042F400325A629A6942F400329A619A69E6
:107D100022F400329A61084A91815A6A032122F4BE
:107D200000325A620222FFF7B5B900BF00E100E05D
:107D300000000240003802400044004008B50248FC
:107D400000F05BFDC0B208BD004400402DE9F04FDB
:107D50004FF000091F46262389B09DF848808A46C7
:107D600014468DF8043083469DF84C509DF85060C1
:107D70008DF805808DF806908DF80790FFF78CFE42
:107D800001A800F009FA0121084600F06FFC01216A
:107D90004FF4003000F082FCB5B1082302930223B7
:107DA0008DF80E908DF80C304FF00309012302A9D5
:107DB00056488DF80F308DF80D9000F0B9FB072272
:107DC0004946524800F0F6FBBEB10423029301235A
:107DD0008DF80F3000234FF002098DF80E30032389
:107DE00002A94A488DF80C908DF80D3000F0A0FBE8
:107DF00007224946454800F0DDFBBAF1450FCDF8B2
:107E000010B043D14FF48063072CADF818304BD13C
:107E10000023ADF81430052F57D14FF480530024C0
:107E2000ADF81630ADF81C40002E59D1ADF81A60EF
:107E300075B1BDF81A3043F00403ADF81A30344B75
:107E40001A6802B1012240F22551324800F0D9FCF3
:107E500004A9304800F072FC01212E4800F0BEFC5D
:107E60000DB1FFF76BFF26238DF8043000238DF84A
:107E7000063001238DF805808DF80730FFF70CFEE2
:107E800001A800F089F909B0BDE8F08FBAF14F0FF1
:107E900002D14FF4C063B7E70023072CADF81830C8
:107EA0000ED14FF4827107E0082C02D14FF48053B9
:107EB000AFE7092CAFD1FF211748FEF787FBAAE7F0
:107EC000082CA5D0092CA6D1F0E70F2F02D14FF432
:107ED0004053A4E7022F0CBF4FF4005300239EE74A
:107EE0000823224640F227710A48ADF81A3000F004
:107EF00088FC40F22661074800F0C0FC224640F2B0
:107F00002661044800F07DFC92E700BF00000240BB
:107F1000001100200044004085E50108F8B5054641
:107F20000024134E134F8021134800F082FC68B1E7
:107F30002946114800F05DFC00240F4D0C4E0D4FFA
:107F40004021284600F075FC48B1F8BD0134B44228
:107F5000E9D94FF4A4713846FEF738FBE3E7013462
:107F6000B442EDD940F251113846FEF72FFBE7E756
:107F7000FFFF0F0085E501080044004008B5064BEF
:107F80000246186000B1012240F22551034800F07A
:107F900038FC012008BD00BF001100200044004053
:107FA00070B5134C40F22551204600F048FCC0B19A
:107FB000104B1D6825B1204600F01FFCC0B2A84739
:107FC00040F226610A4800F03AFC78B140F226619E
:107FD000074800F053FC084B1B683BB1BDE87040FC
:107FE0001847A388054ADBB21370E9E770BD00BFEC
:107FF000004400400011002004110020141F002044
:10800000BFF34F8F0449054BCA6802F4E062134383
:10801000CB60BFF34F8FFEE700ED00E00400FA05F0
:1080200010B5441EE3B2052B03D917211148FEF702
:10803000CDFAFEF7ADFD45F255520F4B1A60DA68E6
:10804000D207FCD4052C06D8DFE804F003090B0D99
:108050000F1101225A604CF6CC421A6010BD022268
:10806000F8E70322F6E70422F4E70522F2E7062206
:10807000F0E700BF85E501080030004038B5224C2C
:10808000236853B95F2000F021FB204D38B1204B0D
:10809000236001232B7000F029FB206838BD5E208F
:1080A00000F014FB18B11B4B23600223F2E75D20A4
:1080B00000F00CFB18B1184B23600323EAE75C20A7
:1080C00000F004FB18B1154B23600423E2E75B20AA
:1080D00000F0FCFA18B1124B23600523DAE75A20AE
:1080E00000F0F4FA18B10F4B23600623D2E75920B1
:1080F00000F0ECFA18B10C4B23600723CAE70B4BD6
:108100002360FF23C6E700BF0C11002010110020E0
:10811000C8C60108D8C60108EEC6010809C701088B
:1081200018C7010827C7010840C70108A9CF0108DF
:1081300038B5084B084D1A7852B9012420461C70F6
:1081400000F0ECFA287020F0FF01204600F0D6FA8B
:10815000287838BD081100200911002010B5044608
:10816000012000F0DBFA20F0FF0121430120BDE8EF
:10817000104000F0C3BA08B5FFF7F0FFFFF740FF6B
:1081800008B5012000F0CAFA10F0FF0F02D101205B
:10819000FFF7F1FFFFF734FF30B5012403780A4DF4
:1081A00003F01F029440C278590952B1074A2B4488
:1081B000D26842781201D2B283F8002345F82140F8
:1081C00030BD2031FAE700BF00E100E000ED00E043
:1081D00008B5084B98420BD101214FF4007000F014
:1081E00069FABDE8084000214FF4007000F062BA5F
:1081F00008BD00BF0024014043680A7923F04073A2
:1082000023F4807343EA02230A6810B513434360E2
:10821000D1E9032313438A6884681343084A224040
:1082200013434A7943EA420383600A7D036B013AB0
:1082300023F0F873D2B243EA0253036310BD00BFC8
:10824000FDF7FFC000234FF04072036003714371DC
:108250008360C0E90323012303757047836819B164
:1082600043F001038360704723F00103FAE7000045
:10827000044B5A6818B142F400025A60704722F465
:108280000002FAE7002701401D2970B51BD9072518
:10829000A1F11E06C46D06EB4606B54024EA0504AE
:1082A00003FA06F62643C665062A38D81F24013A83
:1082B000036C02EB8202944023EA040301FA02F207
:1082C0001A43026470BD13290DD90726A1F11405C4
:1082D000C46805EB4505AE4024EA060403FA05F53B
:1082E0002543C560E0E709290DD90726A1F10A0455
:1082F000056904EB4404A64025EA060503FA04F4E4
:108300002C430461D0E70726446901EB4105AE40E8
:1083100024EA060403FA05F626434661C4E70C2A5C
:108320000CD81F24073AC36B02EB8202944023EA65
:10833000040301FA02F21A43C263C3E7122A0CD8FB
:108340001F240D3A836B02EB8202944023EA04035C
:1083500001FA02F21A438263B4E7182A0CD81F24E8
:10836000133A436B02EB8202944023EA040301FABE
:1083700002F21A434263A5E71F24193A036B02EB8A
:108380008202944023EA040391401943016399E770
:10839000836843F0804383607047806D80B270478C
:1083A0000368194214BF012000207047C9430160CF
:1083B00070470000044B1A6818B142F002021A60BC
:1083C000704722F00202FAE7003C0240044B1A68B0
:1083D00018B142F004021A60704722F00402FAE772
:1083E000003C0240044B1A6818B142F008021A60BF
:1083F000704722F00802FAE7003C0240044B5A683A
:10840000D20741BF034ADA60034ADA60704700BF0F
:10841000003C0240EFCDAB8905040302024A5368D9
:1084200043F0010353607047003C0240014B9861E8
:10843000704700BF003C0240084B9A69D10709D43D
:108440009A69D20508D49B6913F4F05F14BF032026
:10845000042070470120704702207047003C024012
:10846000042313B504468DF80730FFF7E5FF8DF8B8
:1084700007009DF80730012B0AD11CB905238DF8A0
:10848000073007E0FFF7D8FF013C8DF80700F0E761
:10849000002CF3D09DF8070002B010BD10B50446C3
:1084A0004FF40040FFF7DCFF042804BF00232360E3
:1084B00010BD000038B504464FF400400D46FFF7EC
:1084C000CFFF04280BD1064A4FF40040536823F431
:1084D000807353602560BDE83840FFF7C1BF38BDE9
:1084E000003C024038B504464FF400400D46FFF70B
:1084F000B7FF04281BD135B125704FF40040BDE80B
:108500003840FFF7ADBFFF2324F0030504F0030458
:108510002968E40003FA04F421EA04042846FFF77A
:10852000BDFF21462846BDE83840FFF7C3BF38BD30
:108530002DE9F0430022012703250E6807FA02F314
:1085400033EA060431D14FEA420C05FA0CF4E44355
:1085500091F804E0D0F800900EFA0CF804EA09094A
:108560000EF1FF3E48EA0908BEF1010FC0F8008095
:1085700011D8D0F808E004EA0E0E4C7904FA0CF495
:1085800044EA0E048460848824EA03048B799340CF
:108590009BB223438380C36805FA0CF423EA0404E6
:1085A000CB7903FA0CF32343C3600132102AC5D1FF
:1085B000BDE8F08310B50F2401F00703C90800EBF4
:1085C0008100016A9B009C4021EA04010162016A6A
:1085D0009A400A43026210BD204B10B59A6802F01F
:1085E0000C020C2A30D8DFE802F02F2F2F2F072F94
:1085F0002F2F072F2F2F2000194B184A0360936845
:108600001849C3F30313CC5C0368E34043609468E8
:10861000C4F302240C5D23FA04F484609268C2F36C
:10862000C2228A5CD340C36010BD99680E4CC1F36E
:1086300083419A68615C9B68094BC2F381524B434A
:108640000132B3FBF2F3D8E74FF400425B68C3F3A7
:108650004233013302FA03F3CFE700BF0038024090
:108660000024F4004C0200205C020020044BDA6974
:1086700011B11043D861704722EA0000FAE700BF49
:1086800000380240044B1A6A11B110431862704757
:1086900022EA0000FAE700BF00380240044B5A6AA1
:1086A00011B110435862704722EA0000FAE700BF98
:1086B00000380240044B5A6911B1104358617047A9
:1086C00022EA0000FAE700BF003802404309012B0C
:1086D000054B00F01F000CBF1B685B6B23FA00F01A
:1086E00000F00100704700BF00380240024A536B9F
:1086F00043F080735363704700380240002382B018
:108700000193054B0193019B03EB80000190019BBA
:10871000196002B0704700BF50280040002382B0AB
:108720000193054B0193019B03EB80000190019B9A
:10873000186802B0704700BF5028004030B50D46A1
:108740000446028AEB8892B222F440521A43898985
:1087500002828389288923F4B052AB8822F00C026C
:108760000343688985B003431343A381A38A684602
:108770009BB223F440730B43A382FFF72DFFDDE987
:108780000231154A944218BF19461923A2894B4356
:10879000296810044CBF49008900B3FBF1F164253E
:1087A000B1FBF5F3A2891801120405FB13130BD5D5
:1087B000DA003232B2FBF5F202F0070242EA0003BD
:1087C0009BB2238105B030BD1B013233B3FBF5F3FF
:1087D00003F00F030343F3E700380140838919B125
:1087E00043F400538381704723F400531B041B0C94
:1087F000F8E7C1F30801818070478088C0F3080062
:10880000704701F01F0310B5C1F342140121012C80
:1088100001FA03F105D10C3003683AB11943016044
:1088200010BD022C0CBF10301430F5E723EA010113
:10883000F5E70388194214BF012000207047012387
:10884000C1F3421210B5012A01F01F0403FA04F328
:108850000DD182891340028892B26BB10123090ABB
:1088600003FA01F10A4214BF1846002010BD022A83
:108870000CBF028A828AEDE71846F7E70B0A01214E
:108880009940C94389B20180704700002DE9F34146
:108890001F46002304460D46019316461AB90120CF
:1088A00002B0BDE8F08140F6FF7301934FF4003150
:1088B000204600F04CFD002852D10121204600F056
:1088C00016FD4FF2FF71204600F02AFD01212046DF
:1088D00000F0F7FC40F6FF73DFF8AC8101934146EE
:1088E000204600F029FD002841D0394601222046CB
:1088F00000F008FD40F6FF735F4F019339462046B4
:1089000000F025FD002838D0012E42D1002120465C
:1089100000F0EDFC03F04EFD31462046238B00F0C5
:10892000DBFC03F067FD40F6FF73544E01933146C4
:10893000204600F00CFD30B3204600F0EEFC28701D
:1089400040F6FF734E4D01932946204600F0FFFC90
:108950000028A4D0019B5A1E0192002BF4D104E000
:10896000019B5A1E0192002BA0D1002098E7019B89
:108970005A1E0192002BB2D1F7E7019B5A1E0192B9
:10898000002BBBD1F1E7019B5A1E0192002BCED1E7
:10899000EBE7022E25D103F00DFD4FF400612046D8
:1089A00000F0BEFC0021204600F0A1FC238B03F068
:1089B00021FD40F6FF73334E01933146204600F00F
:1089C000C6FC40B10121204600F086FC238A2B70B2
:1089D000238A6B70B4E7019B5A1E0192002BECD1E5
:1089E000C3E740F6FF77033E238BDFF898802E44E1
:1089F000B542019728D1234E3146204600F0A7FC0E
:108A000070B30021204600F072FC204600F085FC87
:108A100040F6FF731B4E287001933146204600F04C
:108A200096FC18B30121204600F056FC204600F0C9
:108A300074FC6870204600F070FCA87080E7019B11
:108A40005A1E0192002B90D04146204600F07FFC38
:108A50000028F4D0204600F060FC05F8010BC7E7C1
:108A6000019B5A1E0192002BC6D17EE7019B5A1E24
:108A70000192002BD1D178E70200001040000010D5
:108A80001000001004000010010003002DE9F34164
:108A90001E460023019340F6FF7304460D46174619
:108AA0000193002A00F081804FF40031204600F04D
:108AB0004EFC002842D10121204600F002FC40F685
:108AC000FF73DFF87C8101934146204600F034FCBF
:108AD00000283CD031460022204600F013FC40F62E
:108AE000FF73534E01933146204600F025FC0028C9
:108AF00033D0297820466E1C00F00DFC3D4440F632
:108B0000FF77DFF83081AE42019731D1494D2946D8
:108B1000204600F01CFC002836D02046012100F041
:108B2000DBFB40F6FF73444D444C0193294620463D
:108B300000F00DFC00282DD1012005E0019B5A1EFC
:108B40000192002BB0D1002002B0BDE8F081019B62
:108B50005A1E0192002BB7D1F5E7019B5A1E0192D4
:108B6000002BC0D1EFE7019B5A1E0192002BEAD0E7
:108B70004146204600F0EBFB0028F4D016F8011B1C
:108B8000204600F0C8FBBEE7019B5A1E0192002B55
:108B9000BDD1D8E7019B5A1E0192002BC6D1D2E766
:108BA000019B5A1E0192002BCDD04FF4003120467C
:108BB00000F0CDFB0028F3D10121204600F081FB1D
:108BC00040F6FF731E4D01932946204600F0B4FB8A
:108BD00010B300223146204600F094FB40F6FF73AC
:108BE000134D01932946204600F0A6FBD0B1204644
:108BF000012100F071FB40F6FF730F4D0F4C019304
:108C00002946204600F0A3FB002895D0019B5A1E60
:108C10000192002BF4D196E7019B5A1E0192002B82
:108C2000D2D190E7019B5A1E0192002BDAD18AE73C
:108C300082000700040000101000001000540040E3
:108C4000010003002DE9F3411E46002304460D46B2
:108C5000019317461AB9012002B0BDE8F08140F631
:108C6000FF7301934FF40031204600F070FB0028A1
:108C700037D10121204600F024FB40F6FF73DFF8D6
:108C8000E08001934146204600F056FB002842D088
:108C900031460022204600F035FB40F6FF732C4E93
:108CA00001933146204600F047FB002839D029784F
:108CB00020466E1C00F02FFB3D4440F6FF77DFF8A6
:108CC0009480AE42019737D1224D2946204600F0CC
:108CD0003EFB0028BFD1019B5A1E0192002BF4D10C
:108CE00004E0019B5A1E0192002BBBD120460121BA
:108CF00000F0F2FA40F6FF73174D184C0193294625
:108D0000204600F024FB20B1019B5A1E0192002B4B
:108D1000F5D10020A0E7019B5A1E0192002BB1D192
:108D2000E4E7019B5A1E0192002BBAD1DEE7019BBA
:108D30005A1E0192002BD9D04146204600F007FB75
:108D40000028F4D016F8011B204600F0E4FAB8E73A
:108D500082000700040000101000001000540040C2
:108D60000100030000232DE9F3410D464FF40031CB
:108D700004461746019300F0EAFA18B9002002B041
:108D8000BDE8F0810FB90120F9E7297820466E1C73
:108D900000F0C1FA3D4440F6FF77DFF86C80AE4248
:108DA00001971FD1184D2946204600F0D0FA28B36C
:108DB0002046012100F090FA40F6FF73134D144C49
:108DC00001932946204600F0C2FA0028DBD0019B1F
:108DD0005A1E0192002BF4D1D0E7019B5A1E01923A
:108DE000002BCBD04146204600F0B1FA0028F4D049
:108DF00016F8011B204600F08EFAD0E7019B5A1EA0
:108E00000192002BCFD1B9E7040000101000001030
:108E1000005400402DE9F3411F46002304460D464F
:108E2000019316461AB9012002B0BDE8F0814FF453
:108E3000003100F08CFA08B90020F5E70121204646
:108E400000F055FA4FF2FF71204600F069FA012157
:108E5000204600F036FA40F6FF73DFF8AC8101934C
:108E60004146204600F068FA00283AD039460122EF
:108E7000204600F047FA40F6FF735F4F01933946F2
:108E8000204600F064FA002831D0012E3BD10021A9
:108E9000204600F02CFA03F08DFA31462046238B51
:108EA00000F01AFA03F0A6FA40F6FF73534E01934E
:108EB0003146204600F04BFAF8B1204600F02DFA7A
:108EC000287040F6FF734E4D01932946204600F06E
:108ED0003EFA0028A7D0019B5A1E0192002BF4D124
:108EE000AAE7019B5A1E0192002BB9D1A4E7019B6E
:108EF0005A1E0192002BC2D19EE7019B5A1E01927D
:108F0000002BD5D198E7022E29D14FF400612046DD
:108F100000F006FA03F04EFA00212046238B00F001
:108F2000E6F903F067FA40F6FF73364E01933146D7
:108F3000204600F00CFA60B103F03CFA0121204613
:108F400000F0CAF9238A2B70238A6B7003F052FA5F
:108F5000B7E7019B5A1E0192002BE8D16CE740F65F
:108F6000FF77033E238BDFF89C802E44B5420197A8
:108F700029D1244E3146204600F0E9F978B300218A
:108F8000204600F0B4F9204600F0C7F940F6FF7320
:108F90001C4E287001933146204600F0D8F920B3CA
:108FA0000121204600F098F9204600F0B6F96870DB
:108FB000204600F0B2F9A87083E7019B5A1E019287
:108FC000002B3FF439AF4146204600F0C0F900289D
:108FD000F3D0204600F0A1F905F8010BC6E7019B8C
:108FE0005A1E0192002BC5D126E7019B5A1E019201
:108FF000002BD0D120E700BF02000010400000107D
:1090000010000010040000100100030038B5204BD0
:1090100008219A691F4842F400129A619A6922F461
:1090200000129A615A6A22F400125A62FEF7B6F8E8
:10903000012308211A461748FDF7EEFF09211548BC
:109040000122FEF727F809211248FEF7BCF8D8B133
:10905000012038BD08212846FEF7A0F8FDF7ECFDF9
:1090600008212846FEF7A0F8FDF7E6FD013CF1D106
:1090700009210848FEF7A7F820B940F27D110648FB
:10908000FDF7A4FA2046E4E73324024DEEE700BFE3
:10909000003802400004024085E501082DE9FF4147
:1090A000444B054698420E4617467CD103F5F233F1
:1090B0005A6A082142F400125A629A693E4842F400
:1090C00000129A619A6922F400129A61FEF766F81A
:1090D000012308211A463848FDF79EFF092136482A
:1090E0000122FDF7D7FF09213348FEF76CF800286D
:1090F00055D0012308211A462F48FDF78DFF042281
:1091000008212D48FEF704F8012309211A462A48B0
:10911000FDF782FF042209212748FDF7F9FF274BBD
:109120009A6942F400129A619A6922F400129A61D3
:10913000684600F0ADF8224B694601934FF4806316
:10914000ADF80A304FF480432846ADF80C30ADF846
:109150000870009600F038F82846012100F0A6F8C3
:10916000012019E008214046FEF718F8FDF764FDDC
:1091700008214046FEF718F8FDF75EFD013CF1D1ED
:1091800009210D48FEF71FF80028B2D10D4840F222
:10919000A511FDF71BFA204604B0BDE8F081332489
:1091A000DFF81480EAE74FF4DA710648FDF70EFAAB
:1091B000BEE700BF005400400004024000380240F7
:1091C0000000FFBF85E501087FB504468688684634
:1091D0000D46FFF701FA029A2B4926F03F06B2FB33
:1091E000F1F13604360C88B20643A6802388274E58
:1091F00023F001031B041B0C23802B68B3421ED8F1
:109200005B00B2FBF3F39BB2042B38BF04230130A5
:1092100080B22084A3832388AA8843F0010323809B
:109220002388698923F481630A4323F002031343EB
:1092300023802A89AB891343238104B070BD4BF688
:10924000FF70EE8886421BBF1920434303EB4303A4
:10925000B2FBF3F30BBFB2FBF3F39BB29BB243F44D
:109260008043C3F30B020AB943F001034FF4967233
:109270004A434FF47A7192FBF1F2013292B243F415
:1092800000432284C6E700BF40420F00A0860100D1
:1092900041F28832044BC0E90023002383604FF47D
:1092A00080438381704700BF0000FFBF038819B16E
:1092B00043F001030380704723F001031B041B0CE0
:1092C000F8E7038819B143F480730380704723F4EF
:1092D00080731B041B0CF8E7038819B143F4007377
:1092E0000380704723F400731B041B0CF8E703880A
:1092F00019B143F480630380704723F480631B0437
:109300001B0CF8E722B141F0010189B201827047DC
:1093100001F0FE01F9E701827047008AC0B2704790
:109320000388B1F5006F1BBF23F400631B0443F4F3
:1093300000631B0C03807047838A008B43EA004361
:1093400021F07F401840431A58425841704700238B
:1093500082B0009301930B0F01900093009B21F0CA
:109360007F4153B1019B14330193019B1B680B4256
:1093700014BF0120002002B07047019B090C183374
:10938000F2E7F8B50E46054680B14F1C384600F0AE
:1093900053FF044640B13A4600210FF036FA3246F8
:1093A000294620460FF00DFA2046F8BD0446FBE79B
:1093B00038B50D46044628B110F02EFA2346204455
:1093C000834201D1002038BD13F8012BAA42F7D106
:1093D0000120F8E737B504460D460FF001F80022EA
:1093E00001A90260204610F043FB04460EF0F8FF8E
:1093F0000368222B08D0019B1B782BB9002C03DBC0
:1094000020462B6003B030BD012300202B60F9E71C
:109410002DE9F04F05464FF0010B002687B0CDE94E
:10942000031206F10903122B8CBF0320022000F067
:1094300003FF0090E8B13246364910F03FF9039B34
:1094400053F82690EDB90024009800F0DFFEBBF140
:10945000000F02D1284600F0D9FE84B1049B0136EA
:10946000B34225464FF0000BDBD1204607B0BDE8E4
:10947000F08FBBF1000F02D1284600F0C7FE002498
:10948000F3E7254B4FF00008B9F1000F08BF9946EC
:10949000484610F0C1F90190009810F0BDF9029013
:1094A0002846494610F0E7F9B8B9284610F0B4F953
:1094B000DDE9012301309B1A08FB030000F0BCFE2C
:1094C00004460028BFD003462F4618F1FF3809D2C2
:1094D0003946184610F098F9B6E7019B08F10108E3
:1094E0001844DEE749463846059310F0C4F9059B59
:1094F000A0EB070A52463946184610F0A7F9009922
:10950000504410F081F9019A029B9244C3185744C9
:10951000DBE700BFF6B3010885E5010830B580B18F
:109520000346021F00F1180452F8045F8D4208D070
:10953000A242F9D11C301A4614680433013401D117
:10954000116030BD8342F6D1FBE770B5044680B1AF
:10955000064600EB8105AE4204D12046BDE87040CE
:1095600000F054BE56F8040B0028F4D000F04EFE74
:10957000F1E770BD2DE9F74F89460092002838D0F9
:109580000027C45D8CBB05468346264600EB070AD0
:10959000D34538D104B10136002E6FD0013738469B
:1095A00000F04AFE8346002866D03A4600210FF0BC
:1095B0002CF9B00000F040FE0446002860D04FF0C7
:1095C00000084146AA4532D131B15846FFF7D9FECD
:1095D000002855D044F82800584600F017FE009B9C
:1095E0001E60204603B0BDE8F08F0137B7F5807FDD
:1095F000C7D100242646204600243146FFF7A5FFA8
:10960000009B1C60EDE79BF800304B4505D10CB189
:10961000002401360BF1010BBAE70FF085F89BF837
:109620000030184443781B0758BF0134F2E72B7809
:109630004B4513D181B15846FFF7A3FE00B308F1A3
:10964000010344F8280000213A46584601930FF0E0
:10965000DCF8019B002198460135B3E701910FF03A
:1096600063F82B7801991844407810F0080F04BF74
:109670000BF801300131EFE70446BCE73446B0E7B0
:10968000584600F0C3FDB6E72DE9F743002506462E
:109690000820884691461F46009500F0CDFD0446FF
:1096A000002868D0C0E90055304610F0B5F8012810
:1096B0000FD133782A2B0CD109F1FF33C4F8008085
:1096C000636022684A4502D263684B4543D32B4B03
:1096D0000EE02D213046FFF76BFE0546C0B902A90A
:1096E00041F8040D3046FFF775FE019B63B1244B32
:1096F0003B6000992846FFF728FF002C37D0204612
:1097000000F084FD002432E0C4E900001D46D8E7E3
:109710006A462D213046FFF72DFF009B0546013B91
:10972000012B01D9174BE3E7002302AE46F8043DB5
:1097300031460068FFF74EFE2060019B0BB1124BD3
:10974000D6E731466868FFF745FE6060019B002B55
:10975000B7D00E4BCCE7424501D3434501D20C4B69
:10976000C6E700992846FFF7F0FE00233B6020463D
:1097700003B0BDE8F0830546BBE700BF26C801087B
:10978000A0C70108BFC70108E8C7010807C801084A
:1097900046C8010838B590B1451E15F8014F0CB9FF
:1097A000204638BD0EF0C0FF23462044427802F028
:1097B0000302022A08BFA4F120032B70EDE7012069
:1097C000EFE708B520B34A1C22D0062920D8DFE8ED
:1097D00001F0040D101316191C00002303600FF094
:1097E000F7F80840431C5842584108BD0023436025
:1097F000F5E700238360F2E700238361EFE70123AD
:10980000C360ECE700230361E9E700234361E6E777
:109810000120EAE770B506460D1F01F1180455F85E
:10982000041F4B1C03D1A542F9D1002070BD304666
:10983000FFF7C7FF0028F6D0F8E708234A4291FB5C
:10984000F3F302F0070201F0070158BF5142012271
:10985000DBB2C9B202FA01F1C25C1143C1547047D4
:1098600008234A4291FBF3F302F0070201F00701DB
:1098700058BF51420122DBB2C9B28A40C15C21EA21
:109880000201C1547047082391FBF3F3DBB2C05CC3
:109890004B4203F0070301F0070158BF5942C9B218
:1098A000084100F0010070472DE9F047089E8A4604
:1098B00090461D46DDF82890074610B11446A24593
:1098C00007D875B9012200240B9B1A602046BDE819
:1098D000F08721463846FFF7D6FF002861D10134D2
:1098E000EDE7099B023B042B04D8DFE803F0282CAA
:1098F0002C3034006B6801336B6028460FF068F839
:10990000013108BFB0F1FF3FDCD031462846FFF7F8
:1099100058FF0028D6D12FB3044621463846FFF71A
:10992000B2FF002841D10134A245F6D10446013EE0
:10993000042E19D8DFE806F02B2D2F313300AB6849
:109940000133AB60D9E7EB680133EB60D5E72B69F6
:1099500001332B61D1E76B6901336B61CDE7002DDA
:10996000E5D1AFE73C46E2E72C6028460FF030F83F
:10997000013108BFB0F1FF3FA4D0B9F1000FA1D071
:1099800049462846FFF746FF00289FD09AE76C60BB
:10999000EBE7AC60E9E7AC61E7E7EC60E5E72C6199
:1099A000E3E7A045DBD1444690E7A045BFD1FAE705
:1099B00000232DE9F04F06468BB01C200C46904644
:1099C000099300F039FC0546002800F0E4801C20D3
:1099D00000F032FC0746002800F0DD804FF0FF3138
:1099E000021F2B1F05F1180043F8041F984242F88C
:1099F000041FF9D100230121D4F800A00DF124099E
:109A0000CDE90031CDE902793C212346524630466A
:109A1000FFF74AFF099900296ED1824502D12846F5
:109A2000FFF77CFD02234FF0010AD4F804B0CDE922
:109A300000A3CDE9025923465A463C2106F108000D
:109A4000FFF732FF099B002B56D183454CD151467D
:109A50002846FFF763FD03234FF0020AD4F808B04D
:109A6000CDE900A3CDE9025923465A46182106F153
:109A70001000FFF719FF099B002B3DD1834546D10C
:109A800051462846FFF74AFD40F26F1BA369059334
:109A9000E368049306F114030693DDF810A006F1C1
:109AA0001303079351460698FFF7EDFE28B1059979
:109AB0000798FFF7E8FE002836D1BBF1010B33D041
:109AC000E36820460133E3600EF082FF013108BFF6
:109AD000B0F1FF3F24D0A36929462046D4F80CA05A
:109AE0000593FFF797FEDDE7424621463046FFF734
:109AF0005FFF09900028AED0284600F087FB17B121
:109B0000384600F083FB09980BB0BDE8F08F424661
:109B100021463046FFF74CFF09900028ECD1B3E70F
:109B200001234FF0000A0993099B002BE4D1049B09
:109B3000534520D104212846FFF7F0FC05230622D7
:109B4000D4F810A0CDE90032CDE90259234652469F
:109B50000C2106F11800FFF7A7FE099B002BCBD1C3
:109B60008245C9D06369A3EB0803042B0CD94FF0DD
:109B7000FF330993C0E7424621463046FFF718FFFE
:109B800009900028B8D1D9E7424621463046FFF770
:109B90000FFF0990B0E74FF0FF330993002DB2D0CB
:109BA0000027A9E72DE9F04F002487B0924606AAC6
:109BB000894642F80C4D2C219846109DFFF7DAFC9F
:109BC000074688B93E4B2B6003993846FFF7BDFC2A
:109BD00007B0BDE8F08FD0F800B072685A451CD2CB
:109BE000304600F013FB0134039BA342ECD957F835
:109BF00024602F213046FFF7DBFBA8B92B46304607
:109C000042465146FFF740FD2B680646002BE2D046
:109C10000028D9D000F0FAFAD6E759464846FFF7AF
:109C20000CFE0BF1010BD8E700232F21304604AACC
:109C30000493FFF79FFC049906464B1E012B04D9A1
:109C4000204B2B60FFF781FCBEE742462B46514676
:109C50000068FFF719FD2A6883462AB108B100F0B1
:109C6000D5FA04993046EDE72D213068FFF7A0FBC7
:109C700018B908F1FF32CBF80420002306A941F8F7
:109C8000043D7068FFF7A6FB059A00901AB10E4AD2
:109C900058462A60E3E7DBF80020DBF80410914225
:109CA00005D230460499FFF750FC584699E7114613
:109CB00048460192FFF7C1FDDDE900321A44ECE7A6
:109CC0006BC801087DC80108A2C801082DE9FF4141
:109CD00000230E460393144602B902AC236048B930
:109CE0000546564B236003992846FFF72EFC04B027
:109CF000BDE8F08103AA2021FFF73CFC039B054649
:109D0000062B02D04E4B2360EDE71A22002130468D
:109D10000EF07BFD009400223C2331462868FFF7BB
:109D200041FF2268002ADED100943C2306F108019D
:109D30006868FFF737FF2268002AD4D100941823FF
:109D400006F11001A868FFF72DFF2368002BCAD188
:109D50006869FFF71FFD07223A496869FFF758FB5A
:109D600080460FF059FD012806F1130706D198F837
:109D700000303F2B04BF2A2388F80030002208233C
:109D8000394640460094FFF70DFF404600F03EFA8A
:109D90002268002AA7D107213846FFF774FD30B1A9
:109DA00011463846FFF749FD0721FFF759FDEF68D7
:109DB00006F1140838460FF02FFD012804D13B7836
:109DC0003F2B04BF2A233B70202300224146384604
:109DD0000094FFF7E7FE00214046FFF741FD2368AE
:109DE000002B80D12F693846FFF7D4FC00287FF480
:109DF0007AAF38460D221449FFF70AFB07460028C0
:109E00003FF471AF183600940D2301223146FFF75D
:109E1000C9FE384600F0FAF9012421463046FFF722
:109E200032FD30B1611E3046FFF707FD2146FFF7D6
:109E300017FD01340D2CF0D155E700BF4AC70108CA
:109E400062C701086802002084020020F0B58DB0CE
:109E5000CDE90023054628B94FF0FF304FF0FF3120
:109E60000DB0F0BD2422002103A80EF0CEFC03A902
:109E700068460EF0A9FB04460028EDD00EF0A8FDC0
:109E80004A1C08BFB0F1FF3F06460F46E4D06269A6
:109E900021462846FFF78CFD0028DDD120460EF034
:109EA00097FD4B1C08BFB0F1FF3FD5D08F4208BFD4
:109EB000864203D020460EF08BFDD1E72368204672
:109EC000013323600EF084FD013108BFB0F1FF3F84
:109ED000C2D0626921462846FFF76AFD0028E9D012
:109EE000BAE770B53C258AB0DDE90E64019496FBB3
:109EF000F5F405FB14640294182493FBF4F505FBB8
:109F00001433CDE90330481E0C2190FBF1F301FB23
:109F100013010023CDE907339DF84030A2F26C72A3
:109F200001A80591069209930EF052FD0AB070BD8A
:109F3000F7B5044602A860E902230EF033FB02697C
:109F4000037A551C426990F804C0077B02F26C71D9
:109F5000067EC2690068A3700033207018BF012319
:109F60002046013284F801C0E7702571A4F805107D
:109F7000E6712272637203B0F0BD30B5457A85B0E8
:109F8000C4788378B0F805200179029505780195A9
:109F9000407800902046FFF7A4FF05B030BD904206
:109FA00071EB0303B4BF012000207047032210B5FA
:109FB000104986B00B78013393FBF2F202EB4202B8
:109FC0009B1A0D4A0B7052F823400278B0F8053006
:109FD000049242781A21039282780292C278019206
:109FE000027920460092054A0FF034FB204606B065
:109FF00010BD00BF5F1100204CC9010811C9010844
:10A00000B1F1004F08BF00281FB502460B4608D02B
:10A0100001A8FFF78DFF01A8FFF7C8FF05B05DF8A5
:10A0200004FB0148FAE700BF43C901082DE9FF47D7
:10A0300003220D462B4900280B78044603F1010347
:10A0400093FBF2F202EB4202A3EB0203264A0B70EF
:10A0500052F8236075F100033EDA4FF0010A4442E2
:10A0600065EB4505214A0023204629460DF0D2FF25
:10A070001E4A07460023204629460DF0CBFF104616
:10A0800019464FF4616200230DF0C4FF4FF4616282
:10A0900080460023204629460DF0BCFF1046194695
:10A0A0003C2200230DF0B6FF3C22814600232046CF
:10A0B00029460DF0AFFFCDF80080CDE901923B4677
:10A0C000BAF1000F0BD00A4A1A2130460FF0C2FA3B
:10A0D000304604B0BDE8F0874FF0000AC2E7054AF9
:10A0E000F2E700BF5F1100204CC901088051010058
:10A0F0002FC9010830C901080FB404B0704700002F
:10A100000FB437B51B4C256855B9032229460120E9
:10A1100002F072FB2B462A462946206002F090FB93
:10A12000154D2A68013A03321ED86421206802F0D6
:10A1300073FD8022002111480EF067FB07AB069AE1
:10A1400080210E4801930FF003FF7F2803DD0C49A7
:10A150000C480FF059FB2B680848984700232068EB
:10A160001A46194602F06CFB03B0BDE8304004B05B
:10A17000704700BFE8110020601100206811002026
:10A18000F1B80108E31100200FB410B50D4CA2B0D6
:10A190002268013A033210D825AB249A802102A804
:10A1A00001930FF0D5FE7F2804DD07490DF18300F0
:10A1B0000FF02AFB236802A8984722B0BDE81040A0
:10A1C00004B0704764110020F1B8010870B504466E
:10A1D000054E4518AC4200D170BD14F8011B304645
:10A1E000FFF78EFFF6E700BF58C9010838B50C46E7
:10A1F0001546FFF785FF20462946FFF7E7FFBDE834
:10A2000038400148FFF77CBF84E5010810B50446DB
:10A2100070B102F023FA204602F00EFA02F0CAF8FA
:10A22000BDE81040034A93880133938002F0E2B8FE
:10A2300010BD00BF161F002070B5234C8AB02268E5
:10A2400005460132226000283BD0632A1F4E0BDDF9
:10A2500003F0E2FF0523002201A903F00FFF03F042
:10A26000F1FB00233060236003F0ECFB336803F55F
:10A270007A73984204D903F0E5FB00233060236031
:10A28000134A144C13781BB92360636001231370C5
:10A2900002F0E4F9284602F0CDF9064668B12A46F4
:10A2A00000210EF0B2FA02F085F8238801332380F2
:10A2B00002F0A0F830460AB070BD638801336380B5
:10A2C000F8E70646F6E700BFF0110020F411002081
:10A2D000EC110020161F0020006800BA70470088AB
:10A2E00040BA80B2704700687047837842781B0498
:10A2F000007843EA02231843704700887047FFF74D
:10A30000F2BF0370130E4370130C8370130AC370F3
:10A310000271052070470B0E03700B0C43700B0A83
:10A320008370C170042070470B0A037041700220D3
:10A3300070470B0A017043700B0C090E8370C170DB
:10A3400004207047A0F14103052B02D83738C0B272
:10A350007047A0F16103052B01D85738F7E7303873
:10A36000C0B20A2828BFFF2070470022013910B56B
:10A370000144441E8C4204D014F8010F08B1002A95
:10A3800001DA104610BDFFF7DDFF0F2802D840EAC2
:10A390000212EFE74FF0FF32F3E738B505460C46FF
:10A3A0000FF0B2F8611B013190FBF1F303FB1100D8
:10A3B000284438BD10B504460FF082F8014B1C60EC
:10A3C00010BD00BFB8020020024B186801301860B1
:10A3D0000FF076B8B80200200078013070470FB453
:10A3E00004B070472DE9FF470F46002104AC254E0D
:10A3F00044F8041D8046924630682246994602F091
:10A400004DFD0128039B31D13BB14FF080521E4BD3
:10A410001A60BFF34F8FBFF36F8FB7F5C87F88BF48
:10A420004FF4C87741463A4618480EF0CAF9184D1D
:10A43000164B21463068AF802B60A5F806A085F842
:10A44000089002F00DFB039B3BB14FF080520E4B86
:10A450001A60BFF34F8FBFF36F8F0E480094002335
:10A4600001220421006804F0A5F8039B3BB14FF0E2
:10A470008052054B1A60BFF34F8FBFF36F8F04B04C
:10A48000BDE8F087FC13002004ED00E0601200201E
:10A490005412002008140020034800230122022146
:10A4A000006804F017B800BF081400201FB503F0BF
:10A4B000CFFA0D4B04AA1860002342F8043D009225
:10A4C00001220A481146006804F074F8039B3BB16E
:10A4D0004FF08052064B1A60BFF34F8FBFF36F8F60
:10A4E00005B05DF804FB00BF041400200814002030
:10A4F00004ED00E01FB5002304AA42F8043D0A4819
:10A50000009280210122006804F054F8039B3BB1C3
:10A510004FF08052054B1A60BFF34F8FBFF36F8F20
:10A5200005B05DF804FB00BF0814002004ED00E056
:10A530001FB5104B1C680346A8B1002304AA42F8BB
:10A54000043D009208210122204604F033F8039BC9
:10A550003BB14FF08052084B1A60BFF34F8FBFF3EF
:10A560006F8F04B010BD01220821204603F0B2FF16
:10A57000F7E700BF0814002004ED00E01FB500233A
:10A5800004AA42F8043D0A48009210210122006802
:10A5900004F010F8039B3BB14FF08052054B1A605A
:10A5A000BFF34F8FBFF36F8F05B05DF804FB00BFA3
:10A5B0000814002004ED00E01FB500230C4904AA94
:10A5C00042F8043D08700B480092402101220068C7
:10A5D00003F0F0FF039B3BB14FF08052064B1A6033
:10A5E000BFF34F8FBFF36F8F05B05DF804FB00BF63
:10A5F000441200200814002004ED00E000487047D9
:10A600003C120020114810B5002303224FF4807142
:10A61000006803F05FFF4FF080520D4B1A60BFF3EC
:10A620004F8FBFF36F8F0B4C206802F083FC40B15B
:10A63000BDE81040002308481A461946006802F099
:10A64000FFB8012003F056FBEEE700BF081400201E
:10A6500004ED00E000140020F8130020F8B5104BC2
:10A660000146186802F0D8FA0446B8B14FF0805697
:10A670000C4F0D4D002303224FF40071386803F096
:10A6800029FF2E60BFF34F8FBFF36F8F386803F041
:10A6900045F92E60BFF34F8FBFF36F8F2046F8BD93
:10A6A000F81300200814002004ED00E0014B1860AE
:10A6B000704700BFF013002070B5044678B10378EE
:10A6C000032B0CD1436853B10025054E1868F2697D
:10A6D00090476068F369056098476560257070BDB4
:10A6E0001812002010B50E480E4C002305222146FA
:10A6F000006802F0A5F8012807D1002363600A4B27
:10A700001B6863B1BDE810401847084B2178084822
:10A710005B6998472046BDE81040FFF7CDBF10BDEC
:10A72000F413002048120020F0130020181200201B
:10A730005EC901087FB50024094E002201A93068D6
:10A7400002F0D8F9651C30B9064BE1B25B690648E6
:10A75000984704B070BD01A8FFF7AEFF2C46ECE7A8
:10A76000F41300201812002085C90108014B186855
:10A77000704700BFF413002010B50446064B010AD1
:10A78000A3F84A00202000F093FBE1B22120BDE8AD
:10A79000104000F08DBB00BF201F002008B5FFF760
:10A7A000EBFF0122014B83F8522008BD201F00203F
:10A7B000002238B50B4B05461D2083F84E100C4681
:10A7C00083F84C2000F0CCFB20F0060040EA440166
:10A7D000C9B21D2000F06CFB2946BDE8384023209B
:10A7E00000F066BB201F002013B5164C0120A368A3
:10A7F0009847002341F6FE720093009B934218DDB8
:10A80000A36802209847002341F6FE720193019B42
:10A81000934212DD0C4BB5211C6C4020A047A021B7
:10A820004120A04700210120234602B0BDE810408E
:10A830001847009B01330093DFE7019B013301932D
:10A84000E5E700BF1812002078CC0108094B07B5D6
:10A850001B6CC2213B209847002341F6FE720193F6
:10A86000019B934202DD03B05DF804FB019B0133C1
:10A870000193F5E778CC01082DE99F488E488F4B6E
:10A880008F4F03608F4B904C8360904B904D436093
:10A89000904BDFF880A2C3608F4BDFF87C9203619E
:10A8A0008E4BDFF878B283618D4BC3613B6898476C
:10A8B00063698C489847002328681A46194601F0B6
:10A8C000BFFF9AF8040068B94FF0FF33194603AA96
:10A8D00003F0B6FD68B9666903F08EFC0146824854
:10A8E000B047EEE741F2883303AA4FF0FF31002072
:10A8F000EEE7039BDE0516D500F098FA002000F085
:10A90000E9FDFB6A9847FFF715FF636977489847A9
:10A910000023D9F800001A46194601F091FF0020E3
:10A9200003F066FACDE7980510D500F07FFAFFF73F
:10A930008DFFFB6A9847FFF7FDFE63696C489847F7
:10A940006421D9F8000002F067F9BAE7D9F80000ED
:10A9500002F0F0FA012803D1636966489847B0E72E
:10A96000DBF8003023B94FF4B5716348FBF72EFED6
:10A97000039B190604D50722604B1A70FFF7B2FE3D
:10A98000039B5A0752D50021286802F045F9012897
:10A990004CD1A3690C209847064688B963690C21FD
:10A9A00057489847334632463146286801F048FFF9
:10A9B000002886D140F27F114F48FBF707FE80E761
:10A9C000DFF85C81A369B8F8040098470346A0B992
:10A9D000B8F80410019062694A489047E26930462D
:10A9E0009047019B28681A46194601F029FF002864
:10A9F0007FF467AF40F28711DEE708F1040203CA73
:10AA000033607060B1601846D8F80010B8F80420C0
:10AA10000DF0D7FE0322394B1A705E60FFF762FE1D
:10AA2000002328681A46194601F00AFF039BDB073A
:10AA300009D50122314B1A7000225A60324A12683D
:10AA40009A60FFF74FFE039BDE0606D505222B4BCF
:10AA50001A7000225A60FFF745FE039B180706D5BF
:10AA60000422264B1A7000225A60FFF73BFE039B1C
:10AA7000990706D50222214B1A7000225A60FFF76F
:10AA800031FE039B9A0606D506221C4B1A701F4AFC
:10AA90005A60FFF727FE039B5B067FF512AF1C4B46
:10AAA0001A78164B32B108221A7000225A60FFF74A
:10AAB00019FE06E70922F7E7F8110020ADA4000807
:10AAC00078CC0108E5A300081812002099A400081A
:10AAD000FC13002031A500087DA50008B9A50008D9
:10AAE000F5A400087FCB010895CB0108B3CB010882
:10AAF000DBCB0108F2CB010885E5010848120020F4
:10AB000008CC01083ECC01080414002045120020A6
:10AB1000441200203C12002000140020F4130020F6
:10AB200054120020044B10B55B6998470446FFF7A8
:10AB30005BFE204610BD00BF78CC0108F0B5724C1A
:10AB4000064625460F460FCE0FC596E80F0085E84E
:10AB50000F0097E8030063696C4E013B033388BF25
:10AB60006B4B85B088BF6361636886E80300013B77
:10AB7000033307D96748636998474FF430716648D3
:10AB8000FBF724FD2368013B033307D9634863695E
:10AB900098474FF431716048FBF718FDA368013BFB
:10ABA000033307D95E48636998474FF432715A48B6
:10ABB000FBF70CFDE368013B033307D95948636990
:10ABC00098474FF433715448FBF700FD2369013B6C
:10ABD000033307D95448636998474FF434714E489A
:10ABE000FBF7F4FCE369013B033304D94FF43571FF
:10ABF0004948FBF7EBFCA369013B033304D94FF44D
:10AC000036714548FBF7E2FC484B0FCB8DE80F004F
:10AC100094E80F0000F0E0F823689847FFF7E4FDA0
:10AC2000434B42205B6C98472228014663693FD121
:10AC30004048984703220021012001F0DDFD3E4BF2
:10AC40001860012001F0A0FE3C4B186020B94FF4C1
:10AC50003D713148FBF7BAFC03220021012001F0CD
:10AC6000CBFD374D286020B94FF43E712A48FBF7E1
:10AC7000ADFC002328681A46194601F0E1FD20B911
:10AC800040F2F9212448FBF7A1FC4FF0FF3128687E
:10AC900001F0C2FF00220C21032001F0ADFD294B81
:10ACA000186078B963692848984740F2FF2103E0AB
:10ACB0002648984740F2EA211748FBF787FC002016
:10ACC00005B0F0BD224B234A1A6033680BB9042348
:10ACD0003360214B1D680DB10120F1E7019333680A
:10ACE000FA2200931D4901231D4802F069FC012846
:10ACF000F2D063691B489847074840F21131FBF7CF
:10AD000065FC2846DCE700BF181200203C1200203A
:10AD1000DFA30008B6C9010885E50108F7C90108E5
:10AD20002ECA010866CA01089FCA0108281200201D
:10AD300078CC0108DBCA0108FC130020F8130020BE
:10AD400000140020F41300200DCB0108F2CA010802
:10AD500038120020D9A300080814002041CB0108B4
:10AD600079A8000849CB010870B5084C054622684F
:10AD70000E4622B940F221310548FBF727FC236833
:10AD800031462846BDE87040184700BF3812002001
:10AD900085E5010800F03AB80120704708B5FFF7D3
:10ADA0002DFC4379002B0CBF8020002008BD000043
:10ADB000002310B5074951F83340DA00844203D824
:10ADC0000A449468844203D80133152BF3D1FEE77B
:10ADD000107910BDE8CC010884B030B503AC84E82C
:10ADE0000F00064C03AD0FCD0FC495E80F0084E8AB
:10ADF0000F00BDE8304004B0704700BF3817002096
:10AE0000014B1878704700BF201F0020C82307B5EA
:10AE10000093002304481A460321006803F0FCFC59
:10AE200003B05DF804FB00BF1014002013B5104CF4
:10AE30000120A368984700230093009BB3F5CC7FC3
:10AE40000FDDA36800209847002342F6FE720193AD
:10AE5000019B934208DD0220A36802B0BDE81040C8
:10AE60001847009B0133E7E7019B01330193EFE7AC
:10AE7000381700202DE9F04107460C4C0D46E368D9
:10AE8000002016469847236947F080009847013D07
:10AE90002E44B54204D1E3680120BDE8F0411847D3
:10AEA000236915F8010F9847F3E700BF3817002012
:10AEB00007B502AB03F8011D01221946FFF7DAFFBF
:10AEC00003B05DF804FB0000134A10B55060134A4C
:10AED000904219D00CF000FA0DA3D3E900230CF036
:10AEE0009FFB0CF00DFD0446C4F307410620FFF75D
:10AEF000DFFFC4F307210720FFF7DAFFE1B20820E4
:10AF0000BDE81040FFF7D4BF054CEDE7AFF300807C
:10AF10000000000080844E40201F0020F01FCB3333
:10AF2000CD3CD9002DE9F04107460C4C0D46E368B5
:10AF3000002016469847236907F07F009847013D97
:10AF40002E44B54204D1E3680120BDE8F041184722
:10AF500023690020984705F8010FF2E73817002011
:10AF600007B501220DF10701FFF7DCFF9DF807008F
:10AF700003B05DF804FB000001282DE9F84F0D46F1
:10AF800003D0022854D000204BE06D4E2720B48B14
:10AF9000FFF7E6FFA4B220F0F800013420440CF0E3
:10AFA0009BF9B37F0022002B3DD1664B0CF058F883
:10AFB000804630208946FFF7D3FF30F0F9030CBFFD
:10AFC0000023604B0022404649460CF049F8804679
:10AFD000284689460CF090F902460B464046494601
:10AFE0000CF03EF896F820300022F3B900230CF064
:10AFF00037F80022544B0CF0E9F9B66904463046A4
:10B000000D460CF069F902460B46204629460CF025
:10B0100007FB00224D4B0CF0D9F90BF0CDFF0CF0E3
:10B020006FFCBDE8F88F0023C0E74FF08043DEE7F8
:10B03000434C226C022A79D8454B03EBC203D3E977
:10B0400000670120636C98400CF056F902460B46ED
:10B05000304639460CF0E4FA02460B4600203949E6
:10B060000CF0DEFA06460F46B4F84A000CF044F93C
:10B070000022384B0BF0F4FF32463B460CF0A6F9A9
:10B080008B46616C824694F84E0094F84C308900EF
:10B09000002BC1F11C0101EB001114BF1420002092
:10B0A00001EBC501081A0CF017F98046606C94F8A2
:10B0B00048308946002B14BF02230023C3EB8000D5
:10B0C0000CF00AF902460B46404649460CF0A8FA35
:10B0D0000BF066FE8046894694F8490004300CF077
:10B0E0000BF942464B460CF071F90022002304464E
:10B0F0000D460CF0FBFBE0B10022134B2046294625
:10B100000BF0AEFF32463B460CF060F952465B4610
:10B110000BF0A6FF00220D4B0CF058F906A3D3E963
:10B1200000230BF09DFF0BF0C3FE78E700260027FD
:10B1300087E700200449E5E72B8716D9CEF7EF3FD4
:10B14000201F00200000F03F0000204000408F4002
:10B15000D0CC010800001140012808B504D0022815
:10B160000AD04FF0FF3006E01120FFF7F9FEC0F3E0
:10B170004700404200B208BD1B20FFF7F1FE8B38AC
:10B18000F8E700000B4B10B55B68044660B902207D
:10B1900098470120FFF7E4FE00F0F8012143012069
:10B1A000BDE81040FFF784BE03280CBF012000203B
:10B1B000EEE700BF3817002013B5C82400230B4862
:10B1C00000941A460321006803F026FB0023084878
:10B1D00000941A460321006803F01EFB0020FFF7CD
:10B1E000D1FF0022034B1A7002B010BD10140020D2
:10B1F00034170020201F002013B5C82400230B485B
:10B2000000941A460321006803F006FB0023084857
:10B2100000941A460321006803F0FEFA0120FFF7AC
:10B22000B1FF0022034B1A7002B010BD10140020B1
:10B2300034170020201F002073B55D4C064663784C
:10B24000DBB2012B03D0022B65D0002538E0402073
:10B2500094F82250FFF784FE0C214020FFF728FECF
:10B260004120FFF77DFE60F00E01C9B24120FFF7DB
:10B270001FFE3520FFF774FE00F0C00141F02001F1
:10B280003520FFF715FE3520FFF76AFE00F03F007E
:10B29000112184F83A003F20FFF70AFE00230D2019
:10B2A00084F82C3084F82D302387E386FFF758FE8E
:10B2B00000F04001EDB241F02E010D20FFF7F8FD46
:10B2C0004FF4C87200213B480DF09FFA0123237010
:10B2D000394B18684FF0FF33002E5BD04FF47A7172
:10B2E00001FB06F20093B2FBF1F20023042103F00C
:10B2F00093FA6378012B52D10520FFF743FF0D200D
:10B30000FFF72EFE40F020010D20C9B202B0BDE8CB
:10B310007040FFF7CDBD94F8513033201BB3FFF7D9
:10B320001FFE40F04101C9B23320FFF7C1FD1921D2
:10B330003B20FFF7BDFD94F8525094F84F30EDB22A
:10B34000E3B11D211120FFF7B3FD4020FFF708FEF8
:10B3500000F033014020FFF7ABFD00210F20FFF785
:10B36000A7FD0021A9E7FFF7FBFD00F0BE0141F0BA
:10B3700001013320FFF79CFD1D21D9E70F2111208A
:10B38000FFF796FD4020FFF7EBFD00F03C0141F098
:10B390000101DFE70093324633460321A7E72DB1D1
:10B3A000052002B0BDE87040FFF7ECBE0620F8E7CC
:10B3B000201F0020141400201014002037B54FF473
:10B3C0007A72642350432B4DB0FBF2F200930421B8
:10B3D0000023286803F020FA0022274B274C1A701C
:10B3E0006378DBB2012B14D0022B26D0022323700A
:10B3F0002C6802F027FB052302460093012100235D
:10B40000204603F009FA032003B0BDE83040FFF7FF
:10B41000B9BE14214020FFF74BFDB0214120FFF7BA
:10B4200047FD8F213520FFF743FD3520FFF798FDBD
:10B4300000F03F0084F83A00D8E794F84F3073B139
:10B44000F5211120FFF734FD4020FFF789FD00F0C2
:10B45000330141F040014020FFF72AFDC6E7F72104
:10B460001120FFF725FD4020FFF77AFD00F03F0196
:10B47000EFE700BF3417002058170020201F0020DE
:10B4800010B5124C6378DBB2012B04D0022B09D02B
:10B4900040F2134101E04FF47F71BDE810400C48C9
:10B4A000FBF794B8FA211120FFF702FD4020FFF7C7
:10B4B00057FD00F0FC014020FFF7FAFC03230720B2
:10B4C0002370BDE81040FFF75DBE00BF201F0020C5
:10B4D00085E5010808B51A4B5A7882422ED058707B
:10B4E0005B780020022B13D0FFF74CFE0120FFF702
:10B4F00037FD00F07F010120FFF7DAFC002140203A
:10B50000FFF7D6FC30214120BDE80840FFF7D0BC52
:10B51000FFF738FE0120FFF723FD60F07F01C9B27D
:10B520000120FFF7C5FC00214020FFF7C1FC0021EE
:10B530004120FFF7BDFC43213120E5E708BD00BFF6
:10B54000201F00201D4B13B5186000231C4C1A4609
:10B5500000944FF47A711B4803F03CF91A4B1860C1
:10B5600020B94FF486711948FBF730F80023009496
:10B570001A464FF47A71164803F02CF9154B1860EF
:10B5800020B94FF487711148FBF720F8FFF74EFC04
:10B590000020FFF79FFF0020FFF7F4FD4FF4C87273
:10B5A00000210D480DF031F9002201210B4B83F8E9
:10B5B000282083F829101A7002B010BD0C14002046
:10B5C00085BB000898CD01083417002085E50108E7
:10B5D0009BCD01081014002014140020201F00200F
:10B5E00073B50E4614460546FFF774FF3046FFF765
:10B5F0006BFC0520FFF7C6FD00230193019BB3F50B
:10B60000CC7F0BDD2846FFF7A7FD0546FFF7D4FDED
:10B61000A542CCBF0020012002B070BD019B0133C8
:10B62000EBE773B500240220FFF754FFFF21112040
:10B63000FFF73EFC0520FFF7A5FD254626460196AF
:10B64000019BB3F5CC7F0DDD2C20FFF789FC00F0CA
:10B650000100A0400134202C45EA0005EFD1284626
:10B6600002B070BD019B01330193E9E700000000C7
:10B670002DE9F04F824687B00093109B0D46019351
:10B680009DF85C309DF85810029393469DF8643005
:10B690009DF8602003930492BDF84460BDF84840D3
:10B6A0009DF84C709DF850809DF854900591FFF7DF
:10B6B00011FFDDE90332BAF1010F06D0BAF1020F32
:10B6C000059968D007B0BDE8F08F7F4C01992561DE
:10B6D0005846C4F818B06161A77784F81F8084F8D1
:10B6E000209084F8212084F82230A6830BF0F4FD0A
:10B6F00002460B4672A1D1E900010BF091FF0CF05C
:10B70000FFF81FFA80FB4FEA1B210220FFF7D0FB56
:10B710005FFA8BF10320FFF7CBFB2846FFF748FBCE
:10B7200001461220FFF7C4FB0198FFF741FB0146D9
:10B730001320FFF7BDFB310A2520FFF7B9FBF1B25B
:10B740002620FFF7B5FBE27F2346DAB9A27FCAB114
:10B7500084F829A041463220FFF7AAFB3020FFF7EA
:10B76000FFFB002F14BF0021802100F06F0040EA92
:10B770000919302041EA0901C9B207B0BDE8F04F0C
:10B78000FFF796BB00224FF4D271504883F829206E
:10B79000FAF71CFFDEE74C489DF800C00564C0F8CE
:10B7A00044B080F849C0A0F84A6080F84C7080F836
:10B7B0004D8080F84E9080F84F109DF80810BBF136
:10B7C0000C0F80F85010824680F8512080F85230DB
:10B7D00072D8BBF1050F60D925B9ABF10B03012B72
:10B7E0005DD804E0012D5AD1BBF10C0F57D10123D4
:10B7F0008AF848301D20FFF7B3FB9AF84810009BE9
:10B8000041EA490141EA870141EAC30141EA851160
:10B81000C9B21D20FFF74CFB1E20FFF7A1FBC4F3AC
:10B82000012100F00C00014341EA0B11C9B21E20B6
:10B83000FFF73EFBE1B21F20FFF73AFB310A202061
:10B84000FFF736FBF1B22120FFF732FB1FB1414673
:10B850002220FFF72DFB9AF84F306BB14B20FFF7FA
:10B860007FFB60F07F01C9B24B20FFF721FB9AF804
:10B8700050102420FFF71CFBBBF1060F4FF03100E6
:10B880000FD1FFF76DFB00F0F80141F00501312009
:10B89000FFF70EFB0C2137206FE74FF0060B00235C
:10B8A000A6E7FFF75DFB00F0F80141F0030131204E
:10B8B000FFF7FEFA0A21EEE74FF00C0B012D8FE7A0
:10B8C0000000000080847E41201F002085E50108E3
:10B8D0002DE9F04F89B01E469DF84C300C4602937E
:10B8E0009DF85C30019205939DF8603000900693BE
:10B8F0009DF86430129D03931A9BBDF85070049319
:10B900009DF854809DF85890FFF7E4FD0920FFF75B
:10B9100027FB82465A20FFF723FB0AF07F01DFF85E
:10B9200060A28346DAF804000791FFF737FA079917
:10B930000843C0B2030600F0F00C2ED5112CCBBF8B
:10B940004BF007020BF0F8025FFA82FB42F0040BA7
:10B950000BF00701072918D1142CA8BF1424052CBB
:10B96000B8BF0524611F4CEA0101C9B20920FFF7E5
:10B970009FFA59465A20FFF79BFA009B012B13D0E0
:10B98000022B6CD009B0BDE8F08F112CA8BF112498
:10B99000022CB8BF0224A11EE5E70E2CA8BF0E247E
:10B9A00044EAE474611CDEE7019B8AF80840CAF8A7
:10B9B0000C309DF80C30CAF81060CAF81850AAF87C
:10B9C0001C708AF81E808AF820908AF82130049B27
:10B9D0000198CAF824300BF07FFC65A3D3E900235B
:10B9E0000BF01EFE0BF08CFF84B2210A0420FFF73F
:10B9F0005FFAE1B20520FFF75BFA28460BF06CFC1A
:10BA000002460B465CA1D1E900010BF009FE0BF0E8
:10BA100077FF84B2210A0220FFF74AFAE1B203203D
:10BA2000FFF746FA390A2520FFF742FAF9B2262035
:10BA3000FFF73EFA3020FFF793FAB8F1000F0CBF82
:10BA40008021002100F06F0040EA0919302041EA0E
:10BA50000901C9B209B0BDE8F04FFFF729BA484A59
:10BA60009DF8083082F83C401664556482F84930ED
:10BA70009DF81430A2F84A7082F84C8082F84F305A
:10BA80009DF818300C2D82F850309DF80C3082F85B
:10BA90004E9082F85130049B1446536562D8052DB0
:10BAA00052D926B9A5F10B02012A4ED803E0012E86
:10BAB0004BD10C2D49D1012284F8482094F84F2015
:10BAC0006AB14B20FFF74CFA60F07F01C9B24B20FE
:10BAD000FFF7EEF994F850102420FFF7E9F91D2044
:10BAE000FFF73EFA9AF84810029B41EA490141EA01
:10BAF000880141EAC30141EA8611C9B21D20FFF75E
:10BB0000D7F91E20FFF72CFA00F00F0141EA0511CA
:10BB1000C9B21E20FFF7CCF9390A2020FFF7C8F977
:10BB20002120F9B2FFF7C4F9062D4FF031000ED1F4
:10BB3000FFF716FA00F0F80141F005013120FFF798
:10BB4000B7F90C21372085E706250022B4E7FFF777
:10BB500007FA00F0F80141F003013120FFF7A8F9DE
:10BB60000A21EFE70C25012E9FE700BFAFF300800D
:10BB70000000000080844E400000000080847E4170
:10BB8000201F002010B5254C2378DBB2012B02D0FA
:10BB9000022B34D010BD6378012B29D100230B2157
:10BBA0003E2084F82C3084F82D302387E386FFF77D
:10BBB0007FF910213F20FFF77BF994F8223003F042
:10BBC000FF029BB10D20FFF7CBF940F02001C9B275
:10BBD0000D20FFF76DF9124B1B68002BDAD0DB68E4
:10BBE000002BD7D0BDE81040002018472270F2E7A4
:10BBF00094F85230002BEED0FFF7FEFAEBE700236B
:10BC000001222370074B1A70054B1B68002BC1D013
:10BC10005B68002BBED0BDE810401847201F0020F5
:10BC20000C1400205817002007B50022154B8DF882
:10BC3000072083F82C2083F82D201A87DA8683F8D2
:10BC40002E2093F8223023B903B05DF804EBFFF700
:10BC5000B3BA3F20FFF784F98DF807009DF807304D
:10BC6000DB0603D510213F20FFF722F90D20FFF757
:10BC700077F940F040010D20C9B203B05DF804EB44
:10BC8000FFF716B9201F00202DE9F04107460D4CA3
:10BC90000D46E368002016469847236907F07F00A9
:10BCA0009847013D2E44B54204D1E3680120BDE828
:10BCB000F0411847236900209847C04305F8010F59
:10BCC000F1E700BF381700200A4601460020FFF7C1
:10BCD000D1B80000F7B5554C064663780D46DBB287
:10BCE000012B04D0022B34D0002528461AE0002373
:10BCF00023878BB2E386A37F13B13220FFF7D8F8F6
:10BD00006B1E3F2B1BD884F83B500025304694F81F
:10BD10003B10FFF7D9FF94F83B30228F13449BB2BE
:10BD20002387606AFFF74AFB6378012B7BD1002DE4
:10BD300079D03F4E3F4D3378002B4DD073E02A46EB
:10BD400031463C480CF03DFD3C23012584F83B3056
:10BD5000DCE794F8513033202BB3FFF701F900F002
:10BD6000BE013320FFF7A4F819213B20FFF7A0F80C
:10BD70002946222084F85C50FFF79AF800210E2013
:10BD8000FFF796F800210D20FFF792F80120FFF74A
:10BD9000E7F830F0F80711D029463046FFF794FF56
:10BDA0000025606DBEE7FFF7DBF800F0BE0141F053
:10BDB00001013320FFF77CF81D21D6E7FFF71CFABD
:10BDC0000197019BB3F5CC7FE6DC019B0133019326
:10BDD000F7E7012001F08EFF3F20FFF7C1F883064F
:10BDE000F7D4E38E218F94F83B205B1A9342208F87
:10BDF0000BDD94F83B102844FFF766FF94F83B30C6
:10BE0000228F13449BB2238795E7E18E238F28442A
:10BE1000C91AC9B2FFF758FFE18E228F238F0B4456
:10BE20009B1A9BB2238703B0F0BD00BF201F0020E8
:10BE300058170020141400200A4601460020FFF77E
:10BE400071B80A4601460020FFF71EBF38B5054607
:10BE50000C46FFF73FFB012D02D0022D0AD038BD62
:10BE6000064B9B7F002BFAD121463220BDE838409B
:10BE7000FFF71EB821462320F8E700BF201F00204F
:10BE80007FB50022654D8DF80B202B780392DBB235
:10BE9000012B2C4604D0022B00F09E8004B070BD14
:10BEA0006B78DBB2012B34D0022BF7D1402112206A
:10BEB000FEF7FEFF1220FFF753F88DF80B009DF8F8
:10BEC0000B30574E13F0200F29D020211220FEF7FF
:10BED000EFFF95F8523003F0FF0203B92A700022F9
:10BEE0005048009203AB0821006802F095FC039BC8
:10BEF0003BB14FF080524C4B1A60BFF34F8FBFF3F2
:10BF00006F8F3368002BC9D01B69002BC6D09847B0
:10BF1000C4E740F21E514548FAF758FBBEE7192026
:10BF2000FFF71EF840B285F8580095F8583095F89C
:10BF300058501B0642BF6DB26D42C5F385054FF0E8
:10BF40001A004CBF6D42AD08FFF70AF8002D40F310
:10BF50000B13B8BF40198B389BB203441BB2A4F833
:10BF60005A301320FEF7FCFF84F85C001020FEF727
:10BF7000F7FF01460D20FEF79BFF94F85C102C485C
:10BF8000FFF75AFF94F8523003F0FF028BB92548AF
:10BF90002270009203AB0821006802F03DFC039B75
:10BFA0003BB14FF08052204B1A60BFF34F8FBFF36D
:10BFB0006F8F3368002B3FF471AF9D68002D3FF405
:10BFC0006DAF94F85C10B4F85A2094F8583012B25F
:10BFD0005BB21748A84761E71248009203AB0821FB
:10BFE000006802F019FC039B3BB14FF080520E4BEE
:10BFF0001A60BFF34F8FBFF36F8F6378022B03D1AB
:10C0000008211220FEF754FF00232370044B1B6805
:10C01000002B3FF443AF1B6877E700BF201F0020D1
:10C020000C1400201014002004ED00E085E5010848
:10C03000141400202DE9FF410025684A8DF80B50AB
:10C0400013780395DBB2012B144605D0022B00F0C8
:10C05000C28004B0BDE8F0815378DBB2012B23D05D
:10C06000022BF6D15E48009503AB2A4608210068F2
:10C0700002F0D2FB039B3BB14FF08052594B1A6048
:10C08000BFF34F8FBFF36F8F80211220FEF710FF99
:10C0900000232370544B1B68002BDAD0DB68002B85
:10C0A000D7D001209847D4E73F20FEF759FF8DF8FD
:10C0B0000B009DF80B309A06CBD59DF80B30DB06B4
:10C0C00016D5E18E4948228FFEF75EF8484E494F5B
:10C0D00094F83A30AB4205DC4748FEF755F8FFF7D5
:10C0E000A3FDB6E7715D3846FEF74EF80135EFE780
:10C0F00094F8293023B940F2D2514048FAF766FA51
:10C1000094F82830022B38D1238F394894F83A100C
:10C110001844FFF796FE238F9BB2002B48D094F86B
:10C120003A30228F13449BB22387238FE28E9A42A8
:10C130008FD82F4DE28E294631480CF042FBFF2369
:10C140002B7011236B70DD23AB70EE23EB7094F832
:10C150002E50E48EFFF768FD234B6DB21B68A4B22E
:10C16000002B3FF476AF9E68002E3FF472AF0023A1
:10C170002A4621462248B0476BE7224D0020EB6853
:10C1800098472B69002098470027DFF8648094F8CF
:10C190003A30BB4203DCEB6801209847BBE72B69D0
:10C1A0000020268F9847B6B24644F0550137EEE797
:10C1B00094F82D30002B92D094F83A100C48FEF7EA
:10C1C000D3FDE086E38EB3F5C87F88D2E38E9BB2C1
:10C1D000002B84D0A3E753783BE700BF201F00204B
:10C1E0001014002004ED00E00C1400209ECD010886
:10C1F00014140020B3CD010884E5010885E5010889
:10C20000A41500203817002010B51A4C2378DBB293
:10C21000012B02D0022B2AD010BD6178C9B20129AE
:10C2200018D00229F8D194F84F30002BF4D0122006
:10C23000FEF73EFE104B1B68002BEDD05C69002C16
:10C24000EAD01C20FEF78CFE2346BDE8104000F02B
:10C250003F00184700231120238784F82D10FEF794
:10C260007FFE4008404240B284F82E00D4E7617857
:10C27000C9B2D6E7201F00200C1400201F4B70B558
:10C280005A78022A05D11B78DBB2012B02D0032B8E
:10C2900013D070BD1220FEF763FEC306F9D510213E
:10C2A0001220FEF705FE164B1B68002BF1D0DB6950
:10C2B000002BEED0BDE8704018471220FEF750FE6C
:10C2C00010F001050E4C0DD005211220FEF7F0FDF7
:10C2D0002368002BDDD09B69002BDAD00120BDE85C
:10C2E0007040184704211220FEF7E2FD2368002B5E
:10C2F000CFD09B69002BCCD02846F0E7201F002030
:10C300000C14002006480068006880F3088862B6B4
:10C3100061B6BFF34F8FBFF36F8F00DF00BF000028
:10C3200008ED00E0002307B501930B4B1B680133B8
:10C3300003D0CA210948FAF749F94FF0500383F3B3
:10C340001188BFF36F8FBFF34F8F019B002BFCD081
:10C3500003B05DF804FB00BFBC02002085E50108C6
:10C360004FF0807340F8043C054B21F0010140F888
:10C37000081C40F80C3C40F8202C4038704700BFA7
:10C3800025C30008000000000000000000000000BD
:10C39000074B19680868B0E8F00F80F30988BFF30D
:10C3A0006F8F4FF0000080F311884EF00D0E704734
:10C3B000641700204FF0500383F31188BFF36F8F91
:10C3C000BFF34F8F084A13680133012B136009D163
:10C3D000064B1B6813F0FF0F04D040F275110448A0
:10C3E000FAF7F4B8704700BFBC02002004ED00E08B
:10C3F00085E5010810B5074C236823B94FF4BE71D9
:10C400000548FAF7E3F82368013B23600BB983F38F
:10C41000118810BDBC02002085E501080000000065
:10C42000EFF30980BFF36F8F0D4B1A6820E9F00F0F
:10C4300010602DE908404FF0500080F3118801F0A2
:10C440007FFC4FF0000080F31188BDE808401968B8
:10C450000868B0E8F00F80F30988BFF36F8F70476A
:10C460006417002008B54FF0500383F31188BFF321
:10C470006F8FBFF34F8F01F0F9FA18B14FF0805270
:10C48000024B1A60002383F3118808BD04ED00E01D
:10C490000022054B05491A600A6041F26701044A0F
:10C4A000116007221A60704710E000E018E000E019
:10C4B00014E000E013B5264B264C1A78D2B2019254
:10C4C000FF221A701B78244ADBB28DF803309DF8E6
:10C4D000033003F0500313700723002223609DF8FC
:10C4E0000310581E090629D402B123602368032BC8
:10C4F00004D04FF49B711948FAF768F82368144A7E
:10C500001B0203F4E06323600024019BDBB2137081
:10C51000134B1A6842F470021A601A6842F07042B3
:10C520001A60FFF7B5FF0F4B1C60FFF7EBFE01F041
:10C5300007FCFFF7F7FE204602B010BD9DF8033060
:10C5400001225B00DBB28DF803300346C7E700BF72
:10C5500000E400E05C1700205917002085E5010881
:10C5600020ED00E0BC02002008B5EFF305830F2B9F
:10C570000AD90D4A9B5C0D4A12789A4204D940F2BE
:10C58000A5210B48FAF722F80A4B0B4A1B681268E0
:10C5900003F4E063934206D9BDE8084040F2B521B8
:10C5A0000348FAF713B808BDF0E300E0591700207C
:10C5B00085E501080CED00E05C17002070B50D4624
:10C5C000064601F037FA0D4B0D491C6862198A4284
:10C5D00007D90C23336001F0D9FA4FF0FF3420461D
:10C5E00070BD1A60074A13685B1B1360064A136824
:10C5F0002B44136001F0CAFAF1E700BFC00200202B
:10C60000CC6F0020C40200206017002008B5EFF3B3
:10C6100005831BB1C2210348F9F7D8FFBDE80840E4
:10C6200001F008BA85E5010801F0B0BA01F002BADC
:10C6300001F0ACBA0CF086B80CF08CB800B58BB039
:10C6400068460CF07FFB034B08981B6818440BB03E
:10C650005DF804FBC4020020002070477047000012
:10C6600000487047CC1F002010B50446FFF7A2FE1B
:10C67000A46BFFF7BFFEB4FA84F0400910BD70B59B
:10C680001546026C0446866B42B905689DB9806800
:10C6900001F02AFEA5600136A66370BD6DB9406841
:10C6A0000CF08FF86368226C1344A26863609342B5
:10C6B00001D3236863600020EDE7C0680CF081F8C7
:10C6C000236CE2685B4221681A448A42E2603EBF02
:10C6D000A2689B18E360022DEDD10EB1013EEAE79E
:10C6E0003046D8E703461A6C10B4084662B1D968E0
:10C6F0009C681144A142D96028BF196810BC28BFAA
:10C70000D960D9680CF05DB810BC704770B50446AC
:10C71000FFF750FE94F8455004F124066DB2002D49
:10C7200014DCFF2384F84530FFF764FEFFF742FE78
:10C7300094F8445004F110066DB2002D12DCFF2372
:10C7400084F84430BDE87040FFF754BE636A002BA4
:10C75000E7D0304601F0F0FB08B101F089FC013D63
:10C760006DB2DCE72369002BE9D0304601F0E4FB31
:10C7700008B101F07DFC013D6DB2DEE738B50D4634
:10C78000044620B940F203111948F9F71FFFFFF7DB
:10C7900011FED4E90F314B432268D0185B1A1344C1
:10C7A000A060E3600020FF23A063626084F844304F
:10C7B00084F8453095B9236963B104F1100001F0A4
:10C7C000BBFB38B14FF080520A4B1A60BFF34F8F5A
:10C7D000BFF36F8FFFF70EFE012038BD04F110008C
:10C7E00002F05AF904F1240002F056F9F2E700BF12
:10C7F00085E5010804ED00E0F8B50D46174606464C
:10C8000020B94FF4BB710D48F9F7E0FE05FB06F0C7
:10C810005030FFF70FFF044648B155B92060C4E916
:10C820000F6501212046FFF7A9FF84F84C702046D0
:10C83000F8BD00F150030360F1E700BF85E5010892
:10C840002DE9FF47884601921E46044620B940F272
:10C85000F1214B48F9F7BAFEB8F1000F06D1236C6D
:10C8600023B140F2F2214648F9F7B0FE022E07D17B
:10C87000E36B012B04D040F2F3214148F9F7A6FE07
:10C8800001F0D0FC30B9019B23B140F2F6213C48C5
:10C89000F9F79CFE0027B946DFF8E8A0FFF78AFD0C
:10C8A000A26BE36B9A4201D3022E19D13246414664
:10C8B0002046FFF7E4FE636A1BB104F1240001F097
:10C8C0003BFB38B14FF080522E4B1A60BFF34F8FB5
:10C8D000BFF36F8FFFF78EFD012004B0BDE8F08736
:10C8E000019D1DB9FFF786FD0020F6E717B902A8E4
:10C8F00001F07CFBFFF77EFD01F09CF8FFF75AFD8D
:10C9000094F84430FF2B08BF84F8449094F84530E5
:10C91000FF2B08BF84F84590FFF76CFD01A902A822
:10C9200001F070FB28BBFFF745FDA26BE36B9A4259
:10C930000ED1FFF75FFD019904F1100001F0C2FA7A
:10C940002046FFF7E3FE01F021F948B10127A5E7F2
:10C95000FFF750FD2046FFF7D9FE01F017F9F5E784
:10C960004FF08053CAF80030BFF34F8FBFF36F8F83
:10C97000ECE72046FFF7CAFE01F008F9B4E700BF74
:10C9800085E5010804ED00E010B502460021012014
:10C99000FFF732FF044638B1002383600360C360B1
:10C9A0001A461946FFF74CFF204610BD2DE9F84303
:10C9B000894690461F46044620B940F2C3312748B5
:10C9C000F9F704FEB9F1000F06D1236C23B14FF43F
:10C9D00071712248F9F7FAFD022F07D1E36B012BA1
:10C9E00004D040F2C5311D48F9F7F0FDFFF7BCFD5A
:10C9F000EFF311864FF0500383F31188BFF36F8F6D
:10CA0000BFF34F8FA26BE36B9A4201D3022F22D167
:10CA100094F845503A466DB249462046FFF72FFE3E
:10CA20006B1C13D1636A0BB901200BE004F12400E5
:10CA300001F082FA0028F7D0B8F1000FF4D00120FD
:10CA4000C8F8000086F31188BDE8F88301356DB29F
:10CA500084F84550E8E70020F4E700BF85E50108C9
:10CA600070B50D46044620B94FF48C612048F9F7A3
:10CA7000ADFD236C23B140F264411D48F9F7A6FDDA
:10CA8000236833B9A36823B140F269411848F9F724
:10CA90009DFDFFF769FDEFF311864FF0500383F31F
:10CAA0001188BFF36F8FBFF34F8FA26BE36B93427D
:10CAB0001CD994F8453001325BB2A2635A1C10D1E4
:10CAC000636A0BB9012009E004F1240001F034FA93
:10CAD0000028F7D0002DF5D00120286086F31188BA
:10CAE00070BD01335BB284F84530EBE70020F5E719
:10CAF00085E501082DE9F04385B00F460192044613
:10CB000020B94FF4A0614248F9F760FD37B9236CB2
:10CB100023B140F204513E48F9F758FD01F082FB81
:10CB200030B9019B23B140F209513948F9F74EFD64
:10CB30000026B046DFF8DC90FFF73CFCA56BD5B1D2
:10CB400039462046013DFFF7CDFDA563236963B15A
:10CB500004F1100001F0F0F938B14FF080522D4B84
:10CB60001A60BFF34F8FBFF36F8FFFF743FC0120B5
:10CB700005B0BDE8F083019D1DB9FFF73BFC002027
:10CB8000F6E716B902A801F031FAFFF733FC00F01E
:10CB900051FFFFF70FFC94F84430FF2B08BF84F8D7
:10CBA000448094F84530FF2B08BF84F84580FFF798
:10CBB00021FC01A902A801F025FAF0B92046FFF7EF
:10CBC00053FDA0B1019904F1240001F07BF9204646
:10CBD000FFF79CFD00F0DAFF38B94FF08053C9F839
:10CBE0000030BFF34F8FBFF36F8F0126A4E72046BD
:10CBF000FFF78CFD00F0CAFFF7E72046FFF786FD40
:10CC000000F0C4FF2046FFF72FFD0028EDD0B6E767
:10CC100085E5010804ED00E02DE9FF41044601919E
:10CC200020B940F291515248F9F7D0FC236C23B15E
:10CC300040F295514E48F9F7C9FC01F0F3FA30B9CA
:10CC4000019B23B140F29A514948F9F7BFFC0025F6
:10CC50002F462E46DFF81C81FFF7ACFBA36BE3B138
:10CC6000013BA363236813B901F0DEFBA0602369D5
:10CC700063B104F1100001F05FF938B14FF0805258
:10CC80003C4B1A60BFF34F8FBFF36F8FFFF7B2FBC0
:10CC90000125284604B0BDE8F081019B4BB925B1C0
:10CCA00040F2E1513248F9F791FCFFF7A3FB002570
:10CCB000EFE717B902A801F099F9FFF79BFB00F025
:10CCC000B9FEFFF777FB94F84430FF2B08BF84F8D8
:10CCD000446094F84530FF2B08BF84F84560FFF7A7
:10CCE00089FB01A902A801F08DF940BB2046FFF79E
:10CCF000BBFCF0B123683BB9FFF75CFBA06801F017
:10CD0000A1FA0546FFF776FB019904F1240001F032
:10CD1000D9F82046FFF7FAFC00F038FF38B94FF099
:10CD20008053C8F80030BFF34F8FBFF36F8F0127D8
:10CD300092E72046FFF7EAFC00F028FFF7E72046DD
:10CD4000FFF7E4FC00F022FF2046FFF78DFC0028EF
:10CD5000EDD0002D9DD0FFF72DFB616A19B1236B3B
:10CD60001968C1F10501A06801F00AFB9DE700BF49
:10CD700085E5010804ED00E02DE9F04385B00F469C
:10CD80000192044620B94FF4CD614248F9F71EFCE8
:10CD900037B9236C23B140F26C613E48F9F716FCB9
:10CDA00001F040FA30B9019B23B140F2716139487A
:10CDB000F9F70CFC0026B046DFF8DC90FFF7FAFA32
:10CDC000A36BD3B139462046E568FFF78BFC636A55
:10CDD000E56063B104F1240001F0AEF838B14FF022
:10CDE00080522D4B1A60BFF34F8FBFF36F8FFFF749
:10CDF00001FB012005B0BDE8F083019D1DB9FFF7DF
:10CE0000F9FA0020F6E716B902A801F0EFF8FFF7EB
:10CE1000F1FA00F00FFEFFF7CDFA94F84430FF2B43
:10CE200008BF84F8448094F84530FF2B08BF84F88D
:10CE30004580FFF7DFFA01A902A801F0E3F8F0B995
:10CE40002046FFF711FCA0B1019904F1240001F084
:10CE500039F82046FFF75AFC00F098FE38B94FF039
:10CE60008053C9F80030BFF34F8FBFF36F8F012697
:10CE7000A4E72046FFF74AFC00F088FEF7E72046CB
:10CE8000FFF744FC00F082FE2046FFF7EDFB002890
:10CE9000EDD0B6E785E5010804ED00E02DE9F843A3
:10CEA00089469046054620B940F2FB612048F9F7D3
:10CEB0008DFBB9F1000F06D12B6C23B140F2FC6160
:10CEC0001B48F9F783FBFFF74FFBEFF311874FF098
:10CED000500383F31188BFF36F8FBFF34F8FAC6B99
:10CEE0001CB395F84460494676B22846FFF7FAFB32
:10CEF000013C731CAC6313D12B690BB901200BE00F
:10CF000005F1100001F018F80028F7D0B8F1000F73
:10CF1000F4D00120C8F8000087F31188BDE8F88339
:10CF2000013676B285F84460E8E72046F4E700BFB2
:10CF300085E5010810B5044620B940F28A7105481C
:10CF4000F9F744FBFFF736FAA46BFFF753FA2046D4
:10CF500010BD00BF85E5010838B5054620B940F28F
:10CF6000A4710648F9F732FBFFF724FAA86BEC6BC3
:10CF7000241AFFF73FFA204638BD00BF85E50108B7
:10CF8000002330B5064A52F8335002EBC3041DB9F2
:10CF900042F83310606030BD0133052BF3D1FAE75E
:10CFA000801F0020002310B5074A02EBC3014C6824
:10CFB000844204D1002042F83300486010BD0133A0
:10CFC000052BF2D1FAE700BF801F002010B5044600
:10CFD00020B94FF4F8610548F9F7F8FA2046FFF751
:10CFE000E1FF2046BDE81040FFF726BB85E50108BC
:10CFF00070B504460D461646FFF7DCF994F8443048
:10D00000FF2B04BF002384F8443094F84530FF2BF5
:10D0100004BF002384F84530FFF7ECF9A36B2BB96C
:10D020003246294604F1240000F066FF2046BDE8A0
:10D030007040FFF76BBB8268436800681344181A9E
:10D04000824298BF801A70472DE9F843054688460A
:10D05000174622B940F244411848F9F7B7FA6C680C
:10D06000AB681E1BBE4228BF3E46A219934204D2A3
:10D0700040F24E411148F9F7A9FAA86932464146F3
:10D0800020440BF09EFBB7420FD9AB68A7EB060913
:10D09000994504D940F256410848F9F797FA4A46AB
:10D0A00008EB0601A8690BF08CFBAB683C44A3427B
:10D0B00098BFE41A6C603846BDE8F88385E501083E
:10D0C0009A422DE9F843164628BF1E460746894670
:10D0D000904686B305688468641BB44228BF344612
:10D0E000A24204D24FF490611448F9F76FFABA687B
:10D0F0002B19934204D940F281411048F9F766FA9E
:10D10000B9692246294448460BF05BFBA6420CD97C
:10D11000B04504D240F289410848F9F757FA321B6A
:10D12000B96909EB04000BF04CFBBB683544AB421A
:10D1300098BFED1A3D603046BDE8F88385E50108EB
:10D14000012A2DE9F04104460F46164630D1042845
:10D1500003D8E8211A48F9F739FABC4203D2F02182
:10D160001748F9F733FA002F04F1250008BF01270B
:10D17000FFF760FA0546C0B100F1240801342246E9
:10D18000552140460BF041FB804504D04FF4996196
:10D190000B48F9F71BFA2422002128460BF035FB37
:10D1A000C5E90247C5F818802E772846BDE8F0810A
:10D1B00018B9EE210248F9F709FA0026CDE700BFB9
:10D1C00085E501082DE9F843044620B940F29111A4
:10D1D0001748F9F7FBF9276AFFF7ECF8206918BB45
:10D1E00063691BBBD4E90269A5693246552128460B
:10D1F00094F81C800BF009FB854204D04FF4996130
:10D200000B48F9F7E3F92046202200210BF0FDFA44
:10D21000A561C4E9026984F81C8027620124FFF734
:10D22000E9F82046BDE8F8830024F8E70446F6E76D
:10D2300085E5010810B5044620B940F2DB11064827
:10D24000F9F7C4F9A3682068626818440138801AA5
:10D25000834298BFC01A10BD85E501082DE9F04F43
:10D2600087B0044616460193894621B94FF40171EF
:10D270004248F9F7ABF924B940F205213F48F9F7E4
:10D28000A5F9237FDA0715D5371DBE4204D34FF425
:10D2900004713A48F9F79AF9019B6BB92046FFF7F8
:10D2A000C9FF05460396002D3BD10025284607B04F
:10D2B000BDE8F08F3746EFE704A800F07DFE4FF0A1
:10D2C000000ADFF8B8B0FFF775F82046FFF7B2FFA5
:10D2D0008742054622D9002001F0F6F9636923B19F
:10D2E00040F229215846F9F771F900F095FF606185
:10D2F000FFF780F800220DF1180858F8143D114688
:10D30000104601F09DF8C4F814A0414604A800F0AE
:10D3100079FE0028D7D0002DC0D0C3E7FFF76AF808
:10D32000F9E7237FDB0720D4B54294BF039503962A
:10D33000039A49462046FFF787FE05460028B4D0E9
:10D340002046FFF778FEE3689842AFD300F072FB07
:10D3500023693BB1002320691A46194601F0BAF847
:10D360000023236100F012FCA0E7BD429DD30422FC
:10D3700003A92046FFF768FEDAE700BF85E501084C
:10D380002DE9F743044617469946884621B940F2ED
:10D39000D1213348F9F71AF924B940F2D2213048A3
:10D3A000F9F714F9237F13F0010F14BF04260026A8
:10D3B000B9F1000F20D0FEF7FDFF2046FFF73BFE3E
:10D3C000864205460CD3002001F07EF9236923B183
:10D3D00040F2F5212248F9F7F9F800F01DFF20612D
:10D3E000FFF708F8AE4212D300224B461146104612
:10D3F00001F026F8002323612046FFF71CFEB0420F
:10D40000054604D80025284603B0BDE8F0837EB168
:10D410002B46324601A92046D4F80090FFF750FE73
:10D42000019BAD1B9F4236BF00271F46C4F80090EA
:10D430002B463A4641462046FFF742FE0546002865
:10D44000E0D000F0F7FA63693BB1002360691A4647
:10D45000194601F03FF80023636100F097FBD2E723
:10D4600085E50108064A13681968064B19B94FF09B
:10D47000FF321A6070471268D268D2685268F8E7C3
:10D48000681700201818002010B5044620B940F293
:10D49000F2610848F9F79AF86269074B9A4207D196
:10D4A000A06A064B984203D0B0FA80F0400910BD44
:10D4B0000020FCE785E5010838180020201800202E
:10D4C000F8B51B4B1B4E1C68054630680F460430F0
:10D4D00001F013FB334640B901203168164EC96A8A
:10D4E0003268884022EA000232606A1C07D137B1F4
:10D4F000196812480431BDE8F84001F0DBBA1A6837
:10D500006419546007D30E4A10681968BDE8F840E2
:10D51000043101F0DBBA0B4A10681968043101F0DC
:10D52000D5FA094B1A68A24288BF1C60F8BD00BF3B
:10D530006018002064170020E81700203818002029
:10D540006C170020681700201818002080B5DFF83D
:10D550006C80164F164D174E2B6863B9164B1B681F
:10D56000012BF8D94FF08053C8F80030BFF34F8F2C
:10D57000BFF36F8FEEE7FEF71DFFFB68DC68201D31
:10D5800001F0BBFA3368013B33602B68013B2B6031
:10D59000FEF730FF04F154000CF000F8206BFFF7A9
:10D5A0004BF82046FFF748F8D6E700BF4C1800209C
:10D5B000D8170020D41700207017002004ED00E0D9
:10D5C0002DE9F84F4FEA820A804650460D469946AB
:10D5D0000B9EFFF72FF80746002800F0B780BC200D
:10D5E000FFF728F80446002800F0AD80076325B94E
:10D5F0004FF458715C48F8F7E9FF5246A521206BBB
:10D600000BF003F9236BAAF1040A9A442AF0070AE3
:10D610006B1E04F134020F3513F8011F02F8011BD1
:10D62000197809B1AB42F7D10A9D4FF0000B042DD8
:10D6300028BF0425271DE562C4E9135B384684F83A
:10D6400043B001F034FAC5F1050504F1180001F00A
:10D650002EFAC4F8B4B0602259462461A561646210
:10D6600084F8B8B004F154000BF0CFF83F4B4A46B1
:10D67000A3653F4B4146E3653E4B50462366FEF7AC
:10D680006FFE206006B13460FEF794FE3A4B3B4ECD
:10D690001A68DFF8248101321A603268002A58D1F2
:10D6A00034601B68012B25D1354801F0F5F9354868
:10D6B00001F0F2F9344801F0EFF9DFF80091334856
:10D6C00001F0EAF9324D334801F0E6F9484601F03D
:10D6D000E3F9284601F0E0F92F4801F0DDF92F4881
:10D6E00001F0DAF92E4801F0D7F92E4BC3F800907B
:10D6F0002D4B1D6001252D4A2D4913680868013303
:10D700001360E26A636405FA02F3034314200B60BA
:10D710001B4B394600FB023001F0CCF9FEF76AFEE4
:10D72000D8F8003063B13368DA6AE36A9A4207D204
:10D730004FF080521F4B1A60BFF34F8FBFF36F8FB4
:10D740002846BDE8F88F3846FEF776FF4FF0FF35E4
:10D75000F6E7D8F80030002BCCD13368DA6AE36AF8
:10D760009A4298BF3460C5E785E5010878EC010866
:10D7700098EC010858EC0108D41700206417002029
:10D78000701700208417002098170020AC17002085
:10D7900000180020C0170020201800204C1800207E
:10D7A00038180020681700206C170020E4170020AC
:10D7B000E817002004ED00E034180020EC170020EA
:10D7C00070B504462A4DFEF7F5FD04B92C68261DF8
:10D7D000304601F092F960B91421E06A254B4143CB
:10D7E0005B5833B90122244982400B6823EA0203C3
:10D7F0000B60A36A1BB104F1180001F07EF91F4A07
:10D800001368013313602B68A34220D131461C48B2
:10D8100001F050F91B4A136801331360FEF7EAFD6B
:10D82000194B1B6893B12B68A3420FD1174B1B6890
:10D8300023B140F2B6411648F8F7C8FE4FF08052C7
:10D84000144B1A60BFF34F8FBFF36F8F70BD124A36
:10D8500004F154001368013B13600BF09FFE206B32
:10D86000FEF7EAFE2046FEF7E7FEFFF7FBFDD5E7F1
:10D870006417002070170020E8170020E41700202C
:10D880004C180020D817002034180020E017002082
:10D8900085E5010804ED00E0D4170020F8B5054641
:10D8A00020B940F24C511748F8F790FE164B1B6810
:10D8B000AB4220D0FEF77EFD144B6C691F68144B01
:10D8C0001E68FEF797FDBC4217D0B44215D0114B2D
:10D8D0009C4208D1AB6A83B995F8B830012B0CBFD4
:10D8E00002200320F8BD0C4B9C4208D0002C0CBF3A
:10D8F00004200120F6E70020F4E70220F2E70420EC
:10D90000F0E700BF85E501086417002068170020D4
:10D910006C170020381800204C18002070B5044601
:10D9200020B940F21C711948F8F750FE184D2B68C9
:10D93000A34229D044B3FEF73DFD2046FFF7A4FDE6
:10D94000F0B1261D304601F0D8F801231149E26AF2
:10D9500008689340034314200B600F4B314600FBD3
:10D96000023001F0A7F82B68E26ADB6A9A4207D31B
:10D970004FF08052094B1A60BFF34F8FBFF36F8F88
:10D98000BDE87040FEF736BD70BD00BF85E50108FB
:10D9900064170020E81700207017002004ED00E055
:10D9A00013B500241A4B00940193502223461949C1
:10D9B0001948FFF705FE01281DD100F0E5FE0128FA
:10D9C00019D14FF0500383F31188BFF36F8FBFF36A
:10D9D0004F8F124B124A1B68543313604FF0FF32C3
:10D9E000104B1A60104B1860104B1C6002B0BDE861
:10D9F0001040FEF75FBD013007D140F604010C482E
:10DA000002B0BDE81040F8F7E1BD02B010BD00BFA4
:10DA100014180020B9CD01084DD500086417002066
:10DA2000300500201818002034180020601800204D
:10DA300085E50108024A136801331360704700BF8F
:10DA4000E0170020014B1868704700BF60180020E5
:10DA500008B5FEF789FD014B186808BD6018002065
:10DA6000014B1868704700BFD41700202DE9F84F0C
:10DA70003A4B1B68002B6AD1394B1C6801341C607F
:10DA80009CB9384D2B681B6823B140F6622136489B
:10DA9000F8F79CFD354B2A68196829601A60344AEA
:10DAA000136801331360FFF7DDFC324D4FF0000BBC
:10DAB0002B68314FA34211D93A68304BD16A1422F6
:10DAC0004A439A58022A28BF4FF0010B2C4A126889
:10DAD000002A0CBF58460120BDE8F88FDFF884A06B
:10DAE000DFF8A490DAF8002012681AB94FF0FF327C
:10DAF0002A60E1E7DAF80020D268D66871688C42C3
:10DB000001D22960D8E706F10408404600F0F5FF8D
:10DB1000B16A19B106F1180000F0EFFF01224FF0D1
:10DB2000140CF06AD9F8003002FA00F11943134BD3
:10DB3000C9F800100CFB0030414600F0BBFF38680C
:10DB4000F16AC26A914228BF4FF0010BCAE70D4A41
:10DB50004FF0000B136801331360B7E7E0170020A4
:10DB6000601800206817002085E501086C17002068
:10DB70001C180020181800206417002070170020BF
:10DB800064180020DC170020E81700202DE9F84376
:10DB90002E4C236823B940F668012D48F8F716FD8E
:10DBA000FEF708FC2368013B236024682CB10024A5
:10DBB000FEF720FC2046BDE8F883264B1B68002BAF
:10DBC000F5D0254D254EDFF8A8801FE0EB68012732
:10DBD000DC6804F1040904F1180000F08EFF4846E7
:10DBE00000F08BFF1420E26A316807FA02F30B435E
:10DBF00000FB02804946336000F05CFF184BE26A8C
:10DC00001B68DB6A9A4201D3164B1F602B68002BFE
:10DC1000DCD10CB1FFF726FC134D2C6844B1012771
:10DC2000104EFFF723FF00B13760013CF9D12C60A3
:10DC30000C4B1B68002BBAD04FF080520B4B1A6074
:10DC4000BFF34F8FBFF36F8F0124B1E7E0170020C0
:10DC500085E50108D417002020180020E8170020CF
:10DC60006417002064180020DC17002004ED00E099
:10DC70007017002038B50C46054620B940F2CA415D
:10DC80001848F8F7A3FC24B940F2CB411548F8F73F
:10DC90009DFC154B1B6823B140F2CC411148F8F7AD
:10DCA00095FCFFF7C7FE114B2A68186814192CBFA2
:10DCB0000121002182422C600CD961B9FFF766FF77
:10DCC00038B94FF080520A4B1A60BFF34F8FBFF341
:10DCD0006F8F38BD09B9A042F0D20021201AFFF79A
:10DCE000EFFBEBE785E50108E01700206018002056
:10DCF00004ED00E010B5044640B94FF080520D4BE2
:10DD00001A60BFF34F8FBFF36F8F10BD0A4B1B68B4
:10DD100023B14FF4A4610948F8F758FCFFF78AFED5
:10DD200000212046FFF7CCFBFFF730FF0028E4D0AE
:10DD3000EBE700BF04ED00E0E017002085E50108F7
:10DD4000244B70B51A68244B12B101221A6070BDC1
:10DD5000224E1A6033681B6B1A68B2F1A53F0BD1D3
:10DD60005A68B2F1A53F07D19A68B2F1A53F03D135
:10DD7000DB68B3F1A53F04D0306831683431F8F77F
:10DD8000F5FB174B1C68B4FA84F41423E4B2C4F115
:10DD90001F046343134DEB5823B940F688311248F2
:10DDA000F8F714FC142202FB04F3E918486808335E
:10DDB00040682B44984202FB045408BF4368486003
:10DDC00008BF4B606368094ADB68336033685433CB
:10DDD0001360BCE7E01700206418002064170020DF
:10DDE000E81700207017002085E5010830050020A5
:10DDF00070B504462A4EFEF7DDFA04B93468251DD5
:10DE0000284600F07AFE60B91421E06A254B4143B0
:10DE10005B5833B90122244982400B6823EA02038C
:10DE20000B60A36A1BB104F1180000F066FE2946DE
:10DE30001E4800F03FFE94F8B8301D4D012B04BF82
:10DE4000002384F8B830FEF7D5FA2A682AB1FEF725
:10DE5000B1FAFFF707FBFEF7CDFA3368A34211D101
:10DE60002B6883B1134B1B6823B14FF4D96112485F
:10DE7000F8F7ACFB4FF08052104B1A60BFF34F8F96
:10DE8000BFF36F8F70BD094A11680D4A1268914245
:10DE900001D13360F6E7BDE87040FFF751BF00BF26
:10DEA0006417002070170020E817002038180020A1
:10DEB00034180020E017002085E5010804ED00E09B
:10DEC000D417002038B50D46044620B940F69F31DE
:10DED0000748F8F77BFB074B20461968183100F01C
:10DEE000F5FD2846BDE838400121FFF7E9BA00BF3B
:10DEF00085E501086417002070B50E4614460546F6
:10DF000020B940F6CA310A48F8F760FB094B2846A9
:10DF10001968183100F0CEFD002C214608BF3046AC
:10DF2000BDE8704018BF4FF0FF30FFF7C9BA00BF1F
:10DF300085E501086417002038B5C368DC6824B99A
:10DF400040F6FA311548F8F741FB04F11805284668
:10DF500000F0D3FD124B1B68E3B9251D284600F0E5
:10DF6000CCFD01230F49E26A086893400343142063
:10DF70000B6029460C4B00FB023000F09BFD0B4B65
:10DF8000E26A1B68DB6A9A4285BF0120084B0020C9
:10DF9000186038BD29460748EFE700BF85E501084E
:10DFA000E0170020E81700207017002064170020F9
:10DFB000641800202018002010B5044620B940F64F
:10DFC0004F410748F8F702FBFEF7F4F9054B1B68D1
:10DFD0002360054B1B686360BDE81040FEF70ABA7A
:10DFE00085E501081C18002060180020034B1B6801
:10DFF0000360034B1B684360704700BF1C18002080
:10E000006018002070B50C46054620B940F6654101
:10E010001448F8F7DBFA24B940F666411148F8F7DE
:10E02000D5FAFEF7C7F9104B1A682368591C0FD0B0
:10E030000E482E6800686968864201D091420ED968
:10E04000521A934209D99B1A23602846FFF7CEFF44
:10E050000024FEF7CFF9204670BD00232360012481
:10E06000F7E700BF85E50108601800201C180020B4
:10E070000122014B1A6070476418002070B50C46ED
:10E080001646054608B91B4A156805F13402626058
:10E09000EA6A052B22612A6B2560E2616A6CA26044
:10E0A000EA6C62614FF00002A2611BD0114909685D
:10E0B000A9420BD12273D6B1296B0A46531A12F822
:10E0C000010BA528FAD09B08238470BD032B237372
:10E0D000F1D1FFF7AFFCAB6A0BB102232373FFF75B
:10E0E00055FDE8E72846FFF7D9FB2073E3E72684D0
:10E0F000EBE700BF641700202DE9F84F0D6881465B
:10E100000C4692461DB300254FF0240B4B6801F1DD
:10E1100008075B68BB424B6004BFCB684B604B6831
:10E12000D3F80C8063680BFB05915B6801229F426A
:10E13000636008BFE36805F1010508BF63606368B9
:10E14000DE6853463046FFF799FFB045EAD12846CE
:10E15000BDE8F88F2DE9F84305461746FFF76AFC3E
:10E160001F4B1B688B4238D84FF0000824264446CA
:10E17000DFF8809009EB080106FB04500122FFF74D
:10E18000BBFFA8F1140818F1640F0444F2D1154B39
:10E190000222196806FB0450FFF7AEFF124B04443D
:10E1A0001968022206FB0450FFF7A6FF044404226C
:10E1B0000E4906FB0450FFF79FFF044406FB045082
:10E1C00003220B49FFF798FF04440FB100233B6083
:10E1D000FFF7DCFC2046BDE8F8830024F8E700BF29
:10E1E000D4170020681700206C1700204C1800205E
:10E1F00038180020C017002008B9064B1868026BB9
:10E200001346981A13F8011BA529FAD0C0F38F0002
:10E21000704700BF64170020014B1868704700BFAB
:10E2200064170020054B1B6833B1054B1B68002B9E
:10E230000CBF0220002070470120704734180020D6
:10E24000E01700202DE9F0410446002836D0234A8B
:10E25000C36A11681746C96A8B4237D2142682698D
:10E260001F4D002AA8BF3A6806FB0353A2BFD26A1B
:10E27000C2F10502826142699A4221D100F104088B
:10E28000404600F03AFC174B48B9E06A4643AA59A9
:10E290002AB901211A68814022EA01021A603A680B
:10E2A0001968D26AE262012404FA02F00843186095
:10E2B0001420414600FB025000F0FCFB204603E026
:10E2C0003B68DB6AC3620120BDE8F0811368C06C63
:10E2D000DC6AA0422CBF00200120F5E76417002073
:10E2E00070170020E8170020F8B5044608B9002090
:10E2F000F8BD1F4B1B68834204D040F67A711D485D
:10E30000F8F764F9236D23B940F67B711948F8F7E3
:10E310005DF9236DE16AE26C013B91422365E6D031
:10E32000002BE4D1251D284600F0E7FB124E134ACE
:10E3300050B91421E76A794373582BB90120136847
:10E34000B84023EA00031360E36CC3F10501A16147
:10E35000E3620124116804FA03F0084310601420FA
:10E36000294600FB036000F0A5FB2046C0E700BF84
:10E370006417002085E5010870170020E8170020C9
:10E38000F8B50D460446002845D0036D23B940F684
:10E39000C9712148F8F71AF9E36C9D4238BF1D4650
:10E3A000E36AAB4237D0236D012B34D11B4B1B6882
:10E3B000A34204D140F6E4711748F8F707F9142690
:10E3C000A269E36A002AE562A4BFC5F10505A5615B
:10E3D000134D626906FB03539A421CD1271D384630
:10E3E00000F08BFBE26A0F4C40B95643AB592BB996
:10E3F00001212368914023EA0103236001231420B3
:10E40000216893400B432360394600FB0250BDE86E
:10E41000F84000F04FBBF8BD85E501086417002007
:10E4200070170020E8170020044B1A681AB1196809
:10E430000A6D01320A651868704700BF6417002032
:10E440002DE9F041214C1E4680460F461546FDF74A
:10E45000B1FF236893F8B830022B16D0012123684E
:10E46000D3F8B42022EA0802C3F8B420236883F862
:10E47000B81056B13046FFF723F84FF08052144BD6
:10E480001A60BFF34F8FBFF36F8FFDF7B3FFFDF738
:10E4900091FF1DB12368D3F8B4302B6023680022AC
:10E4A00093F8B830022B09BF012500252368D3F863
:10E4B000B41004BFB943C3F8B410236883F8B8207C
:10E4C000FDF798FF2846BDE8F08100BF64170020E3
:10E4D00004ED00E0F8B50E4617461D46044620B987
:10E4E00041F219212E48F8F771F8FDF763FF15B1D5
:10E4F000D4F8B4302B60022394F8B85084F8B830C4
:10E50000EDB2042F1AD8DFE807F00E030906150054
:10E51000D4F8B4301E43C4F8B46004E0D4F8B43086
:10E520000133C4F8B430012D12D00124FDF762FF8D
:10E530002046F8BD022DEED10024F7E7D4F8B43020
:10E540000133F0D041F24A211548F8F73FF8EAE7E5
:10E55000261D304600F0D1FA1420124AE36A1168F1
:10E560009D400D431560104A314600FB032000F02A
:10E57000A1FAA36A23B141F259210948F8F726F814
:10E580000A4BE26A1B68DB6A9A42CED94FF080528E
:10E59000074B1A60BFF34F8FBFF36F8FC5E700BF04
:10E5A00085E50108E8170020701700206417002097
:10E5B00004ED00E02DE9F843DDF820800E46914699
:10E5C0001D46044620B941F28C213848F7F7FEFF7A
:10E5D000FDF7CAFFEFF311874FF0500383F3118863
:10E5E000BFF36F8FBFF34F8F15B1D4F8B4302B60EA
:10E5F000022394F8B85084F8B830EDB2B9F1040FA2
:10E600001AD8DFE809F00E0309061500D4F8B43073
:10E610001E43C4F8B46004E0D4F8B4300133C4F845
:10E62000B430012D12D0012087F31188BDE8F883A2
:10E63000022DEED10020F7E7D4F8B4300133F0D04A
:10E6400041F2CF211948F7F7C1FFEAE7A36A23B1E6
:10E6500041F2DA211548F7F7B9FF154B1B6803BBE8
:10E66000251D284600F049FA01231249E26A08688C
:10E670009340034314200B6029460F4B00FB0230EC
:10E6800000F018FA0D4BE26A1B68DB6A9A42CAD99D
:10E690000123B8F1000F01D0C8F80030084A136018
:10E6A000C1E704F118010748EAE700BF85E5010862
:10E6B000E0170020E81700207017002064170020E2
:10E6C000641800202018002038B5054608B9084B0A
:10E6D0001D680024FDF76EFE95F8B830022B04BFCC
:10E6E00085F8B8400124FDF785FE204638BD00BFFF
:10E6F00064170020F8B50F4CFDF75CFE2568ADB936
:10E700000D4F0E4E384600F0C7F9304600F0C4F900
:10E710000B4B2A461F600B4B0C210A201E60FEF794
:10E720006BF8206010B10849FEF72AFCBDE8F840FC
:10E73000FDF760BE9C18002070180020841800208F
:10E74000681800206C180020BECD0108914208B561
:10E75000416000610AD8D21A83699A420DD2084BEF
:10E76000011D186800F0B2F9002008BD9A4201D2DC
:10E77000994202D2011D034BF3E70120F5E700BFE8
:10E780006C1800206818002007B5FFF7B3FF0C4B8A
:10E790001B6843B90B484FF48971F7F717FF002046
:10E7A00003B05DF804FB084BC8220193012307491D
:10E7B000009307480023FEF703FF0028EAD0EFE7A5
:10E7C0009C18002085E50108A0180020C3CD010891
:10E7D000EDE800082DE9F04180462C200D46174653
:10E7E0001E46FDF727FF044688B125B94FF4B671E0
:10E7F0000848F7F7EBFEFFF77DFF069BC4F80080A3
:10E80000C4E9065726626362201D00F050F92046D5
:10E81000BDE8F08185E501082DE9FF410D469046F0
:10E820001F46064620B94FF4C3710F48F7F7CEFED6
:10E830000E4C206878B1052DCDE9015803960DDC0A
:10E84000FFF7F0FC002302280CBF0A9A1A4601A920
:10E850002068FDF7F5FF04B0BDE8F08100233A46DB
:10E8600001A9FEF7A3F8F6E785E501089C1800204A
:10E870002DE9F74300271A4DDFF86C802B681A68E2
:10E8800032B9184A11681360296003B0BDE8F083FB
:10E89000DB68DC681E6804F10409484600F02DF9C5
:10E8A000636A20469847E369012BE7D1A3693344A3
:10E8B0009E4206D2636024614946286800F006F94A
:10E8C000DCE700230097324619462046FFF7A4FFF5
:10E8D0000028D3D140F272314046F7F777FECDE7FA
:10E8E000681800206C18002085E501082DE9F04F1C
:10E8F0004FF00108624D89B0DFF898B1DBF80020D5
:10E90000136843B30024D368D3F80090FFF792F85C
:10E91000FFF798F85B4B82461A681F4690425A4EA2
:10E920001CD31860002C4CD0584B1B681A68B2FAE4
:10E9300082F25209A9EB0A013068FEF759FBFFF792
:10E9400025F998B94FF08052514B1A60BFF34F8FA1
:10E95000BFF36F8F0AE001249946D7E70393FFF7CF
:10E9600087FF039BC3F800A0FFF710F9002205A959
:10E970003068FEF7BFF80028BED0059B002BF5DB02
:10E98000079C636913B1201D00F0B7F8FFF75AF830
:10E990003B688146984201D2FFF76AFF059BC7F8A2
:10E9A0000090092BE2D808FA03F313F4047A57D144
:10E9B00013F0C70F33D19B06D8D52046FDF73CFE98
:10E9C000D4E7814529D8FFF7E1F8DBF80030DB68B0
:10E9D000D3F80CB00BF1040000F08FF8DBF81C301A
:10E9E000012B15D1DBF818104B46524649445846C6
:10E9F000FFF7ACFE60B1009423464A4621465846D4
:10EA0000FFF70AFF20B94FF4F4712846F7F7DEFD4F
:10EA1000DBF8243058469847A8E722468AE7A169E0
:10EA2000069B4A4619442046FFF790FE00289DD0D9
:10EA3000636A20469847E369012B97D1A26906993A
:10EA4000CDF800A00A44534651462046FFF7E4FEA5
:10EA500000288BD140F201312846F7F7B7FD85E752
:10EA6000069BA36123B94FF446712846F7F7AEFD24
:10EA7000A1694B464A4649442046FFF767FE75E7C1
:10EA800085E50108981800209C1800206C180020CB
:10EA900004ED00E0681800204FF0FF3200F1080399
:10EAA0004360C0E902230361002303607047002331
:10EAB0000361704743689A684B608A609A68516046
:10EAC0009960036808610133036070470A6830B5D4
:10EAD000531C0AD103695A684A6091608B6059607F
:10EAE000036808610133036030BD00F108035C680E
:10EAF00025689542EFD82346F9E70369D0E901126A
:10EB00008A60826851605968814208BF5A60002259
:10EB100002611A68013A1A6018687047021C18BF2F
:10EB2000012200210148F8F745BB00BF0004024064
:10EB3000F8F7A0BF38B505460C460020FFF7EEFFFA
:10EB400045F08000FFF7F4FF2046FFF7F1FFBDE836
:10EB500038400120FFF7E2BF08B50120F8F71CF9A3
:10EB60000A20F8F719F90B20F8F716F90720F8F73B
:10EB700013F90520F8F710F9BDE808400420F8F76C
:10EB80000BB90000204B70B59D780446EDB958B91B
:10EB900002211E48F8F708FB23461A460221BDE869
:10EBA00070401A48F8F738BA012805D102211748F1
:10EBB000F8F7F4FA2B46F0E7022823D10246014683
:10EBC000BDE870401148F8F765BA012D14D138B985
:10EBD00004210E48F8F7E8FA002304211A46DEE77C
:10EBE000012804D104210948F8F7D8FAF4E70228EB
:10EBF00008D102460421E3E76A21BDE870400448D9
:10EC0000F7F7E4BC70BD00BFA4180020000002406C
:10EC100085E5010808B50020FFF7B4FFF7F7FEFF10
:10EC20000120FFF7AFFFF7F7F9FF0220FFF7AAFF78
:10EC3000BDE80840F7F7F2BF08B500210120F8F75A
:10EC40009BFE0120FFF76AFF0023094819461A4678
:10EC5000F8F7E2F9B5214020FFF76CFFA021412031
:10EC6000FFF768FFBDE8084000210120FFF762BF01
:10EC70000004024010B5FFF76FFF0120FFF74EFFC1
:10EC800000233A481A461946394CF8F7C5F90021CD
:10EC90000120F8F771FE22787AB1002306211A4686
:10ECA0003248F8F7B9F906213048F8F777FAF7F75C
:10ECB000B5FF19215820FFF73DFFFFF7ABFFFFF726
:10ECC000BBFF63785BB1002304211A462948F8F79B
:10ECD000A3F900230D211A462748F8F79DF90022D1
:10ECE00001212248F8F7D6F900220A211F48F8F737
:10ECF000D1F900220B211D48F8F7CCF90022072199
:10ED00001A48F8F7C7F9002205211848F8F7C2F9A0
:10ED1000002204211548F8F7BDF90523022201213C
:10ED20001248F8F757F8052302220A210F48F8F78E
:10ED300051F8052302220B210C48F8F74BF8052364
:10ED4000022207210948F8F745F80523022219464F
:10ED50000648F8F73FF8094B1B782BB9BDE810407F
:10ED6000BE210748F7F732BC10BD00BF00040240C7
:10ED7000A41800200000024000080240A71800204C
:10ED800085E5010882B0019002AB33F8041D054A05
:10ED90009B78118093700122034B1A7002B0FFF729
:10EDA00069BF00BFA4180020A71800201A4B10B597
:10EDB0005B78D3B10128194C18D104211848F8F711
:10EDC000EDF90D211748F8F7EFF923786BB100231F
:10EDD00004211A461248F8F71FF900230D211A469C
:10EDE0001048F8F719F90023237010BD40B9042129
:10EDF0000B48F8F7D9F90D210A48F8F7CFF9E4E7FD
:10EE0000022204210648F8F745F902220D2105489F
:10EE1000F8F740F90123E7E7A4180020C802002012
:10EE2000000002400008024008B5FFF795FEFFF71A
:10EE3000F1FEFFF701FFF8F7F9FD012200211F485D
:10EE4000F8F728F90220FFF7B1FF0220FFF79AFE3A
:10EE5000022201211948F8F71DF902220A21174858
:10EE6000F8F718F902220B211448F8F713F90222D7
:10EE700007211248F8F70EF9022205210F48F8F78A
:10EE800009F9022204210D48F8F704F90C4B1B780C
:10EE90001BB9E2210B48F7F799FB0B4B1B785BB1D1
:10EEA000002306211A460548F8F7B6F8BDE80840E1
:10EEB00006210248F8F778B908BD00BF00040240F7
:10EEC000A718002085E50108A418002010B5064CFD
:10EED000022220460021F8F7DDF82046BDE8104068
:10EEE00002220121F8F7D6B800140240F8B50F4C01
:10EEF000D4F880329847234610F5617641F1000737
:10EF000004F52072D3E90845A04271EB050401DA4B
:10EF1000C3E90801D3E90645A64277EB050401DA07
:10EF2000C3E9066728339342ECD1F8BDB01800203E
:10EF300010B5044618B9BB210748F7F747FB074B44
:10EF4000D3F880329847D4E90623904271EB03044A
:10EF5000B4BF101A002010BD85E50108B0180020CC
:10EF60002DE9F84F064628B9BDE8F84FDC213448B2
:10EF7000F7F72CBB0023334A1C469246D118097A76
:10EF80002833B14208BF0134B3F5207FF6D1002CFD
:10EF900054D0062E03D940212948F7F717FB2A4BF6
:10EFA00053F83650002D47D1E7212548F7F70EFBDF
:10EFB0004FF0000B65430AEB0B04227AB24235D1C5
:10EFC0006268002A32D02269012A03D1D0211C486C
:10EFD000F7F7FCFAD4E9062319461343104624D068
:10EFE000D4E90889B0EB080061EB090108F0C8FD1D
:10EFF00007462069013808F0A9FD0146384608F0A7
:10F00000B1FE0746284608F0A1FD394608F0F6FD96
:10F01000394608F0E9FC08F0DDFF18EB000249F181
:10F02000000310461946C4E9060125610BF1280BBF
:10F03000BBF5207FBFD101E0012DB9D1BDE8F88F2C
:10F0400085E50108B0180020CCCD01084FF47A7393
:10F05000B0FBF3F341F65832A3F55223A3F618336D
:10F0600093422DD81B4B1C4A0344934228D91B4B77
:10F070001B4A0344934223D94CF24E32194B0344AA
:10F0800093421DD9184B98421CD903F5371303F549
:10F09000D863984218D903F5122303F5F863984210
:10F0A00014D903F5122303F5F863984210D903F538
:10F0B000DB2303F5BA63984294BF0520062070470E
:10F0C00000207047012070470220704703207047DE
:10F0D000042070473F373ACC9E8601007F0F31CC29
:10F0E0003E0D0300AF312ACC40DA8E332DE9F043D8
:10F0F00085B0E0B1D0E903984FF47A740D4B4168C4
:10F10000D3F88C62037AB1FBF4F4062B96BF0A4A5B
:10F110000A4D52F823500778FFF70AFFCDF8008018
:10F12000CDE901903B462A4621460548B04705B047
:10F13000BDE8F083B018002004CE010824CF0108F8
:10F1400031CF010870B5134C054694F894320E4641
:10F1500023B94FF496711048F7F738FA25B940F201
:10F160002D110D48F7F732FA26B94FF497710A4876
:10F17000F7F72CFA0023282202FB03F0215CA942B6
:10F1800003D120444168B14203D00133102BF3D1A5
:10F19000002070BDB018002085E501082DE9F04F72
:10F1A0002E4F9A4697F8943293B00191934623B923
:10F1B00040F241112A48F7F709FA0025FFF796FEB9
:10F1C000A9464FF0FF382C46282303FB0576019A09
:10F1D000F368934218DBBBF1000F10D13046FFF704
:10F1E000A7FE80B3404536D30ED1D4E90823D6E933
:10F1F0000801FAF7D4FE002818BF344604E00021C5
:10F200003046D8470028E9D10135102DDCD1BAF1BC
:10F21000000F01D0CAF80080B8F1000F0FD1B9F18A
:10F22000010F0CD909F1FF314046FBF7B6F812ABDC
:10F2300003EB8000282350F8404C03FB0474204665
:10F2400013B0BDE8F08F12AB03EB890343F8405CC9
:10F2500009F10109C6E780463446D5E7B018002019
:10F2600085E50108000000002DE9F14F0D46044638
:10F2700020B94FF4C2712048F7F7A8F9236923B9E0
:10F2800040F285111C48F7F7A1F9DFF87490D9F81E
:10F29000803298478B4682462069C4E908AB08F063
:10F2A00055FC294608F0AAFC294608F09DFB08F009
:10F2B00035F80FA3D3E9002308F0B2F907F070FD89
:10F2C00008F01EFB1AEB00064BF100078046C4E96C
:10F2D0000667284608F058FED9F88C520246434685
:10F2E000AC466168054801B0BDE8F04F604700BF1B
:10F2F0000000000080842E4185E5010820CE010831
:10F30000B01800202DE9F0410E461746054620B9F9
:10F310004FF4C8711348F7F759F926B940F2911123
:10F320001048F7F753F90021384608F023FE20B9BA
:10F330004FF4C9710B48F7F749F90024DFF828802A
:10F3400014F80830AB4207D108EB04004368B3421D
:10F3500002D13946FFF788FF2834B4F5207FEFD17A
:10F36000BDE8F08185E50108B018002008B5FFF779
:10F370006DFE003018BF012008BD00002DE9F047E8
:10F380003F4F94B097F8943206460D4623B94FF498
:10F39000D9713C48F7F71AF92846FFF7E7FF04460A
:10F3A00058B94FF47A713848D7F89032B5FBF1F17B
:10F3B0009847204614B0BDE8F08729463046FFF74D
:10F3C000C1FE0028F6D18046282303FB0879D9F82E
:10F3D00004202AB108F10108B8F1100FF5D1E9E7CE
:10F3E00097F894321BB977212648F7F7EFF81EB942
:10F3F00078212448F7F7EAF8282200210DEB0200D3
:10F4000009F003FA2846FFF721FE062804468DF886
:10F41000300003D940211B48F7F7D8F80B956D460B
:10F420004FF0280A194B8DF8286003EBC40252688C
:10F4300053F834300AACCDE90D230FCC0FC50FCCF7
:10F440000AFB087A0FC594E803006E46544685E827
:10F4500003000FCE0FC40FCE0FC495E80300D7F8FA
:10F460008C3284E803004146094898474846FFF734
:10F470003DFE9AF80800FFF773FD48469AE700BF83
:10F48000B018002085E50108D4CE0108CCCD0108D4
:10F4900003CF01080D4B10B593F89432044623B9FD
:10F4A0004FF4EA710A48F7F791F86CB163685BB101
:10F4B0000848FAF725FE2046FFF718FE0023207AB9
:10F4C00063602372FFF74CFD002010BDB0180020D0
:10F4D00085E5010894CF01082DE9F041124D07465A
:10F4E00095F89432884623B94FF4F6710F48F7F730
:10F4F0006DF827B940F2ED110C48F7F767F80024D2
:10F5000026462B5DBB4208D128194368434504D1E8
:10F51000FFF7C0FF002818BF06462834B4F5207F47
:10F52000EFD13046BDE8F081B018002085E5010834
:10F5300070B5114C064694F8943223B94FF4FE711D
:10F540000E48F7F743F826B940F2FD110B48F7F7DC
:10F550003DF80025635DB34204D1601943680BB1E7
:10F56000FFF798FF2835B5F5207FF3D1D4F88C321A
:10F570000348BDE870401847B018002085E5010831
:10F5800078CF01082DE9F843154D06460F46904601
:10F590000024A946635DB34209D12B195A6832B1E0
:10F5A000002398450DDC09EB0400FFF773FF2834B6
:10F5B000B4F5207FEED10024A04508DC0120BDE891
:10F5C000F88357F823108A42F1D00133E9E757F85E
:10F5D00024103046FFF7D2FE0028F0D00134EBE7CC
:10F5E000B0180020014B93F894027047B018002027
:10F5F00010B5074C2378FA2B04D94FF40D71054848
:10F60000F6F7E4FF20780130C0B2207010BD00BFD3
:10F61000A818002085E5010884B070B504AC84E822
:10F620000F001C4B93F894121C4631B1BDE870409A
:10F63000D3F89032184804B018474FF42672184691
:10F6400004F5207504AE09F0E0F80FCE0FC533685D
:10F650002B6013B9114BC4F89032D4F88C3213B923
:10F660000E4BC4F88C32D4F8883213B1D4F88432FB
:10F670004BB9D4F88C320A4898470A4BC4F8883200
:10F68000094BC4F88432012384F89432BDE87040F9
:10F6900004B07047B018002060CE0108F9A000083F
:10F6A00099CE010855870108458701082DE93008E2
:10F6B0000F4B03F52072D3E908BC5BEA0C0405D0BC
:10F6C0001BEB00044CEB0105C3E90845D3E906BC7C
:10F6D0005BEA0C0405D01BEB00044CEB0105C3E90D
:10F6E000064528339342E6D1BDE83008FFF7FEBB5C
:10F6F000B018002070B50446044E451814F8011BDC
:10F700003046FAF7FDFCAC42F8D170BD0EDB0108C3
:10F7100070B515460022C0E901150270C0E9033238
:10F72000C0E90522C0E907224262DDE9041204466D
:10F7300000F11C0604F048FC38B929460748FAF7DE
:10F74000DFFC2B210648F6F741FFDDE904233146B3
:10F75000204604F026FC204670BD00BF89B4010895
:10F7600085E501082DE9F04100259DF81860C0E904
:10F7700001120570C0E90335C0E90555C0E9075518
:10F78000456231460446174600F11C0804F020FA91
:10F7900038B939460748FAF7B3FC20210648F6F78E
:10F7A00015FF32464146204604F000FA2046BDE8E7
:10F7B000F08100BF89B4010885E50108F8B500258E
:10F7C000C0E901120570C0E90335C0E90555C0E97B
:10F7D0000755456206990446164600F11C0704F0D9
:10F7E000F7FA38B931460748FAF78AFC202106486B
:10F7F000F6F7ECFE069A3946204604F0D3FA204686
:10F80000F8BD00BF89B4010885E5010810B50446BC
:10F81000006810B1012106F06FFC204610BD000009
:10F82000F0B50125044608270E468DB0564B574AC1
:10F830002946009502A8FFF795FF02A9204605F08A
:10F840003BFD02A8F0F752FE514BCDE900671A4686
:10F850000DEB07000421FFF75BFF0DEB07012046CE
:10F8600005F02AFD0DEB0700F0F740FEF319494AB9
:10F87000019700930DEB0700474B0421FFF748FF6A
:10F880000DEB0701204605F017FD0DEB07001027D3
:10F89000F0F72CFEF3190093404B01971A46042110
:10F8A00002A8FFF735FF02A9204605F005FD203626
:10F8B00002A8F0F71BFE3A4B3A4A00960197042142
:10F8C00002A8FFF725FF02A9204605F0F5FC02A8D3
:10F8D000F0F70CFE0C230026334A00930221334B31
:10F8E00002A8FFF76BFF02A9204605F0E5FC02A87D
:10F8F000F0F7FCFD2E4B2F4A2946009502A8FFF792
:10F9000031FF02A9204605F0D7FC02A8F0F7EEFD72
:10F91000294B2A4A0096022102A8FFF74FFF02A9AD
:10F92000204605F0C9FC02A8F0F7E0FD244B254A6B
:10F930000096022102A8FFF741FF02A9204605F028
:10F94000BBFC02A8F0F7D2FD1F4B204A29460095C8
:10F9500002A8FFF707FF02A9204605F0ADFC02A8A8
:10F96000F0F7C4FD07231A4A00930221194B02A89D
:10F97000FFF724FF02A9204605F09EFC02A8F0F73D
:10F98000B5FD0DB0F0BD00BF2FD00108ADC301081B
:10F9900042D00108E6D30108CDD3010850D00108B8
:10F9A000EED3010818D4010889C3010857D0010813
:10F9B000B0D001088CC301081FD4010890C301080E
:10F9C0005DD4010899C3010898D401085DE40108D9
:10F9D000A2C30108B4D4010870B5044690B0014632
:10F9E000924A01A805F011FA914A214604A805F0AF
:10F9F0000CFA904A214607A805F007FA8E4A2146DC
:10FA00000AA805F002FA8D49204605F0F5F90546E9
:10FA10008B48FAF775FBDDE901239B1A082B06D00A
:10FA20008848FAF76DFBB1218748F6F7CFFDDDE98D
:10FA300004239B1A082B06D08448FAF761FBB521F2
:10FA40008148F6F7C3FDDDE90A239B1A102B06D087
:10FA50007F48FAF755FBB9217B48F6F7B7FDDDE99A
:10FA600007135B1A102B0CD101234A1E01F10F0062
:10FA700012F8016F002E18BF00239042F8D1002B1E
:10FA800053D07448FAF73CFB5DB37348FAF738FB80
:10FA9000674A21460DA805F0B8F97048FAF730FB1F
:10FAA00008210198FFF726FE6D48FAF729FB082187
:10FAB0000D98FFF71FFE6B48FAF722FB10210A98FA
:10FAC000FFF718FE6848FAF71BFB0D980A9A019990
:10FAD00000F0AEFE0DA8FFF799FE6448FAF710FBA0
:10FAE00061E06348FAF70CFB6248FAF709FB0A99F0
:10FAF000019800F0FFFD6048FAF702FB042101982D
:10FB00000844FFF7F7FD5D48FAF7FAFA10215C4860
:10FB1000FFF7F0FD5B48FAF7F3FA10215A48FFF7B8
:10FB2000E9FD5148FAF7ECFAD7E710220A9808F0F5
:10FB300039FE5649444B002818BF19465448FAF775
:10FB4000DFFA002D40D04448FAF7DAFA384A214665
:10FB50000DA805F05AF94F48FAF7D2FA0821019892
:10FB6000FFF7C8FD4C48FAF7CBFA08210D98FFF7CC
:10FB7000C1FD4A48FAF7C4FA10210798FFF7BAFD09
:10FB80004748FAF7BDFA10210A98FFF7B3FD364847
:10FB9000FAF7B6FA0D98079B0A9A019900F05EFEF3
:10FBA0000DA8FFF733FE3048FAF7AAFA0AA8FFF7C4
:10FBB0002DFE07A8FFF72AFE04A8FFF727FE01A8DD
:10FBC000FFF724FE10B070BD2948FAF799FA3548BE
:10FBD000FAF796FA079A0A99019800F0CDFD26489F
:10FBE000FAF78EFA042101980844FFF783FD2E48A6
:10FBF000FAF786FA10212248FFF77CFD2B48FAF726
:10FC00007FFA10212A48FFF775FD2A48FAF778FA9B
:10FC100010212948FFF76EFD2848FAF771FA1A48B3
:10FC20001021FFF767FD104858E700BF42D00108D8
:10FC3000E6D3010818D4010850D00108ADC301086B
:10FC4000E2D00108F9D0010885E5010809D10108D1
:10FC50001AD101082AD1010845D101084BD1010868
:10FC60005CD101086ED1010884E5010816D20108B3
:10FC70008ED1010893D10108C5D10108D7D101085F
:10FC80006C04002003D201089C040020CBD00108A2
:10FC900035D2010852D2010864D2010877D2010896
:10FCA00097D20108E2D201081CD3010888D30108C9
:10FCB0007C0400209FD301088C040020B6D30108E7
:10FCC00010B5084CD4F834221AB95A210648F6F770
:10FCD0007DFCD4F834020023BDE81040032220212B
:10FCE000FEF7F8BBD002002085E50108F0B51F46FD
:10FCF0001446C7B005460E46F122002109A808F0B7
:10FD000084FD09AA1021384603F00AF8204609F0BC
:10FD100083FD07461022002101A808F076FD102F70
:10FD20003A46214628BF102201A808F04AFD09AA38
:10FD300005A901A803F06EF8324605A9284608F087
:10FD400040FD47B0F0BD000037B50E4C0E4D94F8A5
:10FD50002F30022B12D194F8213094F8F321009324
:10FD6000D4F8F4110823012002F08CFF6B6B002003
:10FD70009847042384F82D3003B030BDEB6A9847D0
:10FD80000123F7E7D002002078CC0108044B5A7F0A
:10FD900022B993F8330080F00100704700207047CB
:10FDA000D0020020F0B570279DB006460D463A46B9
:10FDB0000021684608F029FD08212B460DEB0100C3
:10FDC00004AC0B4AFFF792FF2B462046094A10214C
:10FDD00008ADFFF78BFF94E80F0085E80F003A4667
:10FDE0006946304608F0EDFC30461DB0F0BD00BF5E
:10FDF0000BD6010813D6010808B50548FAF780F9B3
:10FE0000044A92F8F831013382F8F83108BD00BF96
:10FE1000BDD50108D00200200022024B83F8F82152
:10FE2000704700BFD002002084B070B58AB00EAC1D
:10FE300084E80F00734C4FF41072254600212046D1
:10FE40000EAE08F0E2FC0FCE0FC596E8030014AB2F
:10FE500085E803000FCB04F1180585E80F000E9B21
:10FE60000BB9694B23600F9B0BB9674B2360109B49
:10FE700023B940F285116548F6F7A8FB129B23B918
:10FE800040F289116148F6F7A1FB119B23B940F2BA
:10FE90008D115E48F6F79AFB139B23B940F291113E
:10FEA0005A48F6F793FBA3690BB90323A36101F04A
:10FEB000FBFE94F8203013B9012384F8203001F0C0
:10FEC000EBFE94F8213013B90E2384F82130636AD5
:10FED0000BB94F4B636201F0D3FEFAF747FCC4F84D
:10FEE00030020138033008D94A4863689847002037
:10FEF0000AB0BDE8704004B0704700220421012020
:10FF0000FCF77AFC0322C4F83C0200210120FCF734
:10FF100073FCC4F8380220B94FF4DD713B48F6F7A2
:10FF200055FB002204210120FCF766FCC4F83C01CB
:10FF300020B94FF4DF713548F6F748FB0022042161
:10FF40000120FCF759FCC4F8400120B940F2C1116E
:10FF50002E48F6F73BFB4FF48163A4F800320023F0
:10FF600084F83430012384F80432FFF73BFB05ADFD
:10FF700068B9A36822690593236807920893E26829
:10FF800063680692009395E80F00FFF745FBFFF7C3
:10FF90002FFB84F8320001F0C7FE23681E4E079342
:10FFA000636806F1A0020893236904960693E36848
:10FFB000F03605930AAB43F81C2D93E803008DE857
:10FFC000030095E80F0002F0E7F80196A3694FF4EB
:10FFD000CD720093114901231148FDF7F1FA012870
:10FFE00004D04FF4F3710948F6F7F0FA0023032226
:10FFF0000421D4F83402FEF76DFA012084F83100B0
:020000040801F1
:1000000076E700BFD0020020F9A0000885E50108CE
:1000100008E6D33347D50108140400207AD5010837
:10002000ED04010810B50F4CD4F8343223B940F276
:10003000EF110D48F6F7CAFA002303220421D4F881
:100040003402FEF747FA42F21071D4F83802FCF796
:10005000E3FD0023D4F838021A46BDE810401946E3
:10006000FCF7EEBBD002002085E5010838B50E4D47
:10007000D5F8383223B94FF400710C48F6F7A6FAD8
:100080000021D5F83802FCF7C7FD0128044608D145
:100090000023D5F838021A461946FCF7D1FB204652
:1000A00038BD0020FCE700BFD002002085E5010834
:1000B00010B5FFF7DBFF68B1074C0023D4F834021A
:1000C00003220821FEF706FAD4F83402BDE81040F6
:1000D000FDF724BC10BD00BFD0020020002313B5E3
:1000E00002A941F8043D4EF65E224EF66023441EFE
:1000F00094428CBF02461A46034BD3F84001FCF7EA
:10010000F9FC019802B010BDD002002038B5FFF70D
:10011000ADFF194B20B15B6818489847002038BDE7
:10012000D3F83C01FCF706FF04460028F6D101464F
:1001300002F02EF905460028F0D0047001F0B4FC5E
:10014000044618B9284602F071F9E7E70C4A13682B
:100150000133136073B913680133136063600423C0
:100160002046237001F0C4FC10B9204601F0AEFC1B
:100170006068D4E71368F1E7D002002082D5010857
:10018000481B0020F0B58BB005460C46174601937E
:10019000FFF76CFF10B100200BB0F0BD4B4ED6F84E
:1001A0003C01FCF7C7FE0028F5D1002F5CD1002CE4
:1001B000F1D12846214602F0EBF805460028EAD0A6
:1001C0009DF80530002B52D004230370FFF714FE76
:1001D0000F2206A903A80AF089FF9DF804303BB15D
:1001E0000D230AA901F8203D012203A80AF08CFF83
:1001F0009DF806303BB102230AA901F8203D0122F7
:1002000003A80AF081FF96F82E2096F82F3093422B
:1002100003D196F83030934217D02023022A18BF1A
:1002200000228DF8083095F8783002A90BBF43F012
:10023000040343F001038DF809208DF8092003A879
:1002400085F8783002220AF05FFF96F8143205999B
:1002500096F8F0011944C9B201F0ECFE844209D9C4
:10026000284602F0E3F896E7E02F94D8A1E70223AE
:100270000370ADE7059A32B1D2B20399284600F077
:10028000A5FF0028ECD06F77284601F00DFC07464B
:100290000028E5D000230E4A836013680133136001
:1002A00083B91368013313607B60022338463B70C7
:1002B00001F01EFC40B9384601F008FC736805489F
:1002C000984768E71368EFE7786865E7D002002091
:1002D000481B0020F1D50108034B93F8141293F842
:1002E000F00101F0A7BE00BFD00200200E2808BF19
:1002F0000120024BD87783F8F0017047D00200202C
:10030000024B83F8200083F8F1017047D0020020EF
:10031000014B83F821007047D002002008B5F9F79F
:10032000DBFF024BC3F8480108BD00BFD00200202C
:10033000034630B5054C00F110052246186859688F
:10034000083303C2AB421446F7D130BD8C04002001
:10035000034630B5054C00F110052246186859686F
:10036000083303C2AB421446F7D130BD7C040020F1
:10037000034630B5054C00F110052246186859684F
:10038000083303C2AB421446F7D130BD6C040020E1
:10039000034630B5054C00F110052246186859682F
:1003A000083303C2AB421446F7D130BD9C04002091
:1003B00010B50446FFF7BCFF2046FFF7C9FF2046F3
:1003C000BDE81040FFF7D4BF30B51025C3B0224CB4
:1003D000F122002105A808F018FA2A46002101A8F8
:1003E00008F013FA94F85B3105AA8DF8053094F8FB
:1003F0005A3129468DF8063094F8593104F5B67013
:100400008DF8073094F858318DF8083094F857314A
:100410008DF8093094F856318DF80A3094F855313A
:100420008DF80B3094F854318DF80C3002F078FCD4
:10043000052305AA04F5C67101A88DF8043002F061
:10044000E9FC062305AA04F5BE7101A88DF8043065
:1004500002F0E0FC43B030BDD00200200246024B67
:100460000068516803C370471C0400200246024B19
:100470000068516803C3704724040020034630B568
:10048000054C00F11005224618685968083303C26C
:10049000AB421446F7D130BD2C040020034630B5E2
:1004A000054C00F11005224618685968083303C24C
:1004B000AB421446F7D130BD3C040020014B987785
:1004C000704700BFD0020020014B83F82E00704718
:1004D000D002002038B5044600680D46884203D09B
:1004E00008B101F0F3FA256038BD00002DE9F041B4
:1004F000F9F76AFF0123764CDFF8DC81754E84F84A
:100500002D300A23744A4FF0FF310020FDF798FF89
:10051000012866D1D8F8000043071AD5337833B1E3
:10052000FAF770F80020FAF7C1F800233370FBF7F0
:1005300041FFFBF75FFF022384F82D300023D4F83E
:1005400038021A461946FCF77BF90020FDF750FCEB
:10055000D7E710F0080721D033787BB941F2883013
:10056000FAF77CF818B99B215C48F6F72FF85C483D
:10057000FAF79CF801233370FFF7E6FB0020FEF743
:10058000A3F84FF4FA61D4F83802FCF745FB0028D1
:10059000B7D1A2215148F6F719F8B2E710F02000C0
:1005A0003FD03378D3B194F82D30042B16D14D4D74
:1005B0003A462946D4F83002FCF7DEFB01280DD17B
:1005C0002B78072B2AD03A462946D4F83002FCF77C
:1005D00091FA012802D12846FAF76EF80020FEF7BA
:1005E00073F83378002B8CD001F096FA054600287A
:1005F00087D00378012B1AD194F82C10A26A01B18C
:1006000092B9B2FA82F238485209F9F779FD2846D0
:1006100001F0E4FA284601F059FA72E701F00CFA09
:10062000DCE7FEF751F86CE701F050FAA56A032306
:1006300084F82D302B78052B46D8DFE803F00345EE
:100640000A0A3A3AD5212548F5F7C0FFFFF77CFBA7
:1006500057E729462548FFF73DFFFFF797FB68B1AD
:1006600001F06CFA054618B9E1211C48F5F7AEFF18
:10067000022328462B7001F08BFAE7E701F05EFABF
:10068000074618B9E8211548F5F7A0FF394628466E
:1006900000F012F97B7E53B14FF47A70FDF72AFB1C
:1006A0003946284600F008F97B68002BF2D038461E
:1006B000E1E70E480021FFF70DFF284600F022FE7B
:1006C000284601F003FAC1E7636809489847F7E74D
:1006D000D00200204C1B00205C1B002085E5010897
:1006E000C1FC0008501B0020E3D40108F8020020E0
:1006F00023D5010830B50430C7B00D46FFF70EFE14
:100700001B4B0DF1050203F10C0153F8040B8B4256
:1007100042F8040BF9D11B880124138000238DF8C3
:100720001330022309AA102128468DF8043002F064
:10073000F7FA09AA05A901A802F06CFB05A8FFF7C2
:1007400027FE09AA102128468DF8044002F0E8FA95
:1007500009AA05A901A802F05DFB05A8FFF728FE7C
:100760001022044B5C771A7783F8442147B030BDE0
:10077000AED50108D002002030B50430C7B00C4619
:100780001546FFF7CBFD284B0DF1050203F10C01D7
:1007900053F8040B8B4242F8040BF9D11B88204616
:1007A000138000238DF813300223012409AA10219D
:1007B0008DF8043002F0B4FA09AA05A901A802F0E4
:1007C00029FB05A8FFF7E4FD09AA102128468DF8AA
:1007D000044002F0A5FA09AA05A901A802F01AFB33
:1007E00005A8FFF7A5FD032309AA05A901A88DF80F
:1007F000043002F00FFB05A8FFF7AAFD042309AAA5
:100800000DEB030005A98DF8043002F003FB05A8E9
:10081000FFF7AEFD1122054B5C771A7783F8442170
:1008200083F8FD4147B030BDAED50108D0020020AD
:1008300038B50D461446FFF711FE2846FFF716FEA1
:100840002046FFF71BFE2046FFF728FE0022024B42
:100850005A7710221A7738BDD002002070B50E46A4
:1008600015461C46FFF7FAFD3046FFF7FFFD284608
:10087000FFF704FE2046FFF711FEBDE8704000229E
:10088000024B5A7711221A77FFF79EBDD002002043
:10089000002310B54168074C1A19106C884202D128
:1008A00092F83C0020B91033B3F5807FF4D10020DA
:1008B00010BD00BFD00200202DE9F04F064689B0E0
:1008C0000C4619B918216C48F5F780FE16B133783B
:1008D000022B03D01A216848F5F778FE33691BB95B
:1008E0001B216548F5F772FE33691B78042B05D090
:1008F000022B03D01D216048F5F768FE00225F4DF2
:10090000337895F8F1716370D5F8F4313946039373
:1009100008AB43F80C2D95F83200594A95F8F0B120
:1009200095F8F2A195F8F391FEF738FC804620B9CE
:100930000123237009B0BDE8F08F059B33B101F0AE
:10094000FBFB03232370059B6360F3E7B36801336C
:10095000012BB36011D1D5F8E42130690132C5F81B
:10096000E421B5F8FE2185F82C300132A5F8FE21EE
:1009700000F0DEF8306900F049FCD5F84821336911
:100980005A60D5F8E4215A8195F8F92142B1002244
:1009900085F8F9211A7A42F004021A72B5F8FA21A0
:1009A000A3F87A20404601F0E5F9034695F8F021D6
:1009B00005EB001130694FF0000880F87D3080F8B9
:1009C0007C2095F804224FF47A7312F00F0208BFCE
:1009D00001225A4307AB019306AB00933C3102F569
:1009E0007A73CDF8188000F0F7FE0028A0D0FDF74C
:1009F00029F8F060D4F8A00084F8008008B101F074
:100A000015FD069B0798C4F8A030C4F80A002246DA
:100A100031461C4800F05EF88022316904F1200064
:100A200007F0CFFE0021039B0798636195F83330F0
:100A3000C4F80A00C4F8881084F810B0677484F809
:100A400012A084F8139021702376B26895F80232D0
:100A5000D4F8A0009A4200D258B1617685F82C10E3
:100A6000003018BF0120617E00900748F9F748FB6D
:100A700060E701216176F3E785E50108D0020020F7
:100A800091080108F80200201AD6010808B5104A9A
:100A900010B10023A2F8FE31937FBBB1B2F8FE3152
:100AA00092F800128B4211D95B1A92F8011293FB53
:100AB000F1F201FB12334BB901F0FEF830B901F04D
:100AC00009F918B9BDE8084001F014B908BD00BF24
:100AD000D002002070B5D2F8A04006461546E4B119
:100AE0000021204601F088FBFFF796F92378204685
:100AF000052B01BF012386F8D1316389A6F8D231D5
:100B0000FFF7C4FFD5F80A10204600F0B5FB237AA2
:100B10005B0701D501232B7270BD2046FFF7B6FF9E
:100B2000D5F80A102046BDE8704000F0A5BB0000D3
:100B3000134B10B49A7F02B3027A93F8F01142F08B
:100B400001020272DA7F914208D193F83C40A4B1CD
:100B500093F84C408CB193F85C4074B1B3F8FE410B
:100B600093F800329C4208D9914206D0037A10BC17
:100B700043F002030372FFF73FB910BC704700BF98
:100B8000D0020020431EDBB21F2B96BF0D4A00236C
:100B9000D35C0A280BD8012202FA00F010F4A46FEB
:100BA00005D0094A92F814221A440E2A07DC074A93
:100BB000107818440E28CCBF002001207047002078
:100BC000704700BF57D60108D00200206F1B0020DD
:100BD00070B5057804462846FFF7D4FF88B1094A66
:100BE000094E1378F5540133137051B1074A247834
:100BF00092F81432D01880F805420846013382F882
:100C0000143270BD6F1B0020601B0020D00200203A
:100C10002DE9F04F002593B0CDE907019DF87080D4
:100C2000B74E0992059345450AD2059B595D5F1958
:100C30000846FFF7A7FF029028B9B248F9F760FA13
:100C400013B0BDE8F08F01391F2900F2A682DFE85A
:100C500011F02000A4022C0054027D016101C401A6
:100C600042025402EB01A40256022C016D026F02F3
:100C7000A402A402A402A402A402A402A402A40244
:100C8000A402A402A402A402A402A402A402A40234
:100C90009102A8EB0503DBB2012B4FF0000400F03A
:100CA000028186F8FD410224FDE0A8EB0503DBB2DA
:100CB000039307238DF8383000231C460193039AD1
:100CC000231D934202DA3B5D032B10D0019B2BB115
:100CD0009DF838306FF300038DF838309DF83830C8
:100CE000072B40F0D2800024DFF81C92C6E03B19AD
:100CF000D3F8012005345FFA82FB0BF00F034FEAB3
:100D00001B1B0693BBF1060FC2F30F23E4B24FF097
:100D100000090F92049303D902F0F003F02B2FD1B6
:100D20004FF6FF73C2F30762049902F07002602A63
:100D300008BF194600230A469A4611465FFA8AF010
:100D40000B930A9201F088F8DDE90A2380B106EBE3
:100D50000A11096C61B106EB0A1191F844104FEACF
:100D6000111C01F00F01594502D8E34598BF034615
:100D70000AF1010ABAF1100FDFD10BB14FF00209ED
:100D8000069B072B05D99DF83C3003F00F030F2B72
:100D900001D149F004099DF83FA00AF0700ABAF1A8
:100DA000600F0CD149F00109BAF1000F0FD0DDE955
:100DB0000132BAF1600F18BF1346019307E0BAF190
:100DC000000FF4D1049801F025F80028EAD19DF82D
:100DD0003830C9F3400269F3000362F34103C9F3F9
:100DE000800969F382038DF8383068E73B19D3F83E
:100DF00001A09DF83830053403F00703072BCDF828
:100E000040A0E4B23AD19DF84030C3F30311CAB216
:100E100086F8F0110AF00F010F290BD021B901213A
:100E200061F303038DF840309DF84030C3F30303B2
:100E300086F8F1319DF84310CAF30F20C1F3021177
:100E400001F010F820B940F275114846F5F7BEFBE5
:100E500096F84431102B09D11AF0706F01BF0122AE
:100E60009DF8433062F303038DF843309DF843301F
:100E70001A0703D0C3F3030386F80232039A231D33
:100E80009A4202DD3B5D032BB0D054B1032312A87C
:100E9000002100F8083DFFF79BFE00210EA8FFF798
:100EA00097FE01F049F92C444AE0A8EB0503DBB2B8
:100EB000052B40F27081781CF9F715FA97F9053087
:100EC0000021002B22DB0CA3D3E9002312184B4195
:100ED000002196F8040210EB020941EB030A099B7A
:100EE000022B03D119F101094AF1000A079BC3E95A
:100EF0001C9A0624D7E700BF6E3DD5120000000003
:100F0000D002002077D6010885E50108A8A3D3E91F
:100F10000023DBE7062312A800F8103D0021FFF7AD
:100F200057FE089B12AC03F01F0304F8083D002194
:100F30009B48FFF74DFE20460021FFF749FE6C1C41
:100F4000E4B2A5423FF47CAE25466CE6A8EB05036F
:100F5000DBB2042B4FF00004A5D9D7F801308DF88F
:100F600034401093DBB2C3F30212052A9CBF86F80B
:100F7000F221E2B2C3F303039CBF42F004028DF8F6
:100F80003420062B9CBF86F8F3319DF834300DF1E8
:100F900041009CBF43F002038DF834306424F9F71C
:100FA000A4F944432046FEF7E1F99DF8343088B1B6
:100FB000C6F8F44143F00103052412A800F8104DCF
:100FC00001218DF83430FFF703FE01210DA8FFF752
:100FD000FFFD68E760F30003EEE7A8EB0503DBB273
:100FE000052B40F2D88057F8010F3B7910900DF196
:100FF00041008DF8443000F0B3FE9DF844200146D6
:101000009DF8400000F0CAFE8DF8340001F094F81D
:10101000072312A800F8103D0021FFF7D9FD002199
:101020000DA8FFF7D5FD64E7A8EB0503DBB2042BA1
:101030004FF000047FF637AFD7F801300DF14100D3
:1010400010938DF8344000F08BFE044602469DF864
:1010500040105448F9F754F82046FEF787F928B1B4
:101060009DF8343043F001038DF834309DF8403062
:101070000F2B2ED801331B0103F12C02334493F8BC
:101080002C10324439B11B6B2BB19DF8343043F036
:1010900002038DF834309DF8343012A803F00303B6
:1010A000032B4FF00A0308BFD46000F8103D012164
:1010B000FFF78EFD01210DA8FFF78AFD9DF8341082
:1010C0003948C1F3400201F00101F9F719F805248C
:1010D000E9E60022DFE7A8EB0503DBB2012B5AD0DB
:1010E0007B78012103F00F0386F80432082312A84D
:1010F00000F8083DFFF76CFDD5E5AC1C20E7A8EB38
:101100000503DBB2012B46D001237A7812A811091E
:1011100002F00F0203FA01F1934086F801320C232A
:1011200086F8001200F8083D0021E3E7EC1C07E711
:10113000A8EB0503DBB2012B2DD0B3687C78984770
:1011400001221A4B8DF83820C3E9000123090A3324
:1011500002FA03F3C6F820320F2312A8002104F08C
:101160000F0400F8083DC6F82442FFF731FD0021C6
:101170000EA8BFE7A8EB0503DBB2012B0BD07B78F1
:101180000BB1022B07D196F830209A423FF48BAD79
:1011900086F8303087E5002485E62C46D1E600BF8E
:1011A000D3040020AED60108CDD60108E804002003
:1011B0006F3DD5120000000038B10078032803D03D
:1011C000431F58425841704701207047037A70B559
:1011D0001B09D61804460F2E00F10C0015461844C2
:1011E00009DC07F0EEFA0120237A05EB131565F30D
:1011F0000713237270BDC3F10F0207F0E2FA237ADE
:10120000002043F0F0032372F4E7000073B5134DA0
:1012100006462A78124CBAB11249FFF7D7FF0F22BF
:101220000021104807F0F1FA00232B7094F8FD31EB
:1012300043B140F2011302A921F8043D02223046D5
:10124000FFF7C4FF02B070BD94F81422002AEDD05D
:1012500004F20521FFF7BAFFE8E700BF6F1B00208B
:10126000D0020020601B0020024B00F00F0083F82A
:1012700004027047D0020020F0B585B00391044607
:1012800010B3FFF799FFF8B10020144B9DF90E1031
:1012900083F8050283F81402207A93F81EC09DF8A3
:1012A0000F200609677F257FBCF1000F05D010F0E5
:1012B000010018BF012083F8FC013EB1009604F143
:1012C0000C032046FFF7A4FC05B0F0BD002FFBD1B6
:1012D000002DF9D00095A36EF3E700BFD0020020E7
:1012E000002310B54168064C1A19106C884202D1CF
:1012F00092F83C0018B91033302BF5D1002010BD06
:10130000D00200202DE9F04F054689B018B10378CE
:10131000043B012B03D91E21BB48F5F757F92B6974
:101320000BB11B781BB11F21B748F5F74FF9B74C2C
:1013300094F8F33194F8F1810393D4F8F43194F8EC
:10134000F0B1029394F8F2A100F0A6FC00F0ACFC1E
:10135000002208AB43F80C2D4146AD4A94F8320008
:10136000FDF71CFF28B9284600F038FC09B0BDE89D
:10137000F08F00F0FFFC059B07469BB100F0DCFE00
:1013800000F0DCFB044618B93B219F48F5F71EF935
:101390002B782046637003232370059B636000F065
:1013A000F7FBE3E7AB68227F0133102AAB602ED155
:1013B000012B09D1D4F8E4310133C4F8E431954B61
:1013C0005B699847A4F8DC01B4F8DC310133A4F878
:1013D000DC31002607AB94F8F39184F8F3610193B4
:1013E00006AB009304EB071141F2707341F28832AF
:1013F0003C312869069600F0EFF9B0B9284600F0B4
:10140000EDFB069801F012F884F8F391AEE7112A8B
:1014100006D1636904F5A6709847A4F8DC01D8E703
:101420004E217948F5F7D2F8D3E7069A84F8F3917C
:1014300012B11378012B06D0284600F0CFFB069896
:1014400000F0F4FF92E7237F102B40F098801023E8
:10145000002684F84431069BDA6803F16307C4F878
:10146000482103F15302002E00F098801121DFF88B
:10147000B4C184F84411664610685168083203C646
:10148000BA42B446F7D1644F03F1230203F1330C9F
:101490003E4610685168083203C662453746F7D1A8
:1014A0005E4F03F1330203F1430C3E46106851686E
:1014B000083203C662453746F7D1594F03F143025C
:1014C00003F1530C3E4610685168083203C662456A
:1014D0003746F7D19A68A2631A7CC2F3030284F8F4
:1014E000F3211A7CC2F3021284F8F221587CFFF730
:1014F000BBFE002394F82E20069812F0FD0F00F199
:10150000120018BF84F82E30C4F8EC31C4F8E8316A
:10151000C4F8E43184F82F3084F8303000F0E4FC73
:1015200000F00AFE012384F8333000F007FB064682
:1015300018B9CA213448F5F749F88022296906F11B
:10154000200007F03EF90023069A0798C6F8A0206D
:1015500094F83320C6F8883032769DF80C2033702A
:10156000F2742B78029AC6F80A0086F810B086F852
:10157000118086F812A07261737030460FE7112B4C
:1015800007D192F82260002E3FF461AF84F8443115
:1015900061E77C211C48F5F719F85CE71021DFF8BA
:1015A00084C084F84411664610685168083203C646
:1015B000BA42B446F7D1184F03F1230203F1330CBA
:1015C0003E4610685168083203C662453746F7D177
:1015D000124F03F1230203F1330C3E4610685168A9
:1015E000083203C662453746F7D10D4F03F1230297
:1015F00003F1330C3E4610685168083203C6624559
:101600003746F7D166E700BF85E50108D002002024
:10161000E112010878CC01088C0400207C04002031
:101620006C0400209C0400202DE9F04385B007469F
:101630000C468DF80F202BB101220DF10F01002077
:10164000F9F718FCFCF7FEF91D4B1E4D1E4E9DF8D8
:101650000F1080469B6A2046984741F288322946FF
:10166000D6F83002FBF746FA40B32B78012B20D195
:101670002846AC68F9F720F84FF47A70A4EB080913
:1016800009FB000006F062FA7968024696F832001B
:10169000FDF738FE00F050FDCDE900499DF80F1030
:1016A000356843467A680948A847204605B0BDE832
:1016B000F0832846F9F700F80024F6E70446F4E73B
:1016C00078CC0108701B0020D002002012D801083D
:1016D0002DE9F84F394E9846736B054689461446F6
:1016E0004FF47A7A9847DFF8DCB0354F0AFB05F201
:1016F00002F59C328032B2FBFAF23249D7F830025E
:10170000FBF7F8F920B9336B98474FF0FF302FE023
:101710009BF80030072B07D15846F8F7CDFF4FF460
:101720007A65F9F737FBE1E7032B366B22D1DBF85B
:10173000045028792968844228BF04464846224636
:1017400007F03FF83F6895F90830B5F90620A988F9
:101750001D48B847B8F1000F05D0EB88A8F8003055
:101760002B7A88F802301748F8F7A6FFB0472046D2
:10177000BDE8F88F042B0BD11248F8F79DFFB04756
:101780003C68FCF75FF901461048A0470020EFE7EE
:10179000052B09D10B48F8F78FFFB0473C68FCF7E1
:1017A00051F901460A48F0E7F2210A48F4F70EFF22
:1017B0000448F8F781FFB047A7E700BF78CC0108DD
:1017C000D00200207C1B0020BAD70108E4D7010812
:1017D000FCD7010885E501082DE9F04F904CC9B010
:1017E0000F4691469846FF2294F8443108A902908A
:1017F000539E00F033FE824618B9002049B0BDE880
:10180000F08F94F8F01194F8F2517A688D4298BFF5
:101810004D1B084694BFEDB20025D4F800B00592E8
:10182000049100F0B3FB039094F8F10100F0C4FBC5
:10183000DDE90412039B00907A48D847FA682846ED
:10184000D4F800B0039200F0A1FB039A03462946A6
:101850007548D84794F8F311D4F8F4210846D4F821
:1018600000B00492039100F091FBDDE903120346FE
:101870006E48D8472368424649466D48984701213B
:10188000029800F0B9FC94F8211094F8F13194F822
:10189000F02100917968002001F0F4F9524600230C
:1018A00008A93846FFF7C0FE82460028A5D0029B53
:1018B0005B4C93F8783013F0050F0AD013F0040F47
:1018C0000CBF0023022394F82F209A4218BF84F8FB
:1018D0002F30FF22002108A806F097FF94F821304E
:1018E0002A460093F9680823012001F0CBF9A9F1F9
:1018F000140005F0F1FC46A3D3E9002305F066FDD2
:1019000005F0FEFF074609F2AB2005F0E5FC42A317
:10191000D3E9002305F05AFD05F0F2FF0546A8F1D2
:10192000140005F0D9FC3AA3D3E9002305F04EFDDD
:1019300005F0E6FFA0F1140BAB4594BFC7EB0B0B12
:10194000C7EB050B4FF47A7505FB07F18146B1FB38
:10195000F5F107A8CDF81CA0FCF78CF9FF2233465F
:1019600008A95846FFF7B4FE421C07463FF445AFAE
:1019700000281ADD2468FCF765F85346024639460C
:101980002C48A0470EB10123F3700023529A9F42C6
:10199000136008DD224BF9B293F8442108A801F046
:1019A00003F9529B1860012028E794F8213094F83D
:1019B000F3210093D4F8F4110823012001F062F917
:1019C00005FB09F107A8B1FBF5F1CDF81CA0FCF768
:1019D00051F908F2AB2005F07FFC0FA3D3E90023F7
:1019E00005F0F4FC05F08CFF3346FF2208A9A0EBBC
:1019F0000900FFF76DFE431C07463FF4FEAE0028CA
:101A0000C3DD002EC1D00223BEE700BFAFF30080CC
:101A10000AD7A3703D0AEF3FA4703D0AD7A3F03F59
:101A2000D0020020F6D6010828D701084ED70108B9
:101A300074D701088FD7010830B5C3B06B46FF22B9
:101A400002A94FF47A60FFF743FE051E24DD002350
:101A5000144C0193D4F8482194F84431E9B202A817
:101A600000F044FE03460190B0B10278052A01D08F
:101A7000032A14D11846002100F0BEFB0198FFF79D
:101A800005F8DDE90010FFF7F7FB0023012201A9AB
:101A9000D4F83C02FAF7D4FE284643B030BD00F03B
:101AA000C5FCF9E7D002002038B5074B0546DB68D6
:101AB00014209847044620B11022002106F0A5FE0C
:101AC0002561204638BD00BFD002002010B5044675
:101AD00050B1006900F0AAFC00232361034B2046AB
:101AE000BDE810401B69184710BD00BFD0020020A0
:101AF000002307B502A941F8040D06481A46D0F89C
:101B00003C01FAF79DFE431E5842584103B05DF870
:101B100004FB00BFD0020020002307B50193064B51
:101B200093F8342022B901A9D3F83C01FAF7E2FF77
:101B3000019803B05DF804FBD0020020064B10B5FD
:101B4000DB68A8209847044618B1A822002106F0B7
:101B50005CFE204610BD00BFD002002010B5044638
:101B600098B1D0F8883013B1203000F049FCD4F897
:101B7000A00020B100F05AFC0023C4F8A030034BB1
:101B80002046BDE810401B69184710BDD002002058
:101B90001FB5104C0190D4F84001FBF7DDF9024667
:101BA00040B903A9D4F84001FAF7A4FF10B1039893
:101BB000FFF7D4FF002301A91A46D4F84001FAF731
:101BC0003FFE20B940F275110348F4F7FFFC04B062
:101BD00010BD00BFD002002085E5010838B50546DC
:101BE000FFF7ACFF044620B94FF4BD710548F4F788
:101BF000EDFC012323702B7820466370BDE838404C
